:020000040000FA
:107800005469616E59696E673130300000000000C4
:1078100054593230302E303830303030625F747925
:10782000424154333247313339474B3634464200B4
:1078300043414E5F5354440000000000000000002C
:1078400043414E5F43485F300000000000000000ED
:1078500043414E5F3530304B6270730000000000D2
:10786000E8070000E0070000DF070000000000005C
:020000040000FA
:1080000058330020DD800000E5800000E78000009C
:108010000000000000000000000000000000000060
:10802000000000000000000000000000EF800000E1
:108030000000000000000000F380000029C30100E0
:1080400081130100C5130100F5130100251401007F
:108050005514010085140100B5140100E514010058
:108060001515010045150100791501008D15010058
:108070009D150100D1150100E1150100F115010068
:108080002516010069160100B1160100F91601005C
:10809000411701008917010099170100CD17010050
:1080A000011801003118010065180100991801003C
:1080B000A9180100B9180100ED18010021190100EB
:1080C000EF3FE8FF0448854600F02CFA00480047DF
:1080D0007D070200C046C04658330020164880473E
:1080E00016480047FEE7FEE7FEE7FEE7FEE7FEE78D
:1080F000FEE7FEE7FEE7FEE7FEE7FEE7FEE7FEE758
:10810000FEE7FEE7FEE7FEE7FEE7FEE7FEE7FEE747
:10811000FEE7FEE7FEE7FEE7FEE7FEE7FEE7FEE737
:10812000FEE7FEE7FEE7FEE7FEE7FEE7FEE7FEE727
:10813000FEE7FEE7FEE700002DC90100C580000054
:1081400030B50B46014600202022012409E00D46EF
:10815000D5409D4205D31D469540491B2546954077
:1081600040191546521E002DF1DC30BD70B50024BB
:108170002546002801DA01244042002901DA0125C0
:108180004942FFF7DDFFAC4200D04042002C00D056
:10819000494270BDF0B51FB40646002082B00546C6
:1081A0004024019100901BE0019922460F46304681
:1081B00000F066F9049A059B801A994110D3104685
:1081C0001946224600F04CF9361A8F410197224693
:1081D00001200021009F00F043F938184D41009024
:1081E0002046641E0028DFDC019B009829463246A9
:1081F00007B0F0BDF0B51FB486B00020009001902C
:1082000002900698069980B204900798090C02041F
:108210000014114307900027089D099806913E46D7
:108220003C4603900398A9B20204000C0390049802
:108230002D0C154348430021224600F011F9C719BF
:10824000714110340E46402CECDB3846029A00F0A7
:1082500007F9009A019B80180090594102980191FA
:10826000103002904028CCDB00980BB0F0BD0346E4
:108270000B439B0703D009E008C9121F08C0042A5A
:10828000FAD203E00B780370401C491C521EF9D24D
:108290007047D2B201E00270401C491EFBD2704709
:1082A0000022F6E710B513460A4604461946FFF7C2
:1082B000F0FF204610BD30B504460020034600E024
:1082C0005B1C934203D2E05CCD5C401BF8D030BD18
:1082D0000321001D401E037812021A43491EF9D5DE
:1082E00010467047034603220870000A491C521EBC
:1082F000FAD518467047024670B54A40D30FDB07DF
:1083000040002DD04A002AD0010E140E00021202A5
:108310000919400A520A8418E50104465443000A28
:10832000120A2E045043A4194219200CC543AA185E
:10833000120C0125AD03521C521912047F3924047A
:1083400000D0521C104301D44000491EC2B20C069A
:10835000C0092018401C4008802A02D003E00020F9
:1083600070BD40084000002900DA0020184370BDAD
:1083700070B502464A40D50F40004A00ED0740085C
:108380005208002814D0002A12D0C40DD30D410287
:108390000120C0055202490A520AE41A09181218AB
:1083A0007D34914201D3641C00E04900002C01DAC5
:1083B000002070BD0023914201D3891A0343400875
:1083C00049000028F7D100290AD0914202D10121A9
:1083D000C90705E0914201D2012101E00121C94311
:1083E000E005C018401900F05CF870BD10B500221F
:1083F0009623114600F05DF810BDC20FD207400071
:1084000040080BD0C10D0723DB01C9184002090544
:10841000400A1143C208400711437047002001463B
:108420007047000010B5002904DB0124E407404236
:108430008C412146002B04DB1C460123DB07524202
:10844000A341994200D1904210BD00000122D20701
:10845000002800DB101A002900DB511A88427047FF
:1084600010B5202A04DB0146203A9140002010BDBF
:10847000914020239C1A0346E3401943904010BDCD
:1084800010B5202A04DB0846203AD040002110BD58
:108490000B46D340D0402024A21A914008431946ED
:1084A00010BD002904DA401C490001D140084000F9
:1084B000704770B40024050C05D11024000402D1CB
:1084C000002921D01124050E01D100020834050F26
:1084D00001D10001241D850F01D18000A41C0028BA
:1084E00001DB4000641C002908D020252E1B0D460E
:1084F000F540A14000D001212943084301061B1B80
:10850000000ADB1D02D5002070BC7047DB0518187F
:1085100080180029F8DA401C4900F5D170BC4008E9
:1085200040007047064C0125064E05E0E36807CC85
:108530002B430C3C98471034B442F7D3FFF7C6FDE9
:10854000B81B0200D81B020070B58C180578401CBF
:108550006B075B0F01D10378401C2A1106D102780A
:10856000401C03E006780E70401C491C5B1EF9D1CC
:108570002B0705D40023521E0DD40B70491CFAE7BB
:108580000378401CCB1A921C03E01D780D70491C27
:108590005B1C521EF9D5A142D8D3002070BD70B526
:1085A00007F08CF80524204618F0A2F8002528468C
:1085B00007F078F8204618F09BF80126304607F0BF
:1085C0004DF8204618F094F8284607F047F8204662
:1085D00018F08EF8304607F065F8204618F088F855
:1085E00070BDB0B507F06AF80524204618F080F891
:1085F0000125284607F056F8204618F079F8284655
:1086000007F02CF8204618F073F8002007F026F841
:10861000204618F06DF8B0BDF0B581B007F03AF81B
:10862000052018F065F808270026012007F016F845
:108630000524204618F05CF8204618F059F807F099
:108640001FF80546204618F053F8002007F006F8FA
:10865000204618F04DF876002E437F1E3806E4D1F0
:10866000F0B201B0F0BD70B50446002006F0F6FF90
:1086700007F024F8052018F03BF80826E0B2C009FE
:1086800007F010F80525284618F032F8012006F00A
:10869000E5FF284618F02CF8002006F0DFFF2846FA
:1086A00018F026F8284618F023F86400761E3006E5
:1086B000E4D1052018F01CF8012070BDF0B583B09E
:1086C000019314460E4607460120384302900325C5
:1086D00004E000F08EF86D1E280631D000F067F837
:1086E0003846FFF7C0FF00F0A7F80028F1D1304668
:1086F000FFF7B9FF00F0A0F80028EAD100F057F822
:108700000298FFF7B0FF00F097F80028E1D1019838
:1087100002280BD3451E0026FFF77EFF2070FFF7CF
:108720003EFF641C761CF0B28542F5DCFFF774FF57
:108730002070FFF756FF00F05CF8202003B0F0BD7A
:10874000102003B0F0BDF0B583B01C46009201913B
:108750000290032504E000F04CF86D1E280623D09B
:1087600000F025F80298FFF77EFF00F065F800287A
:10877000F1D10198FFF777FF00F05EF80028EAD109
:10878000002C0CD00026009F3878FFF76CFF00F01B
:1087900053F80028DFD1761C7F1CA642F4D300F0EA
:1087A00028F8082003B0F0BD102003B0F0BDB0B52C
:1087B00006F084FF0524204617F09AFF012528467D
:1087C00006F04CFF204617F093FF284606F06AFF9C
:1087D000204617F08DFF0025284606F063FF20464F
:1087E00017F086FF284606F039FF642017F080FF57
:1087F000B0BDB0B506F062FF0524204617F078FF43
:108800000025284606F02AFF204617F071FF28466B
:1088100006F048FF204617F06BFF0125284606F0BA
:108820001DFF204617F064FF284606F03BFF64203A
:1088300017F05EFFB0BD0000B0B506F02BFF0524B9
:10884000204617F055FF012006F008FF204617F0DC
:108850004FFF0B4D06F014FF044606F0F9FE002C06
:1088600002D06D1E2804F5D10525284617F040FFDB
:10887000002006F0F3FE284617F03AFF2046B0BD70
:1088800033210000034801780B2901D8491C0170ED
:108890007047C046432F002070B584B00025039573
:1088A00002950195009506F0D3FE0F20C6430E4CAD
:1088B0001036F1B2A0206A461023FFF744FF20468D
:1088C00017F016FF204617F013FF912EF0D3A020CB
:1088D000B0216A461023FFF736FF204617F008FF45
:1088E0000248058004B070BD581B0000362F0020E0
:1088F00070B5022902D2EB24E0B270BD891EEB25CF
:108900000022134605E0401C5B1CDDB2A94225464F
:108910000EDB04786C40154604E034466E1C072DCF
:108920003546F0D26608E407F7D09A246640F4E7AB
:10893000E0B270BDF0B591B00C91417810AA117001
:1089400083781B025918C37804792402E3181B04A6
:1089500059180B0ED3700C0C94700D0A55700B91B6
:1089600008956918099409190A93C9180278D2431D
:108970008918427983791B029A18C379047A2402F0
:10898000E3181B049A188918130A0693C918130CC4
:108990000593C9180792120E04928918827AC37A35
:1089A0001B029A18037B0F90447B2402E3181B04DC
:1089B00098180918020A02928918020C0192891863
:1089C0000D910390000E0E9000200346014606E034
:1089D00032409A40D2B211435B1C082B0ED00126C4
:1089E00035469D400746024602E07F1C042FEFD02B
:1089F00010ACE45D2542F8D0521CF6E70E9C0D98B1
:108A00000019C3B20F98827B934205D0427A9142FB
:108A100002D1002011B0F0BD1021FFF769FF0C99C1
:108A2000CC72019A8A72029A4A72039A0A72049A62
:108A3000CA71059A8A71069A4A71079A0A710A9A46
:108A4000CA70099A8A70089A4A700B9A0A7011B013
:108A5000F0BDF0B58DB055220270002747720B783B
:108A60004370CA79059202728A790492C2714A7976
:108A7000039282710A7902924271CA7A0892427311
:108A80008A7A019202734E7AC6720C7A84720CAAA8
:108A900013704D782D02EB188D78C97809024919A9
:108AA0000904CB18190E01711D0CC57009931B0A1E
:108AB0000B90837038460A91D17007959570069394
:108AC000537031020919089A1202019BD21812043C
:108AD0005118089103990902029A8918059A1202FD
:108AE000049BD2181204511805913D463A4605E000
:108AF0002640AE4032436D1C082D0ED00124214685
:108B0000A9400346064602E05B1C042BF0D00CAFE4
:108B1000FF5C3942F8D0761CF6E70B9B5A72099835
:108B200006994018079940180A994018059A801824
:108B3000110A4018110C4018110E4018089A80189C
:108B4000110A4018110C4018110E4018563898732D
:108B500010211846FFF7CCFE0DB0F0BDF0B58FB078
:108B60000446FF20E070A07060700F20C0430290A8
:108B70000F302070704817F0BBFD704908686328FB
:108B800001D8642008606E4F002038806D4E01903F
:108B9000308008E00B99814222D338881030388029
:108BA00080B2A1286DD206F053FD3978A02003AA27
:108BB0001023FFF783FD30802028EED103AD0BA9F1
:108BC0002846FFF7B7FEE97B8842E6D1287855288A
:108BD000E3D15D48017800290298DBD10846D9E746
:108BE0003888A0284DD8C0B20021019105E006F0D8
:108BF0002FFD3988C8B2A12943D2C1B2A02003AA4F
:108C00001023FFF75BFD3080398810313980202830
:108C100037D103AD07A92846FFF78CFEE97B8842D0
:108C2000E5D128785528E2D14748007800280299F4
:108C300000D1014607988842D9D240490A68962156
:108C400051430B9A824208D90818904219D30BA9B4
:108C50000E222046FFF70BFBC9E78918814210D38B
:108C600007A90E222046FFF702FB0BA80A99818173
:108C700007980B9008980C9009980D9038880190EF
:108C8000B5E72078617809020818A178E278120225
:108C9000511809040818401C24D100200190388084
:108CA000A020B02103AA1023FFF708FD3080202860
:108CB00018D103AD0BA92846FFF73CFEE97B88429B
:108CC00010D1287855280DD11F480078002800D1F0
:108CD00002900B980299884204D20BA90E222046DA
:108CE000FFF7C5FA2078617809020818A178E278C0
:108CF0001202511809040818401C0CD10020E0721F
:108D0000A07260722072E071A07160712071E070D9
:108D1000A070607020700198388020786178090216
:108D20000818A178E27812025118090408180749B6
:108D3000086030880FB0F0BD70110100302F0020A6
:108D4000362F00202C2F00202F2F00203C2F00201A
:108D5000F0B581B000910646214800250570002A33
:108D60002ED01446C036631B71190F200840102204
:108D7000101A834200D303461A480278102A01D001
:108D8000042A1AD1C809FE2707405F2F13D80127EC
:108D9000B8436038C0B29E3282420CD3009A521956
:108DA000C9B2DFB23B46FFF789FC0F490880ED19D5
:108DB000A542D8D304E0082000E004200A49088036
:108DC000094801880020042902D0082900D0012088
:108DD00003490870411E8841400001B0F0BDC04603
:108DE000422F00202E2F0020402F00200A4A01236E
:108DF00013700A4A10700A4A11600A4A0021116071
:108E0000042801D105218901102801D11D208101EB
:108E1000054801807047C0462F2F00202E2F0020CC
:108E2000302F00203C2F0020342F0020F0B587B0D9
:108E3000994D00262E80994B1B688B4224D1994C6A
:108E40002188202925D1029000920196964C002776
:108E50002760964D964E2878062809D806F0F8FB2C
:108E60002068401C2060B042F5D38D480421018069
:108E70002F70904C20880107029B31D08848202118
:108E80000180854D019E0BE001204002844908804D
:108E900006E003A8FFF762FE208081488021018060
:108EA0007F4800883F2807DD874988420BDC40283F
:108EB00012D0802810D010E004280DD008280AD045
:108EC000202809D009E001214A02904204D0C902B9
:108ED000884201D001E002262E80288807B0F0BD2C
:108EE000A128019E00D32780009A012A6A4D1ED135
:108EF000187B012856D1DF719F715F711F711F733D
:108F0000587B012804D1DF729F725F721F725F73FA
:108F100003AF38461946FFF79CFDF87320880028F8
:108F200046D01038C1B2A02003AA102344E0002A82
:108F3000B6D1614801780029B2D00270187859780A
:108F4000090208189978DA781202511809040818E9
:108F50005A490978002901D00F21C943884233D2E8
:108F6000274603AC20461946FFF773FDE0733978B6
:108F7000A02010232246FFF7E6FB029A484908800A
:108F800008288DD13888103038801078517809023F
:108F900008189178D2781202511809040818484923
:108FA00008607DE7597B012911D10128A3D0A7E7EB
:108FB000A02003AA10230146FFF7C5FB384908800B
:108FC0003D48009901706BE70120C0025EE73D4813
:108FD0000078012812D103AC20461946FFF739FD6D
:108FE000E073A020B02110232246FFF7ACFB2C49F0
:108FF00008800828E4D133480770E1E718785978E9
:10900000090208189978DA78120251180904081828
:109010002B490968214A12685118884203D2204816
:1090200040210180CCE725490978002901D00F2192
:10903000C94388422DD203AF384619461C46FFF774
:1090400008FDF8731B480178A02010233A46FFF76B
:109050007AFB134908800828B2D1164908881030D5
:1090600008802078617809020818A178E278120255
:109070005118090408181249086008490A6815219E
:109080005143FFF75DF800299AD101200D4908707E
:1090900096E70120C00291E7482F0020302F0020E2
:1090A000462F00202C2F00204C2F0020432F002083
:1090B000818D5B00362F0020382F00202F2F0020BD
:1090C0003C2F0020442F0020FF010000F0B585B0A8
:1090D0000646434C0027278004921018414A128804
:1090E000904241D201910397404F00200290386096
:1090F0003F4C404D2078052809D806F0A9FA386879
:10910000401C3860A842F5D33748042101800298FA
:1091100020703948018839480278102A01D0042A81
:1091200032D188190346C033049C651A0F240440C9
:109130001020001B854200DB0546DC09603C01264F
:109140003002E7B27F09052F12D3B443E6B29E3254
:10915000B242234C039F0DD301984218D9B2EBB20F
:109160003046FFF7F0FA05E01F482021018011E0AA
:109170001B4C039F1C49088008280BD1E8B21E4AEB
:1091800011880818108005E0012080021649088027
:10919000134C039F144800881F2809DD202813D092
:1091A00001210A0290420FD0890288420CD00CE0C3
:1091B000042809D0082808D10F480088049988425B
:1091C00001D3022700E001272780208802210143E4
:1091D000022902D1084900220A8005B0F0BDC0462C
:1091E000482F0020342F0020462F00204C2F002035
:1091F000432F0020818D5B00502F00202E2F002058
:10920000F0B585B0044600200190042C6FD20CF01C
:109210001BF8002801D10CF097F80020009000BF47
:109220000098401C00900CF00FF803900398002861
:1092300003D0484900988842F2D30398002856D1B9
:10924000042145480BF0E2FF4448454908802101CC
:10925000444A515C4900404A505A41490A88012118
:10926000090300F055F902900120049020013D49C6
:1092700040184078002801D100264BE020013949F0
:1092800040184078012802D13548068842E0200184
:1092900034494018407802282AD120014018057925
:1092A0002901304A515C49002B4A505A2C490A88FE
:1092B0000121090300F02CF9064628012A49431828
:1092C0002801284940180289280140180021C76850
:1092D0003046B84706462801224BC018C2882801EC
:1092E000C0188178304600F087F8064612E02DE07D
:1092F00020011C4940184078032804D02001401860
:109300004078132804D1200116494018868801E0CE
:10931000002004900498002818D020011249431816
:109320002001104940180289200140183146C768C1
:109330000298B847019020010A4BC018C28820014A
:10934000C0188178019800F057F80190019805B095
:10935000F0BD000050C300000A0100208813000087
:10936000040100205412020094120200F8B50546D0
:109370000E4614460020009001211C4801751C482F
:10938000007888431A490870084680780821084305
:109390001749887000208871084600780121084329
:1093A0001349087008460572002717E01048007836
:1093B000802108430E49087000BF0E48007D002838
:1093C000FBD000200B4908750948C0892080A41CE7
:1093D0000748C1890098081800907F1CB742E5D360
:1093E00031460098FEF7ACFE80B2F8BD4061004007
:1093F000005004404060004010B50346012908D1E8
:10940000094CA41A9C4202D99C18A0B20BE0064851
:1094100009E0022906D1934202DD9C1AA0B202E0C3
:10942000002000E0184610BDFFFF000010B5044604
:109430000121202002F014F8002032490870012197
:1094400031480175002031490875152016F038FEA5
:109450002C488078E17808432A498870084680784B
:1094600021780843274988702078802806D108464B
:109470000079E17949000843224908712148807840
:10948000E17A08431F498870A078002803D1084674
:10949000007908710FE0A078012806D119480079F9
:1094A000602108431749087105E0164800798021BA
:1094B00008431449087113488079217908431149F8
:1094C000887108468079617908430E498871207A4D
:1094D000C872607A88720846007838218843094942
:1094E0000870084600786178C9000843054908708B
:1094F000A07A0873084600780121084301490870E2
:1095000010BD000000500440406100404060004039
:10951000F8B504460E461746002E01D100250FE08F
:10952000A64201DC3D460BE00094009C20467843B7
:10953000009031460098FEF703FE0090009885B237
:109540002846F8BD0146042904D28A00024BD218ED
:10955000508800E00020704720290020014604299F
:1095600003D28A00024B985C00E0002070470000A4
:1095700020290020FFB587B004460898844203DA0A
:109580000A988068002802D12448019042E0089897
:10959000001B82B20292002625460A9880680021AC
:1095A0002F463A463346049605910690FEF722FE72
:1095B00005460E46002328463146029AFEF7EAFD8C
:1095C00005460E46304600210A46494050400143B8
:1095D00002D0124801901DE003950A98C068039DCF
:1095E000A84202D30020019014E00A98C1680398B1
:1095F000401A039009990398FEF7A2FD039003987F
:10960000000C0004002802D00448019002E00398F6
:1096100080B2019001980BB0F0BD0000FFFF000088
:1096200010B5084800788021884306490870012158
:1096300005480175002005490875152016F040FD04
:1096400010BD0000005004404061004040600040F8
:10965000F8B505460E4614461F4621462846FEF735
:1096600085FD80B2F8BD0000FFB587B006460A98B8
:109670004068002801D1029035E00A9801684068EE
:1096800008180390002534460021274603980695C4
:109690000491059038462946049B059AFEF7AAFDD9
:1096A00004460D460A984068024600230190204671
:1096B0002946FEF76FFD04460D4600232046294645
:1096C000099AFEF767FD04460D46284607492140E2
:1096D000002359405840014303D00448C04302903E
:1096E00001E0A0B2029002980BB0F0BD0000FFFFB5
:1096F00010B5FE4800688079030016F0C7FC070526
:109700009ED8F5F4F3F2F100F848006840790300C0
:1097100016F0BCFC0805138A2A8A468A638A12F06E
:109720003BFD0020F1490968C873F04800684079A2
:10973000401CEE49096848717DE0ED494969EB4AF2
:109740001268D27A885C12F09FFDE8480068407980
:10975000401CE64909684871E44800684079401CAB
:10976000E2490968487166E00AF04AF8002810D119
:1097700012F08AFDDD4800684079401CDB49096829
:109780004871DA4800684079401CD8490968487136
:1097900005E012F02BFD0020D449096848714AE029
:1097A0000AF02EF8002811D1112012F06DFDCF48DB
:1097B00000684079401CCD4909684871CB48006871
:1097C0004079401CC9490968487105E012F00EFD56
:1097D0000020C649096848712DE00AF011F80028F8
:1097E0001BD1C2480068C07A401CC0490968C872D1
:1097F000BE480068C07ABE49097888420DDB002067
:10980000BA490968C872B94909684862B748006826
:109810008079401CB5490968887112F0E7FC002086
:10982000B2490968487106E012F0E0FC0020AF4937
:109830000968487100BF00BF32E3AC480068407C53
:10984000002817D0AA48C068002803D0A848C168DB
:10985000192088470020A54909684862A348006884
:109860008079401CA1490968887100209F490968D6
:1098700048711BE09D480068406A282807D29B4831
:109880000068406A401C9949096848620EE000205F
:10989000964909684862954800688079401C934958
:1098A000096888710020914909684871F8E28F4879
:1098B00000684079030016F0E9FB080518A42FA4FE
:1098C0004CA480A412F068FC002088490968C87381
:1098D000864800684079401C84490968487197E0CF
:1098E000D4E2C7E230E25DE194E0814949697F4A10
:1098F0001268D27A885C12F0C7FC7C480068407914
:10990000401C7A4909684871784800684079401CD1
:109910007649096848717BE009F072FF002811D18F
:10992000012012F0B1FC714800684079401C6F4979
:10993000096848716D4800684079401C6B490968A6
:10994000487105E012F052FC00206849096848712E
:109950005EE009F055FF002828D164490968C97AFA
:1099600024225143634A12688918604A1268D27BE4
:10997000885C12F089FC5D480068C07B401C5B4934
:109980000968C87359480068C07B242814D3574815
:1099900000684079401C554909684871534800687F
:1099A0004079401C51490968487105E012F01EFCDD
:1099B00000204E49096848712AE009F021FF00287B
:1099C00018D14A480068C07A401C48490968C872E2
:1099D00046480068C07A4649097888420ADB002078
:1099E00042490968C872414800688079401C3F4973
:1099F0000968887112F0FAFB00203C490968487137
:109A000006E012F0F3FB002038490968487100BFF6
:109A100000BF45E2354800684079030016F036FB88
:109A20000A0614B92BB948B978B995B912F0B4FB44
:109A300000202E490968C8732C4800684079401CF2
:109A40002A4909684871ABE029494969274A1268DF
:109A5000D27A885C12F018FC244800684079401CD7
:109A6000224909684871214800684079401C1F4913
:109A70000968487194E009F0C3FE002811D14A201A
:109A800012F002FC194800684079401C1749096827
:109A90004871164800684079401C144909684871AB
:109AA00005E012F0A3FB002010490968487177E037
:109AB00009F0A6FE002824D1FF2012F0E5FB0B4898
:109AC0000068C07B401C09490968C87307480068E2
:109AD000C07B24281BD3054800684079401C0349FB
:109AE0000968487101480068407905E0D007002006
:109AF000142F0020CC070020401CEA490968487157
:109B000005E012F073FB0020E6490968487147E060
:109B100009F076FE002811D1FF2012F0B5FBE148D4
:109B200000684079401CDF4909684871DD480068D9
:109B30004079401CDB490968487105E012F056FB8A
:109B40000020D849096848712AE009F059FE002828
:109B500018D1D4480068C07A401CD2490968C8723C
:109B6000D0480068C07AD049097888420ADB0020D2
:109B7000CC490968C872CB4800688079401CC94943
:109B80000968887112F032FB0020C64909684871E3
:109B900006E012F02BFB0020C2490968487100BFA3
:109BA00000BF7DE1BF4800684079030016F06EFAFF
:109BB0000C0715C32CC349C366C382C39FC312F0ED
:109BC000EBFA0020B7490968C873B64800684079C5
:109BD000401CB44909684871B4E0B3494969B14AC5
:109BE0001268D27A885C12F04FFBAE480068407968
:109BF000401CAC4909684871AA4800684079401C7B
:109C0000A849096848719DE009F0FAFD002811D1C2
:109C1000772012F039FBA34800684079401CA14925
:109C2000096848719F4800684079401C9D4909684F
:109C3000487105E012F0DAFA00209A490968487183
:109C400080E009F0DDFD002811D10C2012F01CFB92
:109C5000944800684079401C9249096848719148CD
:109C600000684079401C8F490968487105E012F08E
:109C7000BDFA00208B490968487163E009F0C0FD16
:109C8000002810D112F000FB864800684079401C83
:109C9000844909684871834800684079401C8149BB
:109CA0000968487105E012F0A1FA00207D490968B1
:109CB000487147E009F0A4FD002811D1132012F0EB
:109CC000E3FA784800684079401C76490968487191
:109CD000744800684079401C72490968487105E081
:109CE00012F084FA00206F49096848712AE009F0EF
:109CF00087FD002818D16B480068C07A401C69496C
:109D00000968C87267480068C07A6749097888425C
:109D10000ADB002063490968C872624800688079DC
:109D2000401C60490968887112F060FA00205D49A2
:109D30000968487106E012F059FA0020594909688B
:109D4000487100BF00BFABE056480068407903008F
:109D500016F09CF9080513872A874787638712F056
:109D60001BFA00204F490968C8734E4800684079C3
:109D7000401C4C49096848717AE04B494969494A95
:109D80001268D27A885C12F07FFA464800684079FF
:109D9000401C444909684871424800684079401CA9
:109DA00040490968487163E009F02AFD002811D193
:109DB000492012F069FA3B4800684079401C394953
:109DC00009684871374800684079401C354909687E
:109DD000487105E012F00AFA00203249096848711A
:109DE00046E009F00DFD002810D112F04DFA2D4883
:109DF00000684079401C2B4909684871294800686F
:109E00004079401C27490968487105E012F0EEF9D5
:109E100000202449096848712AE009F0F1FC002873
:109E200018D120480068C07A401C1E490968C872D1
:109E30001C480068C07A1C49097888420ADB002067
:109E400018490968C872174800688079401C15498C
:109E50000968887112F0CAF900201249096848712E
:109E600006E012F0C3F900200E490968487100BFEE
:109E700000BF15E000200B4909688871094909688D
:109E80004871062007490968C87009E012F0AEF968
:109E9000002004490968487102490968887100BFB7
:109EA00000BF10BDD0070020142F002010B56A4855
:109EB00000684079030016F0E9F8090610C627C6C5
:109EC00044C6608EC60012F067F9634800684079A6
:109ED000401C614909684871BCE0604949695E4AB3
:109EE0001268D27A885C12F0CFF95B48006840793A
:109EF000401C594909684871574800684079401C1E
:109F0000554909684871A5E009F07AFC002811D18B
:109F10007F2012F0B9F9504800684079401C4E4942
:109F2000096848714C4800684079401C4A490968F2
:109F3000487105E012F05AF9002047490968487154
:109F400088E009F05DFC002810D112F09DF942482C
:109F500000684079401C4049096848713E480068E3
:109F60004079401C3C490968487105E012F03EF90F
:109F700000203949096848716CE009F041FC00286B
:109F800022D135480068C07A401C33490968C8723C
:109F900031480068C07A3149097888420FDB0020D7
:109FA0002D490968C8722C4800684079401C2A492C
:109FB00009684871002028490968486208E00020C3
:109FC00025490968487103E0002023490968487160
:109FD00012F00CF93EE020480068407C002816D0C2
:109FE0001E48C068002803D01C48C1681920884753
:109FF00000201949096848621749096848711649DB
:10A0000009688871052014490968C8701AE0124867
:10A010000068406A282807D20F480068406A401C40
:10A020000D49096848620DE000200B490968486243
:10A030000949096848710849096888710520064975
:10A040000968C87006E012F0D1F8002002490968DA
:10A05000487100BF00BF10BDD0070020142F0020A2
:10A0600010B50024F7480068807A01287ED1F548B1
:10A070000068C07900287AD0F2480068807900280A
:10A0800004D0012874D0022873D191E1ED48006812
:10A09000007B24286ED2EB480068C07901287AD171
:10A0A000002475E0E7480068C07A24214843E64967
:10A0B00009684018E3490968097B415CE148006888
:10A0C000C07A24225043E14A12688018DD4A12689F
:10A0D000127B805C814229D0DA480068C07A242152
:10A0E0004843DA4909684018D6490968097B415C48
:10A0F000D4480068C07A24225043D34A126880189A
:10A10000D04A1268127B8154CE480068407B2428D4
:10A1100005D3CC480068007BCA4909684873C94820
:10A120000068007BC7490968887308E0C548006873
:10A13000407B242803D20120C24909688871C148A4
:10A140000068007B401CBF4909680873BD4800686F
:10A15000007B242808D3BB480068407B242803D216
:10A160000120B84909688871B64805E0D3E1CDE11E
:10A1700069E0BAE138E00EE00068007B242804D2F0
:10A18000B04800688079012800D103E0601CC4B2A7
:10A19000242C87D356E0002413E0AA480068C07A34
:10A1A00024214843A94909684018015DA548006871
:10A1B000C07A24225043A44A126880180155601CBA
:10A1C000C4B2242CE9D300209E4909684873232097
:10A1D0009C490968887301209A490968887124207C
:10A1E0009849096808732DE00020964909680873AA
:10A1F00094480068C07A401C92490968C872914826
:10A200000068C07A92490978884217DB8D48006857
:10A21000007C012804D102208A490968887106E07F
:10A22000002088490968887186490968C87100203A
:10A2300084490968C8728349096808740020814903
:10A240000968487161E17F4800684079030015F0B2
:10A250001DFF080513A62AA651A68EA6012079493E
:10A260000968087411F098FF764800684079401C2E
:10A2700074490968487199E075494969714A1268D9
:10A28000D27A885C12F000F86E4800684079401C71
:10A290006C49096848716B4800684079401C6949FD
:10A2A0000968487182E009F0ABFA00281BD16549C2
:10A2B0000968497B491CC8B211F0E6FF6148006893
:10A2C000407B60490968C8735E4800684079401C5B
:10A2D0005C49096848715B4800684079401C5949ED
:10A2E0000968487105E011F081FF002055490968AF
:10A2F00048715BE009F084FA00282BD151490968C4
:10A30000C97A24225143504A126889184D4A12686A
:10A31000D27B885C11F0B8FF4A480068C07B401CC3
:10A3200048490968C87347480068C07B45490968BF
:10A33000897B88421ADD434800684079401C4149C6
:10A34000096848713F4800684079401C3D490968E8
:10A3500048710BE011F04AFF3A480068407B3949E8
:10A360000968C87300203749096848711EE009F080
:10A3700047FA00280CD133490968887124203149F3
:10A380000968C8732F49096848732E49096888739A
:10A3900011F02CFF00202B490968487106E011F0EC
:10A3A00025FF002027490968487100BF00BFACE0C5
:10A3B000244800684079030015F068FE08050F8EF8
:10A3C000268E4C8E688E11F0E7FE1E48006840799C
:10A3D000401C1C490968487185E01D494969194AB2
:10A3E0001268D27A885C11F04FFF164800684079F5
:10A3F000401C144909684871124800684079401CA3
:10A400001049096848716EE009F0FAF9002811D185
:10A41000492011F039FF0B4800684079401C094978
:10A4200009684871074800684079401C0549096877
:10A43000487105E011F0DAFE002002490968487110
:10A4400051E00000D0070020CC070020C807002002
:10A45000142F002009F0D4F9002810D111F014FFB6
:10A460009C4800684079401C9A490968487199489D
:10A4700000684079401C97490968487105E011F06F
:10A48000B5FE00209349096848712CE009F0B8F93D
:10A4900000281AD18F480068C07A401C8D4909688D
:10A4A000C8728C480068C07A8B49097888420CDBF6
:10A4B000002088490968C8728649096888718549F9
:10A4C0000968487183490968C87111F08FFE00203E
:10A4D00080490968487106E011F088FE00207D4936
:10A4E0000968487100BF00BF0FE011F07FFE002037
:10A4F0007849096848717749096888717549096818
:10A50000087374490968C87200BFE2E0002071490D
:10A5100009688872DDE06F480068807A0228F4D10B
:10A520006C480068007A002879D06A480068407951
:10A53000030015F0ABFD0B0711BB25BB41545EBBFF
:10A540007590BB0011F028FE624800684079401CFD
:10A55000604909684871B7E05F494969087811F0B6
:10A5600093FE5C4800684079401C5A49096848716C
:10A57000584800684079401C564909684871A3E072
:10A5800009F03EF9002810D111F07EFE5148006814
:10A590004079401C4F49096848714E48006840792D
:10A5A000401C4C490968487105E011F01FFE00206D
:10A5B00048490968487187E009F022F9002807D165
:10A5C000444800684079401C42490968487103E0EA
:10A5D000002040490968487111F008FE74E011F04C
:10A5E000DBFD3C4800684079401C3A4909684871E5
:10A5F0006AE0394949690978491CC8B211F044FE3A
:10A60000344800684079401C324909684871314833
:10A6100000684079401C2F490968487154E054E0B3
:10A6200009F0EEF800280FD111F088FD29490968DA
:10A630008870012011F0FCFD264800684079401C1C
:10A6400024490968487105E011F0D0FD0020214936
:10A650000968487138E01F480068807811280CD1DB
:10A6600000201C4909680872AA201A4909688870E4
:10A67000002018490968487011E0164800684078C1
:10A68000401C144909684870124800684078032843
:10A6900005D309F055F900200E490968487011F0FA
:10A6A000A5FD00200B49096848710DE011F09EFDE1
:10A6B0000020084909684871064909684870AA20BD
:10A6C00004490968887000BF03E000200149096857
:10A6D000887210BDD0070020142F0020F0B5054669
:10A6E0000C4616461F462088482806DA3A46294670
:10A6F000304604F0EBFF012800D0F0BD2088C000F8
:10A700002E502088401C208000BFF6E710B502467E
:10A710009000074BC018405C002802D00320C043C3
:10A7200010BD01209300024C1B1958540020F7E77C
:10A73000942A002070B5002508E06D1C1B48854256
:10A7400002D20AF02DFE01E0002503E00AF07CFDB4
:10A750000028F2D100BF022100200AF083FD03216E
:10A7600000200AF07FFD052100200AF07BFD072173
:10A7700000200AF077FD002408E00020A1000C4A28
:10A780005054A10089184880601CC4B2042CF4D332
:10A7900001200849087000204870052088700020BA
:10A7A000C87005480549088070BD000050C300000E
:10A7B0002029002006010020881300000401002049
:10A7C000F8B58D480078030015F060FC0604051606
:10A7D0003D5EFDFC0EE10AF0B7FD00208649C87021
:10A7E000487008468078002802D10320087002E0F3
:10A7F000022081490870FDE07F488078002804D05D
:10A800007D488078401E7C4988700AF01DFD002834
:10A810000BD10AF099FD00207749C870084680786E
:10A8200000280FD1032008700CE07348C078401C4A
:10A830007149C8700846C078052803D30520087000
:10A840000AF0AEFDD6E00AF0FFFC00280ED104218C
:10A850006A480AF0DBFC00206749C8704870684805
:10A86000684908800420644908700CE06248C07898
:10A87000401C6149C8700846C078052803D30520EC
:10A8800008700AF08DFDB5E05B49497809015E4A20
:10A89000515C4900594A505A5A490A880121090312
:10A8A000FEF736FE009001255348407800015649D6
:10A8B00040184078002801D100243CE04E48407800
:10A8C0000001514940184078012802D14D480488C0
:10A8D00031E04948407800014B494018407802284F
:10A8E00012D1454949780901474A89180879FEF784
:10A8F00029FE0446404949780901434A89180879E4
:10A90000FEF72CFE054616E03B48407800013E4924
:10A9100040184078032806D0374840780001401896
:10A920004078132806D13448407800013649401851
:10A93000848800E00025002D2FD02F4840780001AA
:10A94000324943182C48407800012F4940180289A9
:10A9500029484078000140182146C7680098B84748
:10A960000646254840780001274BC018C288224877
:10A9700040780001C01881783046FEF73DFD06465C
:10A980001D484078800022494018468001201A491D
:10A99000497889001E4A50540AE000201649497837
:10A9A00089001B4A89184880134949788900505406
:10A9B00011484078401C10494870084640780428E7
:10A9C00009D301E013E007E00AF0BEFC00200A49C9
:10A9D0004870032008700DE00AF036FC002803D10F
:10A9E00001200549087001E00AF0DAFC02E0FFF7F7
:10A9F000A1FE00BF00BFF8BD060100200A01002033
:10AA00008813000004010020541202009412020076
:10AA10002029002010B50AF0E1FB002405E0002009
:10AA2000A100074A5054601CC4B2042CF7D3002084
:10AA3000044908700520887003480449088010BD47
:10AA400020290020060100208813000004010020B6
:10AA500070B50446002000F0AFF8002000F0DAF8EE
:10AA6000002000F09BF8002000F0C4F8002000F067
:10AA700087F8002000F0AEF800BF012000F08EF84B
:10AA8000012000F0B7F8002521E0002000F086F852
:10AA9000002000F0AFF880202040002806D00120E0
:10AAA00000F08AF8012000F0B5F805E0002000F081
:10AAB00083F8002000F0AEF800BF012000F06EF82F
:10AAC000012000F097F86006040E681CC5B2082D3E
:10AAD000DBDB012000F054F8012000F07BF870BDB2
:10AAE00070B504460D46012000F066F8012000F024
:10AAF00091F8002000F052F8002000F07BF80020D0
:10AB000000F03EF8002000F065F800BF012000F0E2
:10AB100045F8012000F06EF8002628E0002000F043
:10AB20003DF8002000F066F880202040002803D087
:10AB3000012000F041F802E0002000F03DF8802004
:10AB40002840002803D0012000F064F802E0002033
:10AB500000F060F800BF012000F020F8012000F0B4
:10AB600049F86006040E6806050E701CC6B2082E71
:10AB7000D4DB012000F004F8012000F02BF870BDB8
:10AB800010B50446002C04D0812103200AF09AFC61
:10AB900003E0802103200AF095FC10BD10B50446A7
:10ABA000002C04D0812104200AF08CFC03E08021D9
:10ABB00004200AF087FC10BD10B50446002C04D018
:10ABC000812102200AF07EFC03E0802102200AF0AD
:10ABD00079FC10BD10B50446002C04D08121044836
:10ABE0000AF070FC03E0802101480AF06BFC10BD04
:10ABF0000107000010B50446002C05D08121072074
:10AC000000020AF05FFC04E08021072000020AF045
:10AC100059FC10BD10B50446002C04D08121044815
:10AC20000AF050FC03E0802101480AF04BFC10BD03
:10AC30000207000010B5F920FFF70AFF8820FFF790
:10AC400007FF9020FFF704FF9820FFF701FF08217E
:10AC50000846FFF745FFE820FFF7FAFE12210846F5
:10AC6000FFF73EFFA020FFF7F3FE70210846FFF735
:10AC700037FFA820FFF7ECFE70210846FFF730FFF2
:10AC8000B020FFF7E5FE70210846FFF729FFB82046
:10AC9000FFF7DEFE00210846FFF722FFC020FFF786
:10ACA000D7FE00210846FFF71BFFC820FFF7D0FEA4
:10ACB00000210846FFF714FFD020FFF7C9FE2F211F
:10ACC0000846FFF70DFFD820FFF7C2FE2F210846E8
:10ACD000FFF706FFE020FFF7BBFE2F210846FFF736
:10ACE000FFFE4020FFF7B4FE00210846FFF7F8FE04
:10ACF0000A20FFF7ADFE002405E000210846FFF71B
:10AD0000EFFE601CC4B25A2CF7DB00240AE00020DE
:10AD10000B4908550B4908550B4908550B4908556F
:10AD2000601CC4B25A2CF2DB8120FFF791FE002098
:10AD3000074908708870C8700871487010BD00001D
:10AD400048260020A2260020FC26002056270020AE
:10AD5000DB00002010B58020FFF77AFE10BD000058
:10AD60000020044908700120034908700020487041
:10AD700070470000E0000020DB00002010B54848CC
:10AD8000007800287AD046488078030015F07EF9D4
:10AD90000604434A535A687E414800794149085C99
:10ADA0003F490979404A515C884209D13C480079C1
:10ADB0003E49085C3A4909793D4A515C88421BD0BA
:10ADC000374800793749085C35490979364A505483
:10ADD000334800793549085C31490979344A50547F
:10ADE0002F48C078002803D004202D49887011E036
:10ADF00001202B4988700DE000202949C8700846C1
:10AE00000079401C0871084600795A2802DB0020AE
:10AE10000871087041E04020FFF71AFE0220204927
:10AE200088703AE01E4A11791079FFF759FE032025
:10AE30001B49887031E00A20FFF70AFE04201849F8
:10AE400088702AE0164A1279194B995C144A1279D3
:10AE5000154B985CFFF744FE0520114988701CE0F3
:10AE60000F480079401C0E490871084600795A289D
:10AE700005DB002008710870C87003E00EE00120B7
:10AE80000749C87000200649887006E00020044980
:10AE900008708870C870087100BF00BF10BD000046
:10AEA000DB00002048260020A2260020FC260020EF
:10AEB0005627002010B511F0A7FD012837D1072033
:10AEC00009F062FA002810D01C480078052805DA3D
:10AED0001A480078401C1949087016E005201749E7
:10AEE00008700020164908700FE015480078052802
:10AEF00005DA13480078401C1149087005E0052068
:10AF00000F49087000200D4908700C48007805288A
:10AF100006D14B22D2000021012013F071FA0BE080
:10AF20007D22D2000021012013F06AFA04E0002201
:10AF30001146012013F064FA10BD00001D0000202E
:10AF40001C00002000200349087248708870486087
:10AF500070470000580A002058221152704710B55F
:10AF600004460121022000F07BFA0021022000F0BB
:10AF700077FA10BD014600205322525C10231A407C
:10AF8000002A08D05322525C0C231A409210032A44
:10AF900018D1032016E05422525A0123DB031A4031
:10AFA000002A0ED05322525C0C231A409210032A1E
:10AFB00005D05322525C9207920F032A01D102203E
:10AFC00000E0012070470246002058239B5A0B40A6
:10AFD000002B01D0012000E0002070470146002234
:10AFE0006020405AFF231B0218400005020F100189
:10AFF000014BC018704700000055044010B5002AEE
:10B000000AD056231B5A0C0223435624235256239C
:10B010001B5A8B43235209E056231B5A0C02A343AD
:10B020005624235256231B5A0B43235210BD0000B3
:10B03000F8B504460D46012700263448844203D162
:10B040000121022000F00CFA2878401EA070208810
:10B05000FF210131084320802088400840002080E3
:10B06000A878401EC1B25A20015568790007000C2B
:10B07000E97909020843A97908435C210853288922
:10B0800081B240200153A868C000C10C4220015386
:10B09000A88981B244200153E868C000C10C462051
:10B0A0000153288A81B2482001532869C000C10C8D
:10B0B0004A200153A88A81B24C2001536869C0001C
:10B0C000C10C4E2001535020005B2979090208432E
:10B0D000502108535020005B2979884350210853A0
:10B0E00000E0761C5020005B4007400F2979884221
:10B0F00002D007488642F4D15020005B4007400F41
:10B100002979884200D000273846F8BD0054044011
:10B11000FFFF000030B5034600201C898C4209DD8A
:10B12000082A05D218244C431D682C19A05C02E0A3
:10B13000002000E0002030BD10B5024613898B428C
:10B1400005DD18234B431468E318987C00E00020C9
:10B1500010BD0146FF22C889C007C00F00280AD0D1
:10B160000120C88100E0521EC889C007C00F002816
:10B1700001D0002AF7D1C889C007C00F00280FD11D
:10B180000220C8810420C881487A400840004872E3
:10B19000487A38239843487200204872012070474B
:10B1A0000020FCE70246507A012318435072507A7F
:10B1B0000B78DB0018435072087A012808D1888880
:10B1C00050814868000C0123DB031843908108E09C
:10B1D000087A002805D15081486880001A4B184031
:10B1E0009081487A012804D1507A40231843507244
:10B1F00006E0487A002803D1507A402398435072E1
:10B200000878002811D1C87A1072087B1070487B2A
:10B210005070887B9070CB7BD370087C10714B7C16
:10B220005371887C9071CB7CD371887A002803D0CD
:10B230000120C002D08101E00820D081FF20013030
:10B24000D081012070470000FC1F0000002904D0BD
:10B25000427A80231A43427203E0427A80239A435F
:10B260004272704730B5024600200F4B5024A45A5A
:10B270000D022C435025AC525024A45A8C43AC529E
:10B2800000E05B1E5024A45A6407640F8C4201D076
:10B29000002BF6D15024A45A6407640F002C01D06F
:10B2A000002000E0012030BDFFFF0000827A8023F3
:10B2B0001A40802A00D081727047000070B50446A1
:10B2C00000250023002D02D0012660200653042013
:10B2D000C88188890126F6033040002808D0012063
:10B2E00010728889C004C0084E893043506006E05F
:10B2F0000020107288890F4E304080105060087A0C
:10B30000D072002304E0CE5C10460C30C6545B1CA7
:10B31000D07A9842F7DCC88904263040002804D14E
:10B32000C889F6023040002801D0002070BDD07AD4
:10B33000FCE70000FC1F00000020024908800249D1
:10B34000088070477A0000207C000020027C802367
:10B350001A40802A00D00174704710B50246FF23BE
:10B36000D089C007C00F00280AD00120D08100E09A
:10B370005B1ED089C007C00F002801D0002BF7D179
:10B38000D089C007C00F002801D0002010BD507A1E
:10B39000012420435072507A3824A0435072C87A56
:10B3A0001072487A00280FD1087B1070487B5070CB
:10B3B000887B9070CC7BD470087C10714C7C54716D
:10B3C000887C9071CC7CD471FF200130D08140000A
:10B3D000D081107ADAE70000F8B504460D46002067
:10B3E000002C00D100BF002A00D100BF012C01D1E8
:10B3F00041263043012A01D112263043022C01D1CB
:10B40000C0263043022A01D130263043134E30701B
:10B4100076788027BE43114F7E70012C08D1FF2122
:10B4200000BF0E4EB3781E460E4033468B42F8D115
:10B430000A4E76784027BE43084F7E70012A0BD112
:10B440000026009603E000BF009E761C0096FF27B2
:10B450006937009EBE42F6D9F8BD000000040240E4
:10B46000002905D0054A12780243044B1A7004E003
:10B47000024A12788243014B1A707047200402403E
:10B48000002905D0054A927E0243044B9A7604E0D7
:10B49000024A927E8243014B9A767047000802402E
:10B4A00001200649087000BF044800788021084048
:10B4B0000028F9D00120024908707047000C0240B2
:10B4C000A001002070B5034614460020002B01D1D6
:10B4D000C0B202E005468035E8B2012902D1051D5F
:10B4E000E8B206E0022903D105460835E8B200E0DB
:10B4F000C0B2012C02D1851CE8B200E0C0B2084DF8
:10B50000A870AD7801263543054EB570002201E0E4
:10B5100000BF521C7D252D01AA42F9D970BD000043
:10B52000000C024070B50024244800792021084016
:10B53000002801D0224D3FE000F046F805462148A2
:10B54000007880210840002836D01E4880780840C6
:10B55000002801D01A4D02E000F036F805461948DF
:10B5600080780007840F022C01DBAD0804E0012C79
:10B5700001D16D0800E000BF124880788007C00F3D
:10B58000002801D02D0101E00C2045430D48007832
:10B590004007840F002C02D1601CC4B207E0032CCA
:10B5A00003D1601C4006040E01E06006040E214633
:10B5B0002846FCF7C5FD0546284670BD000402403C
:10B5C00000127A00000C024000B5C0229178F822E7
:10B5D00011401C4A12781143EA2923D00ADC0A469A
:10B5E000E03A130014F052FD0A181C20242A2A2ADB
:10B5F0002A161A2AED291FD004DCEB2916D0EC29D3
:10B600001CD117E0F02903D0F82917D10E4817E014
:10B610000E4815E00E4813E00E4811E00E480FE00A
:10B620000E480DE00E480BE00E4809E00E4807E01A
:10B630000E4805E00E4803E00E4801E00D4800BF4B
:10B6400000BF00BD201C02400090D003006CDC0253
:10B650000048E80100366E010024F400001BB7002A
:10B6600000127A00808D5B0000093D00C0C62D00ED
:10B6700080841E0040420F0010B50446204600F0B2
:10B68000E1FD002010BD000010B5A8211348FCF713
:10B6900007FE1248124908601248486007200881D6
:10B6A0000020887207220F490D4800F065FA00213A
:10B6B0000B48FFF7FBFDA0210B48FCF7F1FD0A4802
:10B6C0000A4948600A4B05220A49084800F02AFC4A
:10B6D00055210648FFF73AFE10BD00007008002013
:10B6E000500800208C0E0200180900205C08002081
:10B6F00079B60000000E02000C4A127812060B4BBD
:10B700005B781B041A43094B9B781B021A43074BB7
:10B71000DB781A43104642084240D20083085A4060
:10B720001146034A5140034A116070471707002031
:10B73000010200001C070020F8B504460F46A07A5D
:10B740004006400E002874D10025ACE01820684364
:10B7500021680818407C01283CD101211820684349
:10B7600022681018017400260CE018206843216834
:10B7700008180830815D1820684322681018815528
:10B78000701CC6B2082EF0D300211820684322682E
:10B79000101801741820684322681018417418208A
:10B7A0006843226810184161182068432268101805
:10B7B00081742C20684361680818406A002809D009
:10B7C00018236B432268D0182C236B436268D2186D
:10B7D000516A884718206843216808184069FF218A
:10B7E000C94388425DD81820684321680818406919
:10B7F000C119182068432268101841611820684355
:10B800002168081841692C20684362681018806913
:10B81000814246D31820684321680818807C552847
:10B820003FD05521182068432268101881740026E3
:10B8300024E03CE01820684321680818805D2C2132
:10B840006943626851181031895D084018216943C5
:10B850002268511888551820684321680818805DAF
:10B860002C216943626851180831895D0843182109
:10B870006943226851188855701CC6B2082ED9D366
:10B880002C20684361680818806A002809D01823B2
:10B890006B432268D0182C236B436268D218916ADC
:10B8A0008847681C85B22089A84200DD4EE7F8BDB4
:10B8B00010B50446002014F04DFF022841D1214864
:10B8C0000078002802D101201E4908701D48007828
:10B8D00001281FD11B484078401C1A494870214656
:10B8E0005A20FCF72DFC17494978884229D80020B6
:10B8F0001449487008468078401C88700846807853
:10B900000A2803D30020887002200870002014F059
:10B9100051FF16E00B480078022812D10948407800
:10B92000401C0849487021467D20C000FCF708FCF7
:10B9300004494978884204D800200249487014F02C
:10B9400039FF10BD7600002000B587B000216846A1
:10B950000171042141710C480290411003910B497F
:10B96000049105910A480690FFF78EFE01A814F095
:10B9700085FF00F08DFB00F00FF80021054809F06D
:10B980000DFE07B000BD0000FFFF1F00FFFFFF1FFF
:10B9900001BC00000205000010B5FF200230724912
:10B9A00048600020087201200870002048720120C1
:10B9B00088726E48FFF7CDFB6B496C48FFF7F2FBCE
:10B9C00001216A48FFF742FC694867494860002046
:10B9D00008720120087000204872012088726348B4
:10B9E0001030FFF7B6FB604960481030FFF7DAFB14
:10B9F00001215E481030FFF729FC5D48401E5A497E
:10BA00004860002008720120087000204872012060
:10BA1000887256485030FFF79CFB534953485030CA
:10BA2000FFF7C0FB012151485030FFF70FFC504891
:10BA3000C1384D494860002008720120087000207C
:10BA400048720120887249484030FFF782FB46491E
:10BA500046484030FFF7A6FB012144484030FFF73D
:10BA6000F5FBFF2012304049486000200872012099
:10BA7000087000204872012088723C486030FFF74F
:10BA800068FB394939486030FFF78CFB01213748A2
:10BA90006030FFF7DBFBFF20213033494860002096
:10BAA00008720120087000204872012088722F4817
:10BAB000A030FFF74EFB2C492C48A030FFF772FB5B
:10BAC00001212A48A030FFF7C1FB29488F382649B9
:10BAD0004860002008720120087000204872012090
:10BAE00088722248E030FFF734FB1F491F48E030DE
:10BAF000FFF758FB01211D48E030FFF7A7FB3F206F
:10BB00004001194948600020087201200870002097
:10BB100048720120887215482030FFF71AFB12493D
:10BB200012482030FFF73EFB012110482030FFF77C
:10BB30008DFB10480C4948600020087201200870F5
:10BB4000002048720120887208483030FFF701FB5E
:10BB5000054906483030FFF725FB01210348303006
:10BB6000FFF774FB10BD0000582A00201055044058
:10BB700002040000DF070000F0B50B4614464360E6
:10BB80000481002136E0002216E02C254D43466852
:10BB90007519AD5C18274F430668F619B5542C2566
:10BBA0004D4346687519AD5C18274F430668F61972
:10BBB0000836B554551CEAB2082AE6D300251827E2
:10BBC0004F430668F619357418274F430668F6196F
:10BBD000757418274F430668F619B57418274F4334
:10BBE0000668F619F57418274F430668F61975614B
:10BBF0004D1CA9B205898D42C5DC00258572F0BDBA
:10BC000070B50446606800F09FFE0546E27A234660
:10BC10000C332946094800F05FFE094960688842F4
:10BC200003D0491C6068884206D1E17AA28890B2AC
:10BC300022460C3203F08AF870BD00005008002044
:10BC4000DF070000F8B5054600262C46002C2AD058
:10BC500000BF03E00020A055701CC6B2082EF9D327
:10BC600004F0A4FFC000082108400746206888436C
:10BC7000384320606068C000C0081249097849074D
:10BC8000490F49070843606004F090FF012801D183
:10BC9000082000E0002007061F2109060F40606809
:10BCA00088433843606007480088072805DA05485C
:10BCB0000088401C0349088002E0002001490880F8
:10BCC000F8BD00007C000020F8B5054600262C4693
:10BCD000002C4FD000BF03E00020A055701CC6B25E
:10BCE000082EF9D32448007B002809D12088000AB7
:10BCF000000220802088FF2109028843208015E06F
:10BD000005F062F892300004070E2088000A000255
:10BD10003843208005F058F892300002FF210902D4
:10BD20000840074620888843384320801248407BDB
:10BD3000002809D16088000A000260806088FF2125
:10BD400009028843608015E005F02EF99230000466
:10BD5000070E6088000A00023843608005F024F96D
:10BD600092300002FF21090208400746608888439C
:10BD700038436080F8BD00003828002070B50546C3
:10BD800000262C46002C48D000BF03E00020A05520
:10BD9000701CC6B2082EF9D305F022F9012817D17C
:10BDA0001E480088401C80B21C490880032804DB20
:10BDB00000201B490870194908803120207001209B
:10BDC00060705920A0700820E0700020207124E0ED
:10BDD00005F006F9022817D110480088401C80B2EF
:10BDE0000E490880032804DB00200D4908700B4928
:10BDF000088031202070012060705920A070082038
:10BE0000E0700120207108E00020044908802070C3
:10BE10006070A070E0700220207170BD7A00002078
:10BE2000F8000020FEB5054600260020019001F034
:10BE30002BFD074604F0EAFE0A210090FCF796F974
:10BE400080B201902C46002C3AD000BF03E00020C5
:10BE5000A055701CC6B2082EF9D3FF2109026068F4
:10BE60008843390C0902FF22120211400843606026
:10BE7000110260688843390A09041202114008431C
:10BE8000606060680002000A3906090E090608436E
:10BE9000606004F0AFFFFF2806DDFF210904206881
:10BEA0008843401820600BE004F0A4FF0004FF2149
:10BEB00009040840009020688843009908432060E6
:10BEC000FEBDFEB50546002600200190002704F0C7
:10BED00075FC64210090FCF749F980B201900020C4
:10BEE00001F0F4FC87B22C46002C1AD000BF03E00E
:10BEF0000020A055701CC6B2082EF9D3FF210904FA
:10BF00002068884339120904FF22120411400843B3
:10BF1000206020680002000A3906090E090608435D
:10BF20002060FEBDFFB581B004460F460025002607
:10BF3000002000902760039820810498E060002092
:10BF4000207400BF9DE01C206843216808586A01E6
:10BF5000616888501C2068432168081880686A015D
:10BF60006168891848601C20684321680818406887
:10BF70006A016168891888601C2068432168081874
:10BF8000C0686A0161688918C8601C20684321681C
:10BF90000818007C6A016168891808741C206843CD
:10BFA00021680818407C6A016168891848741C205F
:10BFB000684321680818807C6A0161688918888351
:10BFC0001C20684321680818C07C6A0161688918D0
:10BFD000887400206A0161688918C8741C2068434D
:10BFE000216808184068002813D01C206843216885
:10BFF0000818C07C002805D1401E6A0161688918B4
:10C00000C8831AE00020C0436A0161688918C883A8
:10C0100013E01C20684321680818C07C002805D064
:10C0200000206A0161688918C88306E000206A015F
:10C0300061688918C88301200090002607E000216C
:10C040006A016068801814308155701CC6B269019D
:10C0500060684018808BB042F1DC1C206843216886
:10C060000818406900280AD06B016268D21810468F
:10C0700014301C236B432268D21851698847681C0E
:10C08000C5B22089A84200DD5DE7009805B0F0BD8B
:10C0900000B58BB068480790002108A80170684679
:10C0A000017608A84170002064498872082108A818
:10C0B000C170002004E0002209A90A54411CC8B242
:10C0C00008A9C9788142F6DC5D48FFF742F806A965
:10C0D0005B48FFF767F85848401C0790002108A804
:10C0E00001706846017608A84170002053498872A3
:10C0F000082108A8C170002004E0002209A90A5400
:10C10000411CC8B208A9C9788142F6DC4C484030CD
:10C11000FFF71FF806A94A484030FFF743F84520CB
:10C1200000010790002108A801706846017608A860
:10C130004170002041498872082108A8C170002080
:10C1400004E0002209A90A54411CC8B208A9C97810
:10C150008142F6DC3A485030FEF7FBFF06A938482A
:10C160005030FFF71FF8112040010790002108A868
:10C1700001706846017608A8417000202F49887236
:10C18000082108A8C170002004E0002209A90A546F
:10C19000411CC8B208A9C9788142F6DC2848203081
:10C1A000FEF7D7FF06A926482030FEF7FBFF0B203D
:10C1B000C0010790002108A801706846017608A810
:10C1C000417000201D498872082108A8C170002014
:10C1D00004E0002209A90A54411CC8B208A9C97880
:10C1E0008142F6DC16486030FEF7B3FF06A914481A
:10C1F0006030FEF7D7FFFD20C000029000216846A6
:10C2000001730171417381730821C173002004E03F
:10C21000002204A90A54411CC8B26946C97B814264
:10C22000F6DC07481030FEF794FF01A904481030EF
:10C23000FEF7B8FF0BB000BDEE060000582A002044
:10C240008055044030B585B0044600252068019033
:10C25000A1796846C1726179417200210172017051
:10C2600000BF05E020460830415D03A841556D1C24
:10C270006846C07AA842F5D80B22D2010199881AE3
:10C28000914226D007DC1848081A1CD02321090146
:10C29000401A24D111E0FF386F38002802D001285D
:10C2A0001DD104E069461148FFF757F818E06946C8
:10C2B0000E484030FFF751F812E069460B48503005
:10C2C000FFF74BF80CE0694608482030FFF745F8C7
:10C2D00006E0694605486030FFF73FF800E000BF20
:10C2E00000BF05B030BD00002002000080550440B2
:10C2F000F0B585B004460F4600250026207C400698
:10C30000400E55287ED100BF76E169016068401873
:10C31000807C002877D169016068401840686A0114
:10C32000616889188968884209D269016068401883
:10C330004068C0196A016168891848605AE169015A
:10C3400060684018C068AF49884208D869016068D1
:10C350004018C068401C6A0161688918C86069019A
:10C3600060684018C07C002821D1002607E0002129
:10C370006A016068801814308155701CC6B269016A
:10C3800060684018808BB042F1DC1C206843216853
:10C390000818406900280AD06B016268D21810465C
:10C3A00014301C236B432268D218516988476901F5
:10C3B000606840580090690160684018017C6846D8
:10C3C000017100214171690160684018017F684670
:10C3D0008171690160684018417C6846C17100261E
:10C3E00008E06901606840181430815D02A8815539
:10C3F000701CC6B2690160684018808BB042F0DCE6
:10C40000E06801E0FCE01DE0002806D06846E16835
:10C4100088476A0161688918C874690160684018B2
:10C42000C07C002804D16A01616889184860E1E095
:10C430006901606840184068C01B6A01616889181A
:10C440004860D7E069016068401880680028EED035
:10C45000690160684018C08B0028E8D069016068F5
:10C460004018C08B6A0161688918C968884207D181
:10C47000690160684018C08B6249C94388427DD118
:10C4800069016068401840686A01616889188968B4
:10C49000884209D26901606840184068C0196A0181
:10C4A000616889184860A5E000206A016168891800
:10C4B0004860690160684018C0685249884208D8DD
:10C4C000690160684018C068401C6A016168891889
:10C4D000C860002607E000216A01606880181430F7
:10C4E0008155701CC6B2690160684018808BB042EB
:10C4F000F1DC1C20684321680818406900280AD034
:10C500006B016268D218104614301C236B432268FA
:10C51000D2185169884769016068405800906901E4
:10C5200060684018017C6846017100214171690111
:10C5300060684018017F6846817169016068401831
:10C54000417C6846C171002608E0690160684018B6
:10C550001430815D02A88155701CC6B26901606803
:10C560004018808BB042F0DCE068002808D06846B4
:10C57000E16888476A016168891800E015E0C874BD
:10C58000690160684018C07C002804D16A016168B4
:10C59000891848602EE06901606840184068C01B37
:10C5A0006A0161688918486024E01C20684321689A
:10C5B0000818406800280FD00020C0436A01616855
:10C5C0008918C8831C2068432168081840686A01DC
:10C5D00061688918886008E000206A01616889182C
:10C5E000C8836A0161688918886000206A016168EF
:10C5F0008918C860681CC5B22089A84200DD84E69D
:10C6000005B0F0BD0000FFFF7CB500BF19212C482C
:10C610000078FBF795FD04462A4860432A4A8118B2
:10C62000002201200CF0B6FF20460A22504364305D
:10C63000001981B2002201200EF0A6FF01200A227B
:10C6400062431219D1B20A22624312190090D0B289
:10C6500001231A4609F0B6FAFF220721002006F04E
:10C6600067FF0120009001900B20604382B20B20F5
:10C67000604381B2002301200EF0B6FC6F206043BE
:10C6800081B201200FF026FA1048604302460321D0
:10C6900001200BF0FDFC002505E0012128460BF0F0
:10C6A00031FC681CC5B20F2DF7DB21460B2251432C
:10C6B0006431C8B20FF072FC0FF05AFC7CBD000070
:10C6C00073000020672B0000A0860100FCB1010070
:10C6D000002005490870054908700549087005499A
:10C6E000087005490870704774000020750000202C
:10C6F000730000207200002071000020F0B589B0A6
:10C7000000BF00BF00BF00BF00BF00BF00BF00BF31
:10C7100000BF00BF5D4800783C2805DA5B48007820
:10C72000401C5A49087002E03C205849087057489C
:10C7300000781D2805DC56480078401C54490870D4
:10C740000BE053480078002802D15149087004E0FA
:10C750004F480078401E4E49087003214C4800782D
:10C76000FBF704FD4B4948430390052148480078F6
:10C77000FBF7E6FC0446032145480078FBF7F6FC8E
:10C780000B214843643080B20690414909788A0001
:10C7900088180621FBF7EAFCFF21F531484380B2F7
:10C7A000079003213A480078FBF7E0FC0B2148434F
:10C7B000643080B20890032135480078FBF7D6FC3E
:10C7C00035494843354940180490032130480078E2
:10C7D000FBF7CCFC0B2106464E4303212C48007886
:10C7E000FBF7C4FC0B2107464F4303212848007880
:10C7F000FBF7BCFC6F21484380B205900321012068
:10C80000039A0BF045FCE1B201200BF009FAE1B20A
:10C8100001231846069A09F0AFFCFF21F53107986D
:10C82000FBF7A4FCC0B20146029001200AF088F98F
:10C830000022012008990EF0A7FE00220120049991
:10C840000CF0A8FE012005990FF044F90120F9B27F
:10C850000090F0B201231A46029009F0B3F9FF22CA
:10C860000721002006F064FE032109480078FBF749
:10C870007DFC0B21484385B20120009000232A460D
:10C88000294601900EF0B0FB09B0F0BD7500002004
:10C8900074000020FCB10100672B0000A08601009D
:10C8A000002000BF06E00021044A1154044A11543C
:10C8B000411CC8B25A28F6DB704700004826002009
:10C8C000FC2600200348007A002801D10149487065
:10C8D00070470000580A0020FFB581B004460F469B
:10C8E0003D462089A8422DDD18206843216808189C
:10C8F000007C002826D1002609E00498815D1820DC
:10C9000068432268101808308155701CC6B2082E82
:10C91000F3D30121182068432268101841742C2099
:10C92000684361680818006A00280BD018236B431D
:10C930002268D218104608302C236B436268D21844
:10C94000116A884705B0F0BD01460720124BCA1A8C
:10C95000994211D008DCCA1FFA3A002A14D0102AD2
:10C960000CD01F2A14D10DE0322A0FD0C02A07D0D4
:10C97000C12A0DD100200DE001200BE0022009E0CA
:10C98000032007E0042005E0052003E0062001E085
:10C99000072000BF00BF70474103000010B50446E8
:10C9A0007D21C90061430846322103F0A9FE10BD74
:10C9B000FF200B4908700020C0430A4908800A493B
:10C9C0000880FF2009490870094908700949087062
:10C9D0000020094908600949086009490860704752
:10C9E000580000205A0000205C0000205E0000205B
:10C9F0005F000020600000204C000020500000205C
:10CA000054000020014800687047000050000020DA
:10CA100001480068704700004C00002010B505492F
:10CA200009886522514308466421FBF79FFB80B2C9
:10CA300010BD00005A000020014800787047000037
:10CA40005F00002001480078704700005800002077
:10CA500010B50FF0D9FF01282CD100F063F80120A8
:10CA600000F066F803F0B0FE044600F043F804F06E
:10CA7000ABF8044600F04AF804F0D4FA012805D1D6
:10CA800000F03EF8012000F047F805E0002000F03B
:10CA900037F8002000F040F80020134908601348E0
:10CAA0000068134988421ED210480068801C0F4954
:10CAB000086018E000200D4908600B4800680C4928
:10CAC000884204D208480068801C0749086000209A
:10CAD00000F028F8012000F02BF8002000F00AF800
:10CAE000002000F013F810BD500000204C00002082
:10CAF000FFFFFF7F01490880704700005A000020B7
:10CB000001490870704700005F000020014908805B
:10CB1000704700005C000020014908707047000069
:10CB20006000002001490870704700005800002094
:10CB300001490870704700005E0000200021014A92
:10CB40001171704700600040002201494A7570472A
:10CB500000600040002201494A76704700600040B2
:10CB60000021014A11727047006000400021014A13
:10CB700011737047006000400021014A1174704732
:10CB8000006000400021014A1175704700600040BC
:10CB90000021014A117670470060004000220149DF
:10CBA0004A73704700600040002201494A74704790
:10CBB0000060004010B51C4C1C49206888421ED102
:10CBC00006221B49201DFBF776FB002817D11122F6
:10CBD000184920460A30FBF76EFB00280FD10622C9
:10CBE000154920461B30FBF766FB002807D10622BB
:10CBF000124920462130FBF75EFB00280DD000F0E3
:10CC000089FE0A480E490860074813F004FF0C4AE1
:10CC10002821054813F02AFF04E02822214608486D
:10CC2000FBF725FB10BD0000000250007AA7A55AB3
:10CC30002D070020330700202707002021070020B0
:10CC4000642E00200020084908700849087001205F
:10CC5000074908700020074908700748074908601D
:10CC600000200749087070470F0700200E070020BA
:10CC700011070020160700202506000044070020A9
:10CC80002007002070B5044600BF91206043054690
:10CC90000A212846FBF754FA0546284670BD0000D5
:10CCA00070B5A8B0054600240026A0216846FBF711
:10CCB000F7FA00F09FFC1E490A681421694350509E
:10CCC00000211B480268142068431018416018486E
:10CCD00002681420684310188160154840680028D5
:10CCE00024D000BF17E06006060E282E00D316E001
:10CCF0000F480168142060430858B1006A4650503C
:10CD00000B4801681420604308184168701C8000BB
:10CD10001150601CC4B20648007AA042E3DC00BF98
:10CD200062000348694643680220984728B070BDF6
:10CD3000DC2E002030B5A9B000240025A02101A8D8
:10CD4000FBF7AEFA00BF25E06006050E00F052FCCE
:10CD50001F490A6814216143505000211C48026891
:10CD60001420604310184160194802681420604381
:10CD700010188160282D0BD21548016814206043DB
:10CD80000858A90001AA50500021681C80001150C9
:10CD9000601CC4B20E48007AA042D5DC0C48406842
:10CDA000002813D00A48007A4000282806D30848F3
:10CDB000282201A943680220984707E00448007A26
:10CDC0004200034801A943680220984729B030BDBA
:10CDD000DC2E002010B50FF017FE01287ED1FFF7E2
:10CDE00017FE5549884216D20F2054494871887160
:10CDF00008468078002801D1052048704F48807887
:10CE0000052802D100204D49487000204B49087286
:10CE10004872087035E0FA204849487188714849DD
:10CE2000088803F0F9FD4648807800280CD1434972
:10CE3000087008464079C87008468079087100205B
:10CE40008870487048721CE001203C490870084610
:10CE5000407A022805D1012048720020C87008716C
:10CE60000FE03648407A00280BD10220334948723F
:10CE700008464078887008464079C870084680792E
:10CE800008712E4880782D494978884213DD0020AA
:10CE90002A49C87008460079401C08710846007984
:10CEA0008979884222DB002024490871084680786D
:10CEB000401E88701AE021488078204949788842CD
:10CEC00014DA00201D4908710846C078401CC8705B
:10CED0000846C0784979884208DB00E01EE000205F
:10CEE0001649C87008468078401C887014488078BD
:10CEF000002803D10120114908721BE01048008866
:10CF0000732803DB02200D49087213E00C480088E7
:10CF100070280FDC0020094908720BE00020074947
:10CF2000087008464079C87008468079087100206A
:10CF30000872487210BD0000B80B0000B80900204C
:10CF4000800000200020044988704870C870087173
:10CF50000872487270470000B80900200020064996
:10CF600008808870054988704870FA20C870087178
:10CF7000002008724872704780000020B809002025
:10CF800070B503F051FC044603F060FC05460FF059
:10CF90003BFD01282ED105211A48FEF7CDF8552872
:10CFA00004D1002018498870088027E0012D04D1A1
:10CFB000002015498870088020E0012012498870FF
:10CFC0001248844202DB201A84B200E000240A21C5
:10CFD0002046FBF7CBF8052901DB601D84B20C4825
:10CFE000844200DD04460A212046FBF7BFF80649CB
:10CFF000088003E00020044988700880FFF7EAFEFB
:10D0000070BD00005008002080000020AA0A000027
:10D01000C60700001CB500200090019000F0EAFA5D
:10D020000B49086000200B49096808600A4800683D
:10D0300000280CD00749096808680A21FBF780F826
:10D040000090012269460520034B1B6898471CBDD0
:10D05000E0070020D4070020DC070020002008495A
:10D06000488008490880084908800849087008492C
:10D0700088720849088048800120087170470000C4
:10D08000300000202000002022000020240000208A
:10D090003408002028000020F8B503F0A7FB07465D
:10D0A00003F0B6FB0090FFF7CDFC012860D105210D
:10D0B000C548FEF741F8552802D00098012807D14D
:10D0C0000020C2490870C2490880C249887256E0EF
:10D0D000BE480078002810D10120BC4908703D46A8
:10D0E0002846E917890F091889030D0CBA488542AB
:10D0F00000DD0546B648058041E0B648807A40002C
:10D10000B4490F520846867A0EE07000B1490D5AB4
:10D11000701E4000085A7100AE4A5052701E400006
:10D1200011460D52701EC6B2002E08DD7000A949CE
:10D13000095A701E4000A74A105A8142E5DBA548F3
:10D14000807A401CA34988720846807A052816DB3D
:10D15000002088720846C5882846E917890F0918F3
:10D160008D109D48854200DD05469948058006E002
:10D17000002096490870964908809649887294481C
:10D18000058896480088A84257DA94480088281AEB
:10D1900084B292480079012827D190484088A04263
:10D1A0000BDA8E4840880A308C494880084640880F
:10D1B000A04204DD0846448001E088484480874856
:10D1C000448803212046FAF7D1FF84B2192C00DAF3
:10D1D0001924824800880019804908800846008880
:10D1E000A84201DD08460580CDE07C48408814282F
:10D1F00005DD7A48408814387849488002E00020EC
:10D20000764948807548448803212046FAF7AEFFE6
:10D2100084B2192C03DA012070490871B3E06F4819
:10D220000088A04205DD6D480088001B6B4908801E
:10D23000A9E0002069490880A5E068480088A84264
:10D2400059DD66480088401B84B264480079012893
:10D2500027D162484088142805DD6048408814388A
:10D260005E49488002E000205C4948805B48448871
:10D2700003212046FAF77AFF84B2192C03DA022040
:10D28000564908717FE055480088001953490880C5
:10D29000084600885049884275DD08464F49088095
:10D2A00071E04E484088A0420BDA4C4840880A3072
:10D2B0004A49488008464088A04204DD0846448028
:10D2C00001E0464844804548448803212046FAF757
:10D2D0004DFF84B2192C00DA19244048008829191E
:10D2E000884202DA3D4805804DE03C480088001B3A
:10D2F0003A49088047E03948448803212046FAF734
:10D3000035FF84B2192C3EDD34484088142805DDF1
:10D310003248408814383149488002E000202F49C3
:10D3200048802E48448803212046FAF71FFF84B224
:10D330002A480079012813D1192C03DA0220274941
:10D34000087120E025480088001924490880084613
:10D3500000882149884216DD08462049088012E0ED
:10D36000192C03DA01201D4908710CE01B480088C4
:10D37000A04205DD19480088001B1849088002E01A
:10D3800000201649088016480088502804DC1348FD
:10D3900000881349088016E0104800881049098861
:10D3A000884204DD0D4800880D4908800BE00B48D9
:10D3B00000880B490988081A84B2502C03DB0748FF
:10D3C000008807490880F8BD50080020240000208C
:10D3D0002000002034080020E02E0000280000205B
:10D3E0002200002010B5044664204443A1212046B9
:10D3F000FAF7A6FE0446204610BD00007CB50024C6
:10D4000000200190009000F03FFA05460A21FAF74B
:10D4100097FE044601226946042000F085FE00982C
:10D42000401C002814D17D20C0002018114908603C
:10D43000084600680190012201A9032000F0C0FE07
:10D440000120009001226946042000F0B9FE0FE09F
:10D45000009801280CD17D200001201805490860A2
:10D46000084600680190012201A9032000F0A8FEEF
:10D470007CBD00002801002010B501200F49087074
:10D4800000200F49096808600D49096848600C4987
:10D490000968886000F07EF9FFF7BCFDFFF74AFCE1
:10D4A00008480068002807D00122054801680831B3
:10D4B0000020044B1B68984710BD0000AD070020FA
:10D4C000A8070020A407002010B5184800681849D4
:10D4D000884229D117480068002804D01548006800
:10D4E00080471549087015480068002804D0134883
:10D4F000006880471249087012480068002804D06C
:10D5000010480068804710490880104800680028CB
:10D5100005D00E48006880470D49088002E00D489C
:10D520000B49088000F078F810BD0000B807002013
:10D530007856341294070020AC070020980700208A
:10D54000AE0700209C070020B0070020A0070020A5
:10D55000B20700201027000010B50023174C2360ED
:10D56000174C2370174C2370174C2370174C2380D3
:10D57000174C2380174C2370174C13682360174CEB
:10D5800053682360164C93682360164CD36823605D
:10D59000154C1369236000280CD0144B1860134CF1
:10D5A0000B682468A3600023104C246823600F4C90
:10D5B000246863600E4B014C236010BDB807002047
:10D5C000B4070020AC070020AE070020B007002001
:10D5D000B2070020AD070020940700209807002024
:10D5E0009C070020A0070020A4070020A807002017
:10D5F00078563412054800680549884203D1054829
:10D600000068806870470020C043FBE7B80700202F
:10D6100078563412A807002070B500240025002693
:10D620003048007801285CD12F480078002858D174
:10D630002E480078012854D12D4805882D490988A5
:10D64000694308462C49FAF77BFD85B2E1200001C9
:10D65000854207D81921694308460921FAF770FD68
:10D66000044600E0244C254800680068001923495E
:10D67000096808602148006800682049096849680D
:10D68000884207D31D48006800681C49096849683A
:10D69000461A0AE01948006840680021C943081A80
:10D6A0001649096809684018461C1548864218D36F
:10D6B000344601462046FAF743FD04460F48006809
:10D6C00041680F48604308180C4909684860012008
:10D6D0000C49087009480068806800190749096802
:10D6E000886070BDAC070020AD070020AE070020A9
:10D6F000B0070020B207002010270000A807002074
:10D70000A0860100B407002000220C4B1A600C4BCD
:10D710000A681A600B4B4A681A600B4B8A681A60D9
:10D720000A4BCA681A600A4B0A691A60002801D0BD
:10D73000084A1060084A014B1A607047B807002079
:10D7400094070020980700209C070020A0070020D5
:10D75000A4070020A80700207856341210B50A4804
:10D76000006800280ED00948007801280AD100205E
:10D770000649087001220648016808310020024B62
:10D780001B68984710BD0000A4070020B4070020C4
:10D79000A80700201CB50020009001900024FFF78E
:10D7A00029FF04460E480068046000200C490968FF
:10D7B00048600B49096888600A48006800280DD055
:10D7C00007480068006800900548006840680190BC
:10D7D000022269460120034B1B6898471CBD0000CC
:10D7E000BC070020C0070020F8B505460C461646C9
:10D7F0000027002D17D00E480560FFF7FBFE0746F7
:10D800002068B84203D90A480068076003E0084965
:10D81000206809680860064960680968486004492A
:10D82000A0680968C8600348066000F005F8F8BD04
:10D83000BC070020C007002070B500240025FFF7BA
:10D84000D9FE04460F4800680068A04200D903E0F2
:10D850000C4800680068251A0A48006840684019AA
:10D8600008490968886007480068806805490968B0
:10D87000C968884205D903480068C0680149096839
:10D88000886070BDBC070020014800688068704750
:10D89000BC070020002801D0024A1060024A116033
:10D8A00070470000BC070020C00700200549002089
:10D8B00005E00A1D135C044A1354421CD0B2202810
:10D8C000F7DB704700065000902E002001461048FC
:10D8D000026814204843101882680D480368142019
:10D8E00048431818C06882420BD9094802681420BE
:10D8F00048431018C26806480368142048431818A3
:10D9000082600348026814204843101880687047FA
:10D91000DC2E00200021002005E01A4A135C1A4A80
:10D920001354421CD0B20628F7DB1121002006E078
:10D93000164A135C144A921D1354421CD0B28842FA
:10D94000F6DB002006E0124A135C0F4A173213542C
:10D95000421CD0B20628F6DB002006E00D4A135C1C
:10D96000094A1D321354421CD0B20628F6DB0020AF
:10D9700005E00023044A23321354421CD0B201288C
:10D98000F7DB70472D070020682E002033070020AA
:10D99000270700202107002038B50446002000900A
:10D9A000009401226946052000F00AFC38BD000001
:10D9B00008B50020009001226946062000F0B4FB63
:10D9C000684600780C4908736846407848730846F2
:10D9D000007B0A4948730848407B88730648807B6F
:10D9E000C8730548C07B08740020087304480549C3
:10D9F00008600549086008BD38280020C4090020D7
:10DA000071170000840000208800002008B5002065
:10DA1000009001226946062000F086FB68460078E7
:10DA20000F49087368464078487300200D49086024
:10DA300048600872487288720948007B4873084839
:10DA4000407B88730648807BC8730548C07B087498
:10DA5000002008730448054908600549086008BDAE
:10DA600038280020C409002071170000840000201D
:10DA70008800002038B500240025002000900121F6
:10DA8000FE48FDF759FB55280AD002F023FFFC4958
:10DA9000487302F033FFFA4988730120087308E0E5
:10DAA000F848007BF6494873F648407B88730020AD
:10DAB0000873F348407B002804D1F1494873F249C8
:10DAC000086053E0EE48407B012829D1EE48006809
:10DAD000EE49884208D8EC480068401CEA490860D2
:10DAE0000120E749487341E0E648007B022812D054
:10DAF000E448007B03280ED00121E048FDF71CFB21
:10DB0000552803D00320DE4948732FE0DD48007B11
:10DB1000DB4948732AE0DB48007BD949487325E09C
:10DB2000D748407B02280FD10020D749086002F077
:10DB3000FBFE00281AD002F0F7FE401C002815D08A
:10DB40000220CF49487311E0CD48407B032806D11D
:10DB50000020CD4908600320C949487306E0002031
:10DB6000C9490860C748007BC5494873C448807BE1
:10DB7000002804D1C6490860C14988735CE0C048E8
:10DB8000807B012832D1C2480068C049884208D849
:10DB9000BF480068401CBE4908600120B84988732E
:10DBA0004AE0B748807C002801D1B94908600120CB
:10DBB000B3498874B348407B022812D0B148407BF7
:10DBC00003280ED00121AD48FDF7B6FA552803D041
:10DBD0000320AB4988732FE0AA48407BA84988738B
:10DBE0002AE0A848407BA649887325E0A448807BAA
:10DBF00002280FD10020A649086002F0B3FE0028D9
:10DC00001AD002F0AFFE401C002815D002209C491B
:10DC1000887311E09A48807B032806D100209C4934
:10DC2000086003209649887306E000209849086040
:10DC30009448007B924988739148407B9149097BC5
:10DC4000884205D18E48807B8E49497B88425FD0CF
:10DC50008B48407B8B49097B884202D00120884950
:10DC6000C8738748807B8749497B884202D001205E
:10DC7000834908748248407B022803D08048407B57
:10DC8000032803D17E48407B7E4908737C48807B13
:10DC9000022803D07A48807B032803D17848807B10
:10DCA000784948737648407B022803D07448407B0B
:10DCB000032812D17248407B7249097B88420CD0FC
:10DCC0007048017B684601706E48417B6846417030
:10DCD00001226946062000F073FA6948807B022819
:10DCE00003D06748807B032812D16548807B654953
:10DCF000497B88420CD06348017B684601706148CB
:10DD0000417B6846417001226946062000F058FABE
:10DD100002F0EAFD044602F0FDFD0546FEF792FE24
:10DD200001286ED101215548FDF706FA552807D183
:10DD30000020534908724872086048608872CCE03D
:10DD4000FF2C01D0FF2D6AD1FF2C2ED1FF2D2CD01E
:10DD500000204B490872012048724E4808604E4826
:10DD60006843486048686621FAF7EAF94449486020
:10DD7000084640684949884202D9084640494860F7
:10DD80003F48406832304649884206D33C484068A4
:10DD900032304149FA39884203D901203849887222
:10DDA0009BE000203649887297E0FF2C2ED0FF2D93
:10DDB0002CD1012032490872002048723548486051
:10DDC00035486043086008686621FAF7B9F92C49BC
:10DDD0000860084600683149884202D90846284947
:10DDE00008602748006832302D49884205D324480E
:10DDF000006832302B49884204D9012020498872BA
:10DE00006BE0A5E000201E49887266E023481C49AB
:10DE10000860486000208872087248725DE0012046
:10DE20001749087248721C486043086008686621F8
:10DE3000FAF786F9124908600846006817498842CF
:10DE400002D908460E490860134868430C494860E7
:10DE500048686621FAF774F909494860084640683D
:10DE60000E49884202D908460549486004480068BE
:10DE700032300B49884229D3014815E05008002070
:10DE8000C4090020382800208400002070170000FA
:10DE900088000020DE030000BE0A0000AC2600005F
:10DEA000A4060000FC080000006832302C498842BB
:10DEB0000CD82C48406832302B49884206D3294878
:10DEC000406832302649C831884203D901202549AB
:10DED000887202E00020234988722248407B002893
:10DEE00002D12049C87315E01E48407B012802D1A9
:10DEF0001C49C8730EE01B48407B022802D1194917
:10DF0000C87307E01748407B032803D11549C8733D
:10DF1000164808601348807B002802D11149087414
:10DF20001DE01048807B012802D10E49087416E0DC
:10DF30000C48807B022802D10A4908740FE0094886
:10DF4000807B03280BD1074908740848486006E025
:10DF5000002004490872487208604860887238BD21
:10DF6000FC080000C4090020A4060000AC26000044
:10DF7000FFB583B006460D461746002400200290E8
:10DF800000BF1420784380190190002E57D00198CB
:10DF9000002854D02B4806602A4906984860084655
:10DFA000077200BF45E0FFF725FB029020012958CA
:10DFB0000298814204D820012858401C002806D12C
:10DFC000204902980A6814216143505006E020015C
:10DFD00029581C4802681420604311502001401940
:10DFE0004068401C002807D1002116480268142010
:10DFF00060431018416008E0200140194168114851
:10E0000002681420604310184160200140198168A3
:10E010000C480268142060431018C16020014019A8
:10E02000017B084802681420604310180161601CDD
:10E03000C4B20448007AA042B5DC00F005F807B08D
:10E04000F0BD0000DC2E002070B500240025002665
:10E05000FFF7D0FA054600BF4EE02A4801681420B9
:10E0600060430858A84239D8264801681420604304
:10E0700008582E1A23480168142060430818406885
:10E0800081192048026814206043101881601D48DF
:10E09000016814206043081881681A480268142037
:10E0A00060431018C068814224D9164801681420C2
:10E0B000604308180069002803D02046FEF7F0FDF1
:10E0C00018E010480168142060430818C1680D4822
:10E0D000026814206043101881600BE00948016851
:10E0E000142060430818406806490A6814216143F7
:10E0F00051188860601CC4B20248007AA042ACDCAF
:10E1000070BD0000DC2E002010B500BF14244C436D
:10E110002318002805D0002B03D0024C2060626039
:10E12000217210BDDC2E0020F8B505460E461446BF
:10E130002B0011F0ABFF0705131A21282F363D00E5
:10E140001D48FAF70BFD1D4908701B48FAF7C0F887
:10E1500007466421F9F7F4FF30602AE0A004020CBE
:10E1600031461620FAF7F4FD23E0A004020C3146F4
:10E170004820FAF7EDFD1CE0A004020C3146802097
:10E18000FAF7E6FD15E0A004020C3146A020FAF7EC
:10E19000DFFD0EE0A004020C3146B020FAF7D8FDF6
:10E1A00007E06004020C3146C020FAF7D1FD00E020
:10E1B00000BF00BF0020F8BD2A280020E500002095
:10E1C00070B505460E4614462B0011F05FFF07059B
:10E1D0001D242B32393F46003068002802D1FAF75F
:10E1E0005BFB10E064223168514308461C49FAF792
:10E1F00079F800201B490870012264211848FAF7B9
:10E2000015FE1849087029E0A004020C31461620BA
:10E21000FAF75CFF22E0A004020C31464820FAF72E
:10E2200055FF1BE0A004020C31468020FAF74EFF98
:10E2300014E0A004020C3146A020FAF747FF0DE0DD
:10E24000A2B23146B020FAF741FF07E06004020CA9
:10E250003146C020FAF73AFF00E000BF00BF70BDB2
:10E260001C280020E400002000B5AFB050211BA8FE
:10E27000FAF716F800201A90142115A8FAF710F8EA
:10E2800000201290139014901190402101A8FAF7E9
:10E2900007F8002000905149086001221BA9FFF7F0
:10E2A00043FF1B98401C002801D11A9001E01B98E5
:10E2B0001A904B4815904B4816904B4817900020E9
:10E2C00018904A48199015AA1AA94948FFF744F925
:10E2D00002221CA90120FFF727FF1C98401C0028E0
:10E2E00001D1129001E01C9812901C98401C00284B
:10E2F00001D1139001E01D9813903E48149012A98B
:10E300003D48199AFFF770FA08221EA90220FFF76C
:10E310000BFF1E98401C002801D1019001E01E98BF
:10E3200001901F98029035480390012069460874B7
:10E33000801E059032490791012101A80177881EAE
:10E3400009902F490B91012109A80173881E0D9096
:10E350002B490F9101210DA80173042201A929481D
:10E36000199BFFF705FE01221BA90320FFF7DCFE26
:10E3700025491B9808601B98401C002806D1FF20E7
:10E38000F530086001220320FFF71AFF01221BA9C4
:10E390000520FFF7C9FE1B98401C002807D101206B
:10E3A0001A498860012208310520FFF709FF012280
:10E3B0001BA90620FFF7B8FE1B98401C002808D1B7
:10E3C0000021684601704170012269460620FFF76E
:10E3D000F7FE0F48014908602FB000BDE80000209B
:10E3E00045CA000039CA00001DCA0000C1E1000092
:10E3F000B027002076841E00BC2700200F270000D5
:10E400009F860100CC27002028010020382800200A
:10E41000A33AA55A00B585B014216846F9F740FF24
:10E4200000200F4908600F4800900F4801900F48E6
:10E430000290002003900E48049069460D48FFF7B3
:10E4400063F90D480499FFF725FA04210B48049A53
:10E45000FFF75AFE0A480249086005B000BD0000F7
:10E46000E800002045CA000039CA00001DCA0000AB
:10E47000C1E10000B0270020BC270020CC270020ED
:10E48000A33AA55A00200C4908800C4908800C4981
:10E49000088001200B49087000200B4908730B49C4
:10E4A00008804880012008710020074948800880C2
:10E4B0000749086070470000380000203A0000203B
:10E4C00040000020420000204008002044000020BE
:10E4D0003C000020F8B502F0C3F9064602F0CAF984
:10E4E0000746FEF7AFFA012865D10521AB48FCF7D6
:10E4F00023FE552807D10020A9490870A9490880A2
:10E50000A94988805FE0012F07D10020A449087045
:10E51000A4490880A449888055E0A14800780028D3
:10E5200008D101209E49087035460A2068439D495C
:10E53000088048E09C48007B42009B48801D865232
:10E54000801F047B11E061009748801D455A601EC2
:10E5500041009548801D415A62008152601E410071
:10E560009148801D4552601EC4B2002C0ADD610036
:10E570008D48801D415A601E42008B48801D805A84
:10E580008142E0DB8848007B401C874908730846CD
:10E59000007B032807DB00200873084605890A2052
:10E5A0006843804908807F4800887F49888001202F
:10E5B0007B49087007E00020794908707949088094
:10E5C00079490873888077480088784908607448DA
:10E5D0000078002815D0084600686C21484373492C
:10E5E0000860642171480068F9F7AAFD6F49086066
:10E5F000084600686E49884206D908466B4908609B
:10E6000002E0002069490860684800686949098893
:10E61000884203D2654800680F2804D26348008806
:10E62000644908800AE06348008860490968401A24
:10E630000F2803D35D4800885E4908805A48008847
:10E64000401C59490880084600880A282CDB002015
:10E6500008805948008857490988884203DA012010
:10E660005649087108E05448008852490988884290
:10E6700002DD02205149087150480079012840D13B
:10E680004C4800884C49098888420DDB494801887C
:10E6900049480088FF309130814206DD46480088B5
:10E6A000FF3073304449088077E04248018842488F
:10E6B00000889630814205DD3F48008878303E4929
:10E6C00008806AE03B4801883B480088323081423C
:10E6D00005DD394800881E30374908805DE035483F
:10E6E0000188354800880A30814205DD32480088BB
:10E6F0000A303149088050E02E4800882E490880B1
:10E700004BE02E480079022847D12A4800882A4940
:10E710000988884239DA27480088FF309130264935
:10E720000988884206DA24480088FF38733822496D
:10E7300008802AE01F48008896301F4909888842CF
:10E7400005DA1D48008878381B4908801DE0194803
:10E750000088323018490988884205DA164800884E
:10E760001E381549088010E0124800880A30124906
:10E770000988884205DA104800880A380E4908805E
:10E7800003E00C4800880C4908800B4800880849C1
:10E79000884202DB084608490880F8BD500800207E
:10E7A0004200002038000020400800203C000020EB
:10E7B000C6070000400000203A000020440000206E
:10E7C00000200849088008490880084908804880D6
:10E7D000012008710020064948800880054908602A
:10E7E000704700003A000020400000204400002054
:10E7F000400800203C000020002004490870044923
:10E800000870002103480176704700008C0000204A
:10E810008D000020380A002070B500250024FEF786
:10E8200011F9012863D103213448FCF785FC5528F0
:10E8300008D100203249087032490870002132485E
:10E84000017659E02F480078002807D102F0A8F897
:10E850002B49087001202B4908704DE001202949FF
:10E86000087002F09DF82849097E8900264A603A1E
:10E8700050502548047E10E0A000234960390D5C0B
:10E88000601E80000858A1001F4A603A5050601E68
:10E89000800011460D50601EC4B2002C0ADDA0009D
:10E8A000194960390958601E8000174A603A1058AB
:10E8B0008142E1D31448007E401CC1B21248017667
:10E8C000007E1E2818DB00210F48017601466039C2
:10E8D000896B0246603AD26B89180246603A126C24
:10E8E00088180321F9F72CFC0549087004E0002082
:10E8F000034908700349087070BD000050080020EB
:10E900008C0000208D000020380A0020F0B5A9B04E
:10E9100004460E460025002700202890A0216846C6
:10E92000F9F7BEFCFEF766FE26490A68142161432A
:10E93000505024480168142060430818C068B04251
:10E940000CD220480168142060430818C1681D4893
:10E950000268142060431018416005E019480168FE
:10E96000142060430818466016484068002826D0E6
:10E97000002517E06806070E282F00D316E011487F
:10E980000168142068430858B9006A4650500D4881
:10E9900001681420684308184168781C80001150F1
:10E9A000681CC5B20748007AA842E3DC00BF6A00D1
:10E9B0000448694643680220984701202890289817
:10E9C00029B0F0BDDC2E002010B500F0F5FD00F000
:10E9D000D7F810F075FA00F00DFB00F001F810BD4B
:10E9E00070B541480078912800D070BD00F0BEF8A5
:10E9F000012876D13D4800883D4908800846807846
:10EA0000F021884320303A49887008468078000910
:10EA100000013549097A0907090F0843344988700C
:10EA20003148807A401E3049887208460089401C6F
:10EA3000088108460089C988884216DA08202C49CE
:10EA4000887200240EE0284841882848001D415C57
:10EA50002748C01C015524484088401C2249488052
:10EA6000601CC4B2072CEEDB2DE01F4800891E4954
:10EA7000C98888421CD11C4800791B498978401AF2
:10EA8000C5B2681C1A49887200240EE016484188F5
:10EA90001648001D415C1648C01C015512484088AC
:10EAA000401C11494880601CC4B2AC42EEDB0AE055
:10EAB00000F00EFD00200C4908700C49088809215F
:10EAC00000F0B8F991E7012000F0C4FC084A917AFF
:10EAD0001088921C00F070F905490888002100F0A8
:10EAE000C1F800BF81E70000182C0020B42B0020E3
:10EAF000442B00201B49097E002932D01949897E08
:10EB00000C225143174A515A174A118000200CE039
:10EB10001449897E0C225143124A8918891C0A5CC7
:10EB20001149891C0A54411CC8B20828F0DB0D4960
:10EB3000897E0C2251430B4A8918897A0A4A9172BC
:10EB40000121D1720749097E491E064A11761146F4
:10EB5000897E491C91761146897E022901DB0021BC
:10EB600091767047102B0020382B00200349487BFA
:10EB7000012802D10021014A51737047282C00203E
:10EB800010B533484068002861D13148007B03004C
:10EB900011F07CFA07590512212E3D4A59002D48E3
:10EBA0000078002807D000202A4908702A490888E0
:10EBB000012100F03FF947E026480078002809D0FD
:10EBC00000202449087025494A8808880123091D26
:10EBD00000F040F938E01F480078002807D00020F6
:10EBE0001C4908701C490888022100F023F92BE019
:10EBF00018480078002809D00020164908701749E5
:10EC00004A8808880923091D00F024F91CE01148EE
:10EC10000078002807D000200E4908700E490888A7
:10EC2000092100F007F90FE00A480078002809D010
:10EC300000200849087009494A8808880323091DEB
:10EC400000F008F900E000BF00BF00F041FC10BD7B
:10EC5000282C0020182C0020B42B0020502B002042
:10EC60007047000070B504460D4634480088A04245
:10EC700063D1002D61D13248007822284ED004DCC7
:10EC800020283DD0212856D141E0902802D091285B
:10EC900051D115E02A48C08801280AD1002028490E
:10ECA000087000F015FC27490888002100F0C2F820
:10ECB00005E0032000F0CEFBA020214908703BE0D6
:10ECC0001F4800891E49C98888420AD100201C4972
:10ECD000087000F0FDFB1B490888002100F0AAF82D
:10ECE0000DE01748807A002806D000F0F1FB1449A7
:10ECF000087B00F091FB02E0032000F0ABFB1BE07F
:10ED0000062000F0A7FB11200D49087014E0062032
:10ED100000F0A0FB11200A4908700DE0002008490E
:10ED2000087000F0D5FB08494A8808880923091DA6
:10ED300000F090F800E000BF00BF70BD2C2B002059
:10ED4000182C0020B42B0020502B002070B5034657
:10ED5000184C247E022C00DB70BD164C647E0C2502
:10ED60006C43144D2B5300200AE0155C114C647E5B
:10ED70000C2674430F4EA419A41C2554441CE0B265
:10ED80008842F2D30B4C647E0C267443094EA419BE
:10ED9000A1723446247E641C35462C762C46647E53
:10EDA000641C6C762C46647E022C01DB00246C769D
:10EDB00000BFD1E7102B0020F0B585B007460D4607
:10EDC00016461A480780002406E031781748801C50
:10EDD0000155761C601CC4B2AC42F6DB2C4605E043
:10EDE000AA211248801C0155601CC4B2082CF7DB14
:10EDF0000E480088019008216846C17200214172C6
:10EE000001720170002406E00848801C015D03A81F
:10EE10000155601CC4B2082CF6DB69460448FCF7B7
:10EE20009CFA01200149887205B0F0BD2C2B00200E
:10EE30009055044070B504460D46294620460FF013
:10EE400061FF70BD70B504460D46294620460FF09F
:10EE500067FF70BDF8B504460D4616461F463B4693
:10EE60003246294620460FF05CFFF8BDF8B507464C
:10EE70000E4615465C480078002804D00921384623
:10EE8000FFF7D8FFF8BD002D01D0602D04DD09216A
:10EE90003846FFF7CFFFF5E7544807804580002448
:10EEA00006E031785148001D0155761C601CC4B243
:10EEB000AC42F6DB00204C49487008468580FF20B4
:10EEC00088727F2008730846808808282EDA01207F
:10EED000C88008468088488001200881434800880F
:10EEE0004349088008468078F0218843404988706B
:10EEF00008468078000900013B4909790907090F94
:10EF000008433B49887038480079401C88720024C7
:10EF100007E03648001D015D3548C01C0155601CE6
:10EF2000C4B231488088A042F3DC4AE00721681C63
:10EF3000F9F71CF9002907D0072128460830F9F70E
:10EF400015F92949C88005E00721681CF9F70EF971
:10EF50002549C8800620244948800120088123488B
:10EF600000882349088008468078F02188431030C3
:10EF70001F49887008468078000900011A4989886D
:10EF80000905090F08431A49887008464088FF217F
:10EF900009028843144989880902FF22120211409C
:10EFA00008431349488008208872002407E00F486E
:10EFB000001D015D0E48001D0155601CC4B2062CE9
:10EFC000F5DB012000F046FA094A917A1088921C7C
:10EFD000FFF7F2FE902004490870054908880021D7
:10EFE000FFF740FE00BF4DE7182C0020B42B002097
:10EFF000442B002010B5FFF77DFD1448C07A00288F
:10F0000022D0124880780009002806D0012807D0B5
:10F0100002280AD0032810D10CE000F0A5F90FE077
:10F0200000F09EF800F062FA0AE000F011F800F03B
:10F030005DFA05E000F000F902E0FFF711FE00BF05
:10F0400000BF00200149C87210BD0000382B00200D
:10F0500010B540480078112800D010BD3E48008807
:10F060003F214901884200D0F7E73B4880780007FC
:10F07000000F3849097A0907090F88420CD000208F
:10F080003449087000F024FA34494A880888042377
:10F09000091DFFF7DFFEE0E72E480089401C2D49DF
:10F0A00008810846807A401E887208460089C9880F
:10F0B00088421BDA2848807A082800D0CDE700244F
:10F0C0000EE02548C01C015D224842882348001DEF
:10F0D000815420484088401C1E494880601CC4B2AE
:10F0E000072CEEDB062000F0B5F930E019488088E7
:10F0F00018494988401A1849897A884203DA16481B
:10F10000807A082800D0A8E700240EE01248C01C2E
:10F11000015D104842881148001D8154601CC4B232
:10F120000C484088401C0B4948800A4840880949DF
:10F1300089888842EADB00200649087000F0C8F997
:10F1400006494A8808880023091DFFF783FE00BF8F
:10F1500083E70000182C0020382B0020502B0020C3
:10F1600070B53248007880210840802800D170BDF9
:10F170002F4800883F214901884200D0F7E72C48FA
:10F18000807A082800D0F2E72948807805072D0FFB
:10F190002D0227484088000A0543082D00DAE6E7DB
:10F1A00000202249487006204880084685800120BA
:10F1B0000881082088720020C8728988481C0721AD
:10F1C000F8F7D4FF002909D0184989880846083083
:10F1D0000721F8F7CBFF1549C88007E01349898854
:10F1E000481C0721F8F7C2FF1049C8801048008862
:10F1F0001049088008464580002407E00C48001D9F
:10F20000015D0C48001D0155601CC4B2062CF5DBE5
:10F21000042000F01FF9102004490870054A5188A5
:10F220001088FFF70FFE00BFA1E70000182C002098
:10F23000382B0020502B002010B548480078A0281B
:10F2400008D046480078912804D044480078A12886
:10F2500000D010BD424800883F21490188420AD0B1
:10F26000404908880921FFF7E5FD00F031F9002049
:10F270003A490870EDE73A48807A08280AD03949B7
:10F2800008880921FFF7D6FD00F022F90020334954
:10F290000870DEE7324880780007000F002804D0AD
:10F2A00001282DD002284BD136E02C484078002888
:10F2B00000D050E02A48C078002803D10120274917
:10F2C000487003E02648C0782449887223480078B3
:10F2D00091280BD022480079002803D101201F4932
:10F2E000087303E01E4800791C49087391201B49EC
:10F2F000087000F0EDF81949087B00F08DF82AE05D
:10F3000016484078002800D025E0A1201349087055
:10F31000032000F09FF81EE010484078002800D03D
:10F3200019E00E480078A02809D10E490888082164
:10F33000FFF780FD00F0CCF80020084908700AE0D3
:10F34000084908880521FFF775FD00F0C1F8002085
:10F350000249087000BF00BF00BF7AE7182C0020E8
:10F36000382B0020B42B002010B5284800788021CD
:10F370000840802800D110BD24480078002806D01D
:10F38000234800883F214901884200D0F3E7204804
:10F39000807A1F4989780907090F884203DD1C48D4
:10F3A000807A082800D0E6E7194880780007000F27
:10F3B000002805D0164880780007000F072800DDD8
:10F3C000D9E713480088134908801148807800075E
:10F3D000000F4880002407E00D48C01C015D0D4867
:10F3E000001D0155601CC4B20A484088A042F3DCED
:10F3F00000200649087000F06BF806494A88088822
:10F400000023091DFFF726FD00BFB4E7182C0020DC
:10F41000382B0020502B00207F2805DC7D21C900DF
:10F4200041430A4A91600DE0F12808DBF92806DC27
:10F430000107090F64225143044A916002E0044924
:10F44000024A91600221014A51737047282C002022
:10F4500018F0010000B5030010F018FE0729050B95
:10F4600011171D2329000121144A117314495160F9
:10F4700022E00221114A1173114951601CE003215D
:10F480000E4A11730F49516016E004210B4A1173A3
:10F490000D49516010E00521084A117300215160A7
:10F4A0000AE00621054A11730849516004E0002171
:10F4B000024A1173516000BF00BF00BD282C00201C
:10F4C000A8610000F824010028230000F049020090
:10F4D0000020014908737047282C00200249098840
:10F4E0000918014A11807047282C002010B52F48B8
:10F4F0000078102818D12E48408860280ADD2D4851
:10F50000807800090001801C2A4988702220274940
:10F51000087025E027488078000900012549887097
:10F520002020224908701BE020480078112816D1BD
:10F530001E48807A002800D010BD1C484078002862
:10F5400000D0F9E70820194988721A488078000924
:10F5500000011849887020201449087000E0EBE78A
:10F56000FD20C0001349088008468078F0218843B8
:10F570003030104988700846C0780020C8700846AE
:10F58000007914200871032088720220FFF762FFBF
:10F59000084A917A1088921CFFF70EFC05490888EA
:10F5A0000021FFF75FFB00BFC6E70000182C00201A
:10F5B000502B0020442B0020244A118852888A4274
:10F5C00042D0224A52888A4204DA204A52888A1A51
:10F5D00090B207E01D4A52880023DB439A1A521C5E
:10F5E000521890B2194A5180127B002A10D0174A43
:10F5F0005268002A0CD0154A5268824205D9134A33
:10F600005268121A114B5A6002E000220F4B5A60E6
:10F610000E4A527B022A17D10C4A9268002A0CD05B
:10F620000A4A9268824205D9084A9268121A074B20
:10F630009A6002E00022054B9A60044A9268002A10
:10F6400002D10122014B5A7370470000282C002080
:10F6500010B506F07DF810BD00BF704710B5044628
:10F660008020204301460320400205F02BFF10BDFF
:10F6700010B510210320400205F024FF10BD00004A
:10F6800010B50224024805F06DFF0446204610BD67
:10F690000106000010B50021014805F013FF10BD60
:10F6A0000106000010B504468020204301460248B0
:10F6B00005F008FF10BD00000106000010B5102184
:10F6C000014805F0FFFE10BD0106000030B50346FD
:10F6D0000C46002101250D48834201D0002B01D1A9
:10F6E000022030BD012A01D10120FAE7002108E003
:10F6F000C8002058984202D100252846F1E7481C4E
:10F7000081B29142F4DB2846EBE70000FFFF0000E6
:10F71000002000BF14E00021C200134B9950C2002A
:10F72000D2189180C200114B9950C200D21891801A
:10F73000C2000F4B9950C200D2189180411C88B270
:10F740004828E8DB0B490C4A11600C495160002144
:10F7500091600B4911610B49D16000210A4A118067
:10F760000A4A117070470000881F0020C82100203D
:10F77000082400202D0C0100741F0020C90C01007A
:10F78000730D0100650D0100D6000020DA00002095
:10F79000F0B585B00646674F3846039002900025C5
:10F7A000002400200190009063480068002803D0E6
:10F7B00061490868804707465F484068002803D0D1
:10F7C0005D494868804703905B488068002803D003
:10F7D000594988688047029057480069002803D03B
:10F7E00055490869804700905348C068002803D0F5
:10F7F0005149C86880470546482D00DD48250098D6
:10F80000002876D0002D74DD4C480088A8420BDA21
:10F810002B463A4649494A48FAF760FF2B46474982
:10F820004748039AFAF75AFF44480088002833DD16
:10F8300042480088A84202D10020404908800024A4
:10F8400015E0E0003F490858E1003D4A5158884220
:10F850000BD0E00011460858E1003A4A5050E00051
:10F8600011460858E100384A5050601C84B2AC423E
:10F87000E7DB0120354908702C460BE00020E10051
:10F88000314A5050E1002F4A5050E1002C4A50506C
:10F89000601C84B2482CF1DB2B4800682549884263
:10F8A00046D0294880882A49884205DA2648808837
:10F8B0008019254988803BE000202349888008463C
:10F8C00000680190012D33DD002408E0601CC000B9
:10F8D0001D490858E1001C4A5050601C84B2681E43
:10F8E000A042F3DC691EC900174A019850501FE07E
:10F8F000FFE7002015490870002414E00020E10013
:10F90000114A5050E10089188880E1000C4A50509B
:10F91000E10089188880E1000A4A5050E100891806
:10F920008880601C84B2482CE8DB002003490880F2
:10F9300005B0F0BDFFFF0000741F0020D6000020BE
:10F94000C821002008240020881F0020DA000020A1
:10F95000881300002E480078401C2D4908702D485F
:10F960000078401C2B4908702B480078401C2A491D
:10F9700008702A480068401C28490860084600684A
:10F98000FF219131884202D9002024490860204893
:10F990000078C82802D900201D4908701D48007849
:10F9A000842802D900201B4908701B480078502881
:10F9B00002D9002018490870194818490968405CA4
:10F9C00018490870184812490978405C17490870AE
:10F9D000174810490978405C1649087016480E49C6
:10F9E0000978405C15490870154809490978405C58
:10F9F00014490870144806490978405C1349087096
:10FA0000134803490978405C1249087070470000A8
:10FA100053070020540700205507002058070020F6
:10FA2000EF1502004C0700207F1702004D07002051
:10FA3000471802004E0700209319020050070020CB
:10FA4000CB1802004F070020E319020051070020E5
:10FA5000AB1A02005207002010B58200054BD218E5
:10FA6000525C012A04D100228300024C1B195A5413
:10FA700010BD0000942A002010B50446204600F076
:10FA80004FFA204600F002F810BD000010B5044601
:10FA9000B248007800287DD1B1480088B149884239
:10FAA00078DAB148007800284FD0B04800780028B4
:10FAB00003D0AB480088AE490880AE4800780028E3
:10FAC00018D1A7480188AA4800880F30814206D380
:10FAD0000120A8490870A2480088A5490880A048CC
:10FAE0000088A349098888421CDA9D480088A049FB
:10FAF000088017E09E480188994800880F308142AD
:10FB000006D300209B4908709548008898490880D2
:10FB10009348008896490988884203DD9048008808
:10FB20009349088093480078002857D1924800787C
:10FB3000042803D08D480078002807D08848008822
:10FB4000822803DA05208C490870A1E08A480078F1
:10FB5000032803D085480078002809D08048008811
:10FB6000FF211931884203DA0420834908708FE0AD
:10FB700081480078022803D07C48007800280AD009
:10FB800077480088FF21AF31884204DA03207A49A0
:10FB900008707DE0E0E078480078012803D07348E1
:10FBA0000078002808D06E4800887449884203DA3B
:10FBB0000220714908706BE06F480078002803D07C
:10FBC0006A480078002863D0654800886B49C831CE
:10FBD00088425DDA01206849087059E0654800787C
:10FBE000012855D164480078012803D05F48007887
:10FBF000002809D05A4800886049C831884203DB90
:10FC000000205D49087043E05B480078022803D07B
:10FC100056480078002808D0514800885749884243
:10FC200003DB01205449087032E053480078032870
:10FC300003D04E480078002809D049480088FF21A9
:10FC4000AF31884203DB02204B49087020E04A486C
:10FC50000078042803D045480078002809D040489F
:10FC60000088FF211931884203DB032042490870D4
:10FC70000EE041480078052803D03C480078002871
:10FC800006D037480088822802DB04203A490870F1
:10FC9000FCF7BEFE3349643988425DD338480068BA
:10FCA00000193749086031480078002808D0002042
:10FCB0002E490870324908602F4800783149087091
:10FCC00000F082FD00281FD12D4800682E4988428F
:10FCD00039D300202A4908602A4800782649097843
:10FCE000884205DA27480078401C264908702AE037
:10FCF0002448007820490978884224DD214800788A
:10FD0000401E204908701EE01D4800681F498842B7
:10FD100019D300201A4908601A4800781649097852
:10FD2000884205DA17480078401C164908700AE036
:10FD30001448007810490978884204DD1148007899
:10FD4000401E104908700F4800780B490978884216
:10FD500002D100200A49086010BD00000B000020FD
:10FD6000020000201C0C00001200002008000020EF
:10FD7000040000200A00002006000020C602000047
:10FD80001800002007000020C05D0000407E050034
:10FD900000200B4908700B49087001200A490870BF
:10FDA0000A49087000200A4908700A4908700A497F
:10FDB00008800A4908800A4908800A490870704783
:10FDC0000600002007000020080000200900002095
:10FDD0000A0000200B0000200C0000200E00002074
:10FDE000100000201200002000200B4908700B4971
:10FDF000087001200A4908700A49087000200A4961
:10FE000008700A4908700A4908800A4908800A49A6
:10FE100008800A490870704706000020070000208B
:10FE200008000020090000200A0000200B0000202C
:10FE30000C0000200E000020100000201200002006
:10FE4000F1B5002730480078002809D00320F9F7E1
:10FE500085FB002804D00320F9F774FB2B490880A8
:10FE60002B4800880A2847D30020294908802948C0
:10FE70000078282829D20320F9F764FB07460024DC
:10FE800007E060002449085AB84200DD05E0601C24
:10FE9000C4B2204800788442F3DB00BF1D480578D7
:10FEA00008E0681E40001C49085A69001A4A50526E
:10FEB000681EC5B2A542F4DC600017490F52154810
:10FEC0000078401C1349087016E000260F2405E056
:10FED00060001149085A8619601CC4B2192CF7D366
:10FEE0000A213046F8F72CF9084908800020094912
:10FEF0000870012009490870054801880098081811
:10FF000003490880F8BD000009000020020000201D
:10FF10001600002000000020E4070020120000204E
:10FF20003A4909881E2928DA0021394A1180394ABC
:10FF3000118039490988394A914207DC38490978E2
:10FF4000002914D034490988914210DD0121354A35
:10FF500011700021344A1170344A1170304A117006
:10FF60000121334A11700021324A11704CE02A49B4
:10FF700009880918284A118046E024490988274A37
:10FF8000643291422BDB0021234A1180214A1180E7
:10FF90001F490988AF221201914207DC20490978E4
:10FFA000002916D01A490988914212DD02211D4A02
:10FFB000117000211C4A117005211C4A117000218A
:10FFC000174A117001211A4A11700021194A117043
:10FFD0001AE00F49098809180D4A118014E0002120
:10FFE0000D4A11800A4A11800A4909880B4A914238
:10FFF00005DD00210B4A1170094A117004E0054922
:020000040001F9
:1000000009880918034A1180704700000200002087
:10001000100000200C0000200E000020B80B000093
:10002000090000200B00002006000020070000202F
:10003000080000200A0000200148007870470000F6
:10004000B80900200148007A70470000B809002074
:100050000148807870470000B809002001480088F6
:100060007047000080000020F8B5002300250095AF
:100070000024002200BF94E001259D40ACB20D8811
:1000800025400095009DA5426FD11A468D79012D1E
:100090000DD1464D03263602AD192D5C0126964042
:1000A0003543424E03273F02F61935540CE03F4DCD
:1000B00003263602AD192D5C01269640B5433B4E12
:1000C00003273F02F6193554CD78002D4ED1374D18
:1000D00060352D5CCE78002E01D1012600E000268F
:1000E0009640B543314E603635548D78002D2ED173
:1000F0002E4D19267601AD192D5C8E78002E01D17A
:10010000012600E000269640B543284E19277F01BE
:10011000F61935540D79002D0ED1244D50352D5C36
:100120000E79002E01D1012600E000269640B5434D
:100130001E4E5036355423E01C4D50352D5C0E7943
:1001400096403543EEB2194D50352E5418E0174DF8
:1001500019267601AD192D5C8E7896403543134EE5
:1001600019277F01F61935540AE018E00F4D603564
:100170002D5CCE7896403543EEB20C4D60352E5452
:100180004D79012D0AD1094D30352D5C012696405F
:100190003543EEB2054D30352E5400E000BF5D1CF6
:1001A000ABB2082B00DA67E7F8BD0000000004409E
:1001B000FFB5074615461E4600243846019900F053
:1001C0001FF8002802D0012004B0F0BD00240CE08C
:1001D0000A2060430949085CB04204D12946204600
:1001E00000F05EF807E0601C84B20A206043034917
:1001F000085C0028ECD100BF0020E5E7AC0100203E
:100200000246002A03D1402901DD01207047032A5C
:1002100003D1022901DD0120F8E7042A03D12029B6
:1002200001DD0120F2E7052A03D1202901DD0120AB
:10023000ECE70C2A03D1102901DD0120E6E70D2AA5
:1002400005D1012903DD402901DA0120DEE70E2A6C
:1002500003D1202901D10120D8E70020D6E70000F2
:1002600010B5064A03231B02D218125C8A43034BC3
:10027000032424021B191A5410BD0000000004407E
:1002800010B5064A03231B02D218125C0A43034B23
:10029000032424021B191A5410BD0000000004405E
:1002A00070B502460020B1E00A2353435A4C1B1993
:1002B0005B1C440004191B199B788B427DD10A23D7
:1002C0005343554C1B195B1C440004191B195B78E4
:1002D000082B33D10A2353434F4C1B195B1C44009A
:1002E00004191B574D4C4E4D6419E35C0124234304
:1002F0000A245443484D6419641C45004519645749
:10030000464D474EAD192B550A235343424C1B19FA
:100310005B1C440004191B57404C35466419E35CD0
:10032000022423430A2454433B4D6419641C4500B2
:1003300045196457394DAD192B5564E00A235343D1
:10034000354C1B195B1C440004191B195B78092BE5
:1003500034D10A235343304C1B195B1C440004194D
:100360001B572E4C2E4D6419E35C402423430A2472
:100370005443294D6419641C450045196457274DA1
:10038000274EAD192B550A235343234C1B195B1CD5
:10039000440004191B57214C35466419E35C802442
:1003A000A3430A2454431C4D6419641C4500451999
:1003B00064571A4DAD192B5525E025E00A23534308
:1003C000154C1B195B1C440004191B57134C144D8E
:1003D0006419E35C0A2454430F4D6419641C4500FE
:1003E0004519641965780124AC402343DCB20A2323
:1003F0005343094D5B195B1C450045195B57074D7D
:10040000074EAD19EC5404E0431CD8B2032800DABF
:100410004AE700BF70BD0000AC01002000000440AE
:1004200075080000F8B50024FCF70CFB012861D129
:1004300000F082FB0446FF220721002003F078F839
:10044000012C21D100F098FC00280ED000F0A8FB70
:10045000054600F099FB0646012003460246294660
:100460000090304605F0AEFB50E000F099FB0546E9
:1004700000F08AFB06460120002302462946009030
:10048000304605F09FFB41E0022C21D100F074FCC6
:1004900000280ED000F084FB054600F075FB0646F0
:1004A00001200346024629460090304605F08AFBAB
:1004B0002CE000F075FB054600F066FB06460020C8
:1004C00001231A4629460090304605F07BFB1DE0CB
:1004D00000F052FC054600F063FB064600F054FBBA
:1004E0000746012003462A4631460090384605F06B
:1004F00069FB0BE00020034602460146009005F030
:1005000061FB00220721104603F012F8F8BD00003D
:10051000FEB5002471480078012824D1FCF792FA36
:10052000012812D1FCF770F800BF0BE0182C02D1A3
:10053000601CC4B204E0FF222146002002F0F8FF54
:10054000601CC4B2242CF1DBC6E0FCF7A9F900243E
:1005500006E000222146104602F0EAFF601CC4B209
:10056000242CF6DBB8E0FCF76DFA012876D1FCF715
:100570004FFA5B4988426ED300F00CFB064600F050
:1005800023FB07460A21F7F7DBFD054632462946DD
:1005900001200AF0F9FF00F029FD064600F0CEFC2C
:1005A0000A210290F7F7CCFD054600F0F3FA074662
:1005B0003246294608F0EEFFFFF734FF00F0AAFAB2
:1005C00005462946012007F02BFB00F0F7FA064606
:1005D000FF21F531F7F7CAFDC5B22946012006F023
:1005E000AFFAFFF729FD0546FFF738FD0646FFF78E
:1005F0002FFD07462B4632463946012005F0BCFD4B
:1006000000F0E8F80546294601200BF063FA00F0F7
:10061000B5FC054600F0C2FB064600F0B5FC0746F7
:1006200000F0C2FB00233A46014600960195029075
:1006300001200AF0D9FC00F075FC054600F06CFCC6
:10064000064600F075FC07462A46314607F020FDB5
:1006500042E003E0FFE7FCF751F83DE0FCF720F94A
:1006600000222321104602F063FF002222211046BF
:1006700002F05EFF00220721104602F059FF00221F
:100680000821104602F054FF00220921104602F012
:100690004FFF00220A21104602F04AFF00221321D8
:1006A000104602F045FF00221121104602F040FFE3
:1006B00000221221104602F03BFF00220E211046BC
:1006C00002F036FF00220F21104602F031FF002217
:1006D0001021104602F02CFFFEBD00000101002099
:1006E000B80B000001490860704700008007002037
:1006F00002480068401C0149086070477C070020E0
:10070000F3B581B0064600200E49086000F01EF8DF
:10071000044600F01BF805462F1B3046029903F0F3
:10072000B3FE00900AE000F011F805462F1B0648C2
:100730000068002802D0044800688047009887427B
:10074000F1D3FEBD7C07002080070020014800682F
:10075000704700007C0700200B490978012901D16E
:1007600001200FE008490978022901D1022009E09F
:1007700005490978032901D1042003E00121024A37
:1007800011700120704700001107002010B5094BBF
:100790001B8899B20A12C8B2D3433133064C237076
:1007A000C3432333637013465633A3700346713338
:1007B000E37010BD4407002017070020014800889F
:1007C00070470000200000200148008870470000AA
:1007D0003800002001480078704700008C0000209D
:1007E00001480078704700008D00002010B50022FD
:1007F00005210648FAF78EFC040201220521034870
:10080000FAF788FC201880B210BD000050080020C4
:1008100010B5062205210348FAF77CFCC006C00F7C
:1008200010BD00005008002010B504220521064824
:10083000FAF770FC0402052211460348FAF76AFC35
:10084000201880B210BD00005008002010B506220C
:1008500005210248FAF75EFCC01110BD50080020C7
:1008600010B5022205210248FAF754FC10BD000021
:100870005008002010B5062205210348FAF74AFC6B
:100880008006C00F10BD00005008002010B50422E3
:1008900002210348FAF73EFCC007C00F10BD00005C
:1008A0005008002010B5052202210348FAF732FC57
:1008B000C007C00F10BD00005008002010B5002276
:1008C00004210348FAF726FC4006400F10BD000043
:1008D0005008002010B5042201210248FAF71AFC42
:1008E000801110BD5008002010B5002201210248DF
:1008F000FAF710FC10BD00005008002010B50522CA
:1009000001210348FAF706FC8007800F10BD0000A4
:100910005008002010B5012211460248FAF7FAFBF0
:1009200010BD00005008002010B5002206210C4820
:10093000FAF7F0FB0402012206210948FAF7EAFB64
:1009400020180402022206210548FAF7E3FB2018CA
:100950000402032206210248FAF7DCFB201810BD2E
:100960005008002010B5042206210C48FAF7D2FBEB
:100970000402052206210948FAF7CCFB20180402DC
:10098000062211460548FAF7C5FB20180402072283
:1009900006210248FAF7BEFB201810BD50080020BF
:1009A00010B5022203210248FAF7B4FB10BD000083
:1009B0005008002010B5032200210248FAF7AAFBD4
:1009C00010BD00005008002010B50022114602485A
:1009D000FAF7A0FB10BD00005008002010B504225B
:1009E00000210248FAF796FB10BD000050080020D5
:1009F00010B5012200210248FAF78CFB10BD00005F
:100A00005008002010B5052200210248FAF782FBA9
:100A100010BD000050080020322815DA3C498978C2
:100A2000012903DD01213A4A517070E03849897883
:100A3000002905DD2F286ADC0021354A517066E067
:100A40000021334A517062E03E2817DA322815DB64
:100A50002F498978022903DD02212D4A517056E081
:100A60002B498978012905DD3B2850DC0121284AE2
:100A700051704CE00121264A517048E0502817DAA5
:100A80003E2815DB22498978032903DD0321204A0A
:100A900051703CE01E498978022905DD4D2836DC7D
:100AA00002211B4A517032E00221194A51702EE096
:100AB000622817DA502815DB15498978042903DDE7
:100AC0000421134A517022E011498978032905DD78
:100AD0005F281CDC03210E4A517018E003210C4AE8
:100AE000517014E073280FDA62280DDB0849897809
:100AF000042905DD70280ADC0421054A517006E04E
:100B00000421034A517002E00521014A51707047E7
:100B1000B809002001480078704700000700002055
:100B20000148006870470000881F002001480078D5
:100B300070470000F5000020014800787047000071
:100B4000F4000020F8B5002600240025FCF79CFEE8
:100B500007460A21F7F7F4FA054609480068854276
:100B600000D303E006480068461B34467D200001A0
:100B7000844200D30446034804600068F8BD0000C6
:100B8000280100202401002001480078704700005F
:100B9000F900002001480079704700003828002043
:100BA0000148407870470000F90000200148007AB1
:100BB0007047000038280020002070470148008856
:100BC000704700002200002010B50024FFF7E2FF6C
:100BD00000280AD10A4800880A49884202DB0846F0
:100BE000074908800648048808E005480088FCF7A3
:100BF000F9FB84B20448844200DB0446204610BD61
:100C00003A000020C6070000CE040000002005497D
:100C10000988054A914202DB1146024A11800149C6
:100C2000088870473A000020C6070000F8B5002782
:100C3000002500260024FFF7C7FE0546FFF7D8FE73
:100C40000646F020284000110A2805DBF020284045
:100C50000011C01C044303E0F020284000110443AD
:100C600024022807000F0A2804DB2807000FC01CF5
:100C7000044302E02807000F04432402F020304020
:100C800000110A2805DBF02030400011C01C04438D
:100C900003E0F02030400011044324023007000F2D
:100CA0000A2804DB3007000FC01C044302E03007B1
:100CB000000F0443002C01D10248F8BD27463846F6
:100CC000FBE70000FFFF0000F8B500270025002625
:100CD0000024FFF783FE0546FFF794FE0646F0204A
:100CE000284000110A2805DBF02028400011C01C14
:100CF000044303E0F02028400011044324022807A5
:100D0000000F0A2804DB2807000FC01C044302E080
:100D10002807000F04432402F020304000110A2865
:100D200005DBF02030400011C01C044303E0F0203C
:100D300030400011044324023007000F0A2804DB6E
:100D40003007000FC01C044302E03007000F0443CB
:100D5000002C01D10248F8BD27463846FBE70000C9
:100D6000FFFF000010B50024FFF724FE04462046D4
:100D700010BD012070470000014800787047000056
:100D80004D07002001480078704700004F07002001
:100D90000148C07B70470000C40900200148007A68
:100DA00070470000C409002010B5002405480088E1
:100DB000323084B264212046F7F7D8F984B2204655
:100DC00010BD0000C409002070B500240749086860
:100DD000FBF758FF05466421F7F7B2F984B20448DF
:100DE000844200DD0446204670BD0000C409002096
:100DF000DE03000010B5002400F016F8012801D130
:100E000003240CE000F010F8022802D1FF2437344C
:100E100005E00A2103480088F7F7A8F984B22046C4
:100E200010BD00000200002001480078704700005B
:100E30000B00002010B50024044804F093FB0028A8
:100E400001D0012400E00024204610BD030700006B
:100E500010B50024044804F085FB002801D00124CB
:100E600000E00024204610BD0507000010B5002456
:100E7000044804F077FB002801D0012400E000249E
:100E8000204610BD0707000010B50024062004F01E
:100E900069FB002801D0012400E00024204610BD99
:100EA00010B50024052004F05DFB002801D00124CA
:100EB00000E00024204610BD10B50024044804F0D2
:100EC00051FB002801D0012400E00024204610BD81
:100ED0000607000010B50024044804F043FB002876
:100EE00001D0012400E00024204610BD03050000CD
:100EF00010B50024044804F035FB002801D001247B
:100F000000E00024204610BD040500000148807A5E
:100F100070470000C4090020014880787047000035
:100F2000580A00200148406870470000580A002015
:100F30000148407870470000580A002070B500242E
:100F4000FFF728FE002803D1FCF79EFC04460DE0C5
:100F5000FFF720FE012806D1FCF796FC0546FCF7BA
:100F600041FA044602E0FCF78FFC0446204670BDBF
:100F70000148007C70470000C40900200148407A05
:100F800070470000C409002010B50024054880887F
:100F9000323084B264212046F7F7E8F884B2204664
:100FA00010BD0000C409002070B50024074948683E
:100FB000FBF768FE05466421F7F7C2F884B20448DF
:100FC000844200DD0446204670BD0000C4090020B4
:100FD000DE0300000148007B70470000C4090020C8
:100FE0000148007870470000F800002070B5002428
:100FF000FFF7D0FD002803D1FCF768FC04460FE0A2
:10100000FFF7C8FD012807D10020FCF75FFC05466B
:10101000FCF7E8F9044603E00020FCF757FC04461F
:10102000204670BD01480078704700004200002053
:1010300070B505460024032D00D170BD002D01D0F0
:10104000012D1BD181210320800204F03BFA802175
:10105000134804F037FA32211248FFF751FB0024FD
:1010600009E0A200104BD2189178A200985A04F01F
:1010700029FA601CC4B23B2CF3DB0FE0022D0DD12A
:10108000002409E0A200094BD2189178A200985AD6
:1010900004F018FA601CC4B23B2CF3DB00BFCCE7B1
:1010A00002060000A0860100280C0200140D0200B8
:1010B000F8B5002100240023002200BF0AE001252A
:1010C0008D40ABB205881D402C469C4200D10A469B
:1010D0004D1CA9B21029F2DB0588FF2D1FDC284D1D
:1010E0006D7E0688B543264E757635462D7E06887C
:1010F000B543234E357635466D7E8678F607F60F76
:10110000964035431E4E757635462D7E86780227ED
:101110003E40760896403543194E357622E0184D0C
:10112000ED7E0688B543164EF5763546AD7E0688CB
:10113000B543134EB5768578ED07ED0F1646083E9C
:10114000B5400F4EF67E35430D4EF5768578022676
:1011500035406D081646083EB540094EB67E35430B
:10116000074EB5760025009505E000BF6D462D7849
:101170006D1CEEB200966D462D78012DF5D9F8BDA7
:10118000206B0440C107C90F002905D00021394A4E
:101190001171002238490A7102210140002905D04D
:1011A0000021344A1172002233490A72042101409D
:1011B000002905D000212F4A117300222E490A73FD
:1011C00008210140002905D000212A4A117400227B
:1011D00029490A7410210140002905D00021254A1F
:1011E0001175002224490A7520210140002905D0EB
:1011F0000021204A117600221F490A764021014031
:10120000002904D000221B494A711B494A718021E0
:101210000140002904D0002216494A7216494A7238
:10122000FF2101310140002904D0002211494A73F5
:1012300011494A73012149020140002904D00022CA
:101240000C494A740C494A74012189020140002961
:1012500004D0002207494A7507494A750121C9028D
:101260000140002904D0002202494A7602494A7608
:10127000704700000060004000610040C107C90FD6
:10128000002905D001223C490A7100213B4A117115
:1012900002210140002905D0012237490A720021AC
:1012A000364A117204210140002905D00122324939
:1012B0000A730021314A117308210140002905D029
:1012C00001222D490A7400212C4A11741021014079
:1012D000002905D0012228490A750021274A1175E5
:1012E00020210140002905D0012223490A7600214E
:1012F000224A117640210140002905D001221E49D1
:101300004A7100221D494A7180210140002905D0FF
:10131000012219494A72002218494A72FF210131FB
:101320000140002905D0012213494A7300221349C4
:101330004A73012149020140002905D001220E49CA
:101340004A7400220D494A74012189020140002992
:1013500005D0012208494A75002208494A75012131
:10136000C9020140002905D0012203494A76002222
:1013700002494A767047000000610040006000406A
:1013800010B50C480078002803D00B4A50689168CB
:10139000884708484078002803D0084A5068916878
:1013A000884704488078002803D0054A506891682F
:1013B000884710BD00600040FC0200207C04002033
:1013C000FC05002010B508480079002803D0074A22
:1013D00010695169884704484079002803D0044ABD
:1013E00050689168884710BD00600040FC020020F2
:1013F0008804002010B50848007A002803D0074A66
:10140000D069116A88470448407A002803D0044A0A
:1014100050689168884710BD00600040FC020020C1
:101420009404002010B50848007B002803D0074A28
:10143000906AD16A88470448407B002803D0044A58
:1014400050689168884710BD00600040FC02002091
:10145000A004002010B50848007C002803D0074AEB
:10146000506B916B88470448407C002803D0044AA5
:1014700050689168884710BD00600040FC02002061
:10148000AC04002010B50848007D002803D0074AAE
:10149000106C516C88470448407D002803D0044AF2
:1014A00050689168884710BD00600040FC02002031
:1014B000B804002010B50848007E002803D0074A71
:1014C000D06C116D88470448407E002803D0044A40
:1014D00050689168884710BD00600040FC02002001
:1014E000C404002010B50848407F002803D0074AF4
:1014F0005068916888470448007F002803D0044A58
:10150000906DD16D884710BD00600040D004002070
:10151000FC02002010B508484078002803D0074A94
:1015200050689168884704480078002803D0044A2E
:10153000506E916E884710BD20600040DC04002092
:10154000FC02002010B509480079002803D0084AA1
:10155000106F516F88470548001D4078002803D060
:10156000044A50689168884710BD00002060004020
:10157000FC020020E804002010B5034AD06F783246
:101580009168884710BD0000FC02002010B5024A97
:1015900050689168884710BD8003002010B5094845
:1015A000007C002803D0084A5068916888470548A5
:1015B00010304078002803D0044A5068916888476A
:1015C00010BD0000206000408C0300200C050020AE
:1015D00010B5024A50689168884710BD98030020F2
:1015E00010B5024A50689168884710BDA4030020D6
:1015F00010B50948007F002803D0084A5068916858
:10160000884705481C304078002803D0044A5068B9
:101610009168884710BD000020600040B0030020A2
:101620003005002010B50C480078002803D00B4A84
:1016300050689168884708484078002803D0084AD5
:1016400050689168884704488078002803D0054A8C
:1016500050689168884710BD40600040BC0300207E
:101660003C050020BC06002010B50D48007900287C
:1016700003D00C4A5068916888470948001D40789B
:10168000002803D0084A5068916888470448001D24
:101690008078002803D0054A50689168884710BDBB
:1016A00040600040C803002048050020C806002014
:1016B00010B50D48007A002803D00C4A5068916894
:1016C0008847094808304078002803D0084A506805
:1016D00091688847044808308078002803D0054A7C
:1016E00050689168884710BD40600040D4030020D6
:1016F00054050020D406002010B50D48007B0028BA
:1017000003D00C4A50689168884709480C304078EB
:10171000002803D0084A50689168884704480C3074
:101720008078002803D0054A50689168884710BD2A
:1017300040600040E003002060050020E00600203B
:1017400010B50D48007C002803D00C4A5068916801
:101750008847094810304078002803D0084A50686C
:1017600091688847044810308078002803D0054AE3
:1017700050689168884710BD40600040EC0300202D
:101780006C050020EC06002010B5024A50689168F4
:10179000884710BDF803002010B50948007E0028D6
:1017A00003D0084A50689168884705481830407847
:1017B000002803D0044A50689168884710BD000093
:1017C00040600040040400208405002010B5094852
:1017D000007F002803D0084A506891688847054870
:1017E0001C304078002803D0044A5068916888472C
:1017F00010BD000040600040100400209005002053
:1018000010B508480078002803D0074A506891684E
:10181000884704484078002803D0044A50689168FB
:10182000884710BD606000401C0400209C0500201B
:1018300010B509480079002803D0084A506891681B
:1018400088470548001D4078002803D0044A5068A6
:101850009168884710BD00006060004028040020A7
:10186000A805002010B50948007A002803D0084ACE
:10187000506891688847054808304078002803D0B0
:10188000044A50689168884710BD000060600040BD
:1018900034040020B405002010B5024A5068916855
:1018A000884710BD4004002010B5024A5068916876
:1018B000884710BD4C04002010B50948007D002861
:1018C00003D0084A5068916888470548143040782A
:1018D000002803D0044A50689168884710BD000072
:1018E0006060004058040020D805002010B5094869
:1018F000007E002803D0084A506891688847054850
:1019000018304078002803D0044A5068916888470E
:1019100010BD00006060004064040020E405002069
:1019200010B50948007F002803D0084A5068916824
:10193000884705481C304078002803D0044A506886
:101940009168884710BD000060600040700400206E
:10195000F005002010B5FE4800688079002806D008
:1019600001286ED002286DD003286CD104E2F8481B
:101970000068407903000EF089FB0A0614BC2BBCFA
:1019800047BC67BC9BBC0AF007FC0020F049096813
:10199000C873EF4800684079401CED4909684871F8
:1019A000AEE0EC490969EA4A1268D27A885C0AF02A
:1019B0006BFCE74800684079401CE54909684871BC
:1019C000E34800684079401CE1490968487197E0A4
:1019D00001F016FF002810D10AF056FCDC48006820
:1019E0004079401CDA4909684871D9480068407953
:1019F000401CD7490968487105E00AF0F7FB002050
:101A0000D349096848717BE001F0FAFE002811D142
:101A100001200AF039FCCE4800684079401CCC49CE
:101A200009684871CA4800684079401CC84909687B
:101A3000487105E00AF0DAFB0020C54909684871E1
:101A40005EE05FE0FEE0A3E101F0DAFE002828D1CD
:101A5000BF490968C97A24225143BF4A12688918CC
:101A6000BB4A1268D27B885C0AF00EFCB84800685A
:101A7000C07B401CB6490968C873B5480068C07B84
:101A8000242814D3B24800684079401CB049096842
:101A90004871AF4800684079401CAD4909684871F9
:101AA00005E00AF0A3FB0020A9490968487127E076
:101AB00001F0A6FE002815D1A5480068C07A401C98
:101AC000A3490968C872A2480068C07AA149097888
:101AD000884207DB00209E490968C87201209C49A2
:101AE000096888710AF082FB0020994909684871E9
:101AF00006E00AF07BFB002095490968487100BFA9
:101B000000BF4FE192480068407903000EF0BEFA32
:101B1000080513912A91479170910AF03DFB00202E
:101B20008B490968C8738A4800684079401C884915
:101B30000968487184E087490969854A1268D27A40
:101B4000885C0AF0A1FB824800684079401C80490B
:101B5000096848717E4800684079401C7C490968E2
:101B600048716DE001F04CFE002811D126200AF0EA
:101B70008BFB774800684079401C754909684871BB
:101B8000734800684079401C71490968487105E054
:101B90000AF02CFB00206E490968487150E001F002
:101BA0002FFE00281DD101200AF06EFB6848006856
:101BB000C07B401C66490968C87365480068C07BE3
:101BC000242814D3624800684079401C60490968A1
:101BD00048715F4800684079401C5D490968487158
:101BE00005E00AF003FB002059490968487127E025
:101BF00001F006FE002815D155480068C07A401C47
:101C000053490968C87252480068C07A5149097836
:101C1000884207DB00204E490968C87202204C49FF
:101C2000096888710AF0E2FA002049490968487198
:101C300006E00AF0DBFA002045490968487100BF58
:101C400000BFAFE042480068407903000EF01EFA82
:101C50000805138B2A8B478B638B0AF09DFA0020B3
:101C60003B490968C8733A4800684079401C3849C4
:101C7000096848717EE037490969354A1268D27AA5
:101C8000885C0AF001FB324800684079401C30490A
:101C9000096848712E4800684079401C2C49096841
:101CA000487167E001F0ACFD002811D125200AF051
:101CB000EBFA274800684079401C254909684871BB
:101CC000234800684079401C21490968487105E0B3
:101CD0000AF08CFA00201E49096848714AE001F0B8
:101CE0008FFD002810D10AF0CFFA1948006840791A
:101CF000401C174909684871154800684079401C24
:101D000013490968487105E00AF070FA002010498B
:101D1000096848712EE001F073FD002815D10C48C8
:101D20000068C07A401C0A490968C87208480068FF
:101D3000C07A08490978884207DB0020044909680D
:101D4000C87203200249096888710AF04FFA05E059
:101D5000D0070020142F0020CC07002000201249BB
:101D60000968487106E00AF041FA00200E49096846
:101D7000487100BF00BF15E000200B490968887159
:101D8000094909684871062007490968C87009E0CF
:101D90000AF02CFA002004490968487102490968D0
:101DA000887100BF00BF10BDD007002010B56A4881
:101DB0000068407903000EF069F9090610C627C6CD
:101DC00044C6608EC6000AF0E7F9634800684079AF
:101DD000401C614909684871BCE0604909695E4A74
:101DE0001268D27A885C0AF04FFA5B480068407942
:101DF000401C594909684871574800684079401C9F
:101E0000554909684871A5E001F0FAFC002811D194
:101E10004F200AF039FA504800684079401C4E497A
:101E2000096848714C4800684079401C4A49096873
:101E3000487105E00AF0DAF900204749096848715D
:101E400088E001F0DDFC002810D10AF01DFA4248BC
:101E500000684079401C4049096848713E48006864
:101E60004079401C3C490968487105E00AF0BEF918
:101E700000203949096848716CE001F0C1FC002874
:101E800022D135480068C07A401C33490968C872BD
:101E900031480068C07A3149097888420FDB002058
:101EA0002D490968C8722C4800684079401C2A49AD
:101EB00009684871002028490968486208E0002044
:101EC00025490968487103E00020234909684871E1
:101ED0000AF08CF93EE020480068407C002816D0CB
:101EE0001E48C068002803D01C48C16819208847D4
:101EF000002019490968486217490968487116495C
:101F000009688871052014490968C8701AE01248E8
:101F10000068406A282807D20F480068406A401CC1
:101F20000D49096848620DE000200B4909684862C4
:101F300009490968487108490968887105200649F6
:101F40000968C87006E00AF051F9002002490968E2
:101F5000487100BF00BF10BDD0070020142F002023
:101F600010B50024F7480068807A01287ED1F54832
:101F70000068C07900287AD0F2480068807900288B
:101F800004D0012874D0022873D191E1ED48006893
:101F9000007B24286ED2EB480068C07901287AD1F2
:101FA000002475E0E7480068C07A24214843E649E8
:101FB00009684018E3490968097B415CE148006809
:101FC000C07A24225043E14A12688018DD4A126820
:101FD000127B805C814229D0DA480068C07A2421D3
:101FE0004843DA4909684018D6490968097B415CC9
:101FF000D4480068C07A24225043D34A126880181B
:10200000D04A1268127B8154CE480068407B242855
:1020100005D3CC480068007BCA4909684873C948A1
:102020000068007BC7490968887308E0C5480068F4
:10203000407B242803D20120C24909688871C14825
:102040000068007B401CBF4909680873BD480068F0
:10205000007B242808D3BB480068407B242803D297
:102060000120B84909688871B64805E0D3E1CDE19F
:1020700069E0BAE138E00EE00068007B242804D271
:10208000B04800688079012800D103E0601CC4B228
:10209000242C87D356E0002413E0AA480068C07AB5
:1020A00024214843A94909684018015DA5480068F2
:1020B000C07A24225043A44A126880180155601C3B
:1020C000C4B2242CE9D300209E4909684873232018
:1020D0009C490968887301209A49096888712420FD
:1020E0009849096808732DE000209649096808732B
:1020F00094480068C07A401C92490968C8729148A7
:102100000068C07A92490978884217DB8D480068D8
:10211000007C012804D102208A490968887106E000
:10212000002088490968887186490968C8710020BB
:1021300084490968C8728349096808740020814984
:102140000968487161E17F480068407903000DF03B
:102150009DFF080513A62AA651A68EA6012079493F
:10216000096808740AF018F8764800684079401C3D
:1021700074490968487199E075490969714A12689A
:10218000D27A885C0AF080F86E4800684079401C7A
:102190006C49096848716B4800684079401C69497E
:1021A0000968487182E001F02BFB00281BD16549CA
:1021B0000968497B491CC8B20AF066F861480068A2
:1021C000407B60490968C8735E4800684079401CDC
:1021D0005C49096848715B4800684079401C59496E
:1021E0000968487105E00AF001F8002055490968BE
:1021F00048715BE001F004FB00282BD151490968CC
:10220000C97A24225143504A126889184D4A1268EB
:10221000D27B885C0AF038F84A480068C07B401CD2
:1022200048490968C87347480068C07B4549096840
:10223000897B88421ADD434800684079401C414947
:10224000096848713F4800684079401C3D49096869
:1022500048710BE009F0CAFF3A480068407B3949F1
:102260000968C87300203749096848711EE001F009
:10227000C7FA00280CD133490968887124203149F4
:102280000968C8732F49096848732E49096888731B
:1022900009F0ACFF00202B490968487106E009F0FD
:1022A000A5FF002027490968487100BF00BFACE0C6
:1022B00024480068407903000DF0E8FE08050F8E01
:1022C000268E4C8E688E09F067FF1E4800684079A4
:1022D000401C1C490968487185E01D490969194A73
:1022E0001268D27A885C09F0CFFF164800684079FE
:1022F000401C144909684871124800684079401C24
:102300001049096848716EE001F07AFA002811D18D
:10231000252009F0B9FF0B4800684079401C0949A5
:1023200009684871074800684079401C05490968F8
:10233000487105E009F05AFF002002490968487118
:1023400051E00000D0070020CC070020C807002083
:10235000142F002001F054FA002810D109F094FF46
:10236000644800684079401C6249096848716148C6
:1023700000684079401C5F490968487105E009F030
:1023800035FF00205B49096848712CE001F038FAFC
:1023900000281AD157480068C07A401C554909687E
:1023A000C87254480068C07A5349097888420CDBE7
:1023B000002050490968C8724E49096888714D4922
:1023C000096848714B490968C87109F00FFF00207E
:1023D00048490968487106E009F008FF00204549AE
:1023E0000968487100BF00BF0FE009F0FFFE002040
:1023F0004049096848713F49096888713D49096841
:1024000008733C490968C87200BF71E0002039496F
:10241000096888726CE037480068807A022867D1C2
:1024200034480068007A00285ED03248006840795D
:10243000002804D001280CD0032846D11BE009F065
:10244000ABFE2C4800684079401C2A490968487155
:1024500049E0002009F018FF264800684079401C38
:10246000244909684871234800684079401C214983
:102470000968487137E009F059FE002812D11D485B
:1024800000684078401C1B4909684870194800687A
:102490004078032812D301F053FA00201549096847
:1024A00048700BE00020134909680872AA201149FE
:1024B0000968887000200F490968487009F096FE85
:1024C00000200C49096848710DE009F08FFE0020DA
:1024D000084909684871074909684870AA200549F0
:1024E0000968887000BF03E000200249096888720B
:1024F00010BD0000D0070020142F0020F8B50446BE
:102500000D4600260C2060431D49085C002801D0C0
:102510000120F8BD0C2060431949401885600C204B
:10252000604340188068002801D10120F1E70121B3
:102530000C206043124A115400222046E317DB0EA0
:102540001B185B115B01E31A9B000E4FDB19E717A9
:10255000FF0E3F197F11DA550DF0CAFD002220460B
:10256000E317DB0E1B185B115B01E31A9F00064BA0
:10257000FB18E717FF0E3F197F11DA553046C8E701
:10258000FC020020006000400061004000BFFEE748
:1025900009480088401C0849088008460088074907
:1025A000884208DD06480078002804D00846024921
:1025B0000880012088707047F0000020DC050000D2
:1025C000F400002010B515488078012824D1144863
:1025D000007801280CD113480078012808D1002088
:1025E00011498870084602F08BFD00200D490870E3
:1025F0000B48007802280CD10C480078012808D13B
:10260000002009498870084602F07AFD0020074939
:10261000087000200249087010BD0000F000002082
:10262000F4000020F6000020F9000020F700002050
:102630007047000010B500F05DFE012803D10020B6
:1026400001490880887010BDF0000020F0B50546F3
:102650000E46174600243A463146284600F058FEFA
:1026600000BF42E000202101394A12685052210186
:10267000374A12688918488000212001344A1268BC
:10268000801881802001324A12688018C1802001A0
:102690002F4A12688018017220012D4A1268801892
:1026A000417220012A4A1268801881722001284A4A
:1026B00012688018C17200202101254A1268891809
:1026C000087300212001224A1268801841730020FB
:1026D00021011F4A126889188873002120011C4AB1
:1026E00012688018C173601CC4B21A484078A042B6
:1026F000B8DC64201849096808807D20C0001649AC
:102700000968488015481449096888807D200001BF
:1027100011490968C88010490968088110480E49A4
:10272000096848810F480C490968888140000A49B6
:102730000968C8813220084909680882FF20F530FD
:10274000054909684882044909688882F0BD00008B
:1027500090070020840700208C0700204C04000014
:10276000102700003075000038B5002404E0002078
:1027700013490855601C84B2282CF8D301216846FF
:10278000417001706A460F490D48FFF75FFF7D21D8
:10279000C900322000F0ACF90B490C4800F0C6F932
:1027A0000948643000F058F90748C83000F064F96F
:1027B000074800F077F9074800F08AF938BD0000B3
:1027C00048280020E011020028230000B80B000078
:1027D000542400001027000010B524480078002879
:1027E00003D10120214908703EE0204800780128EB
:1027F00010D11F480078012808D100201D49887099
:10280000084602F07DFC0020194908700220174993
:10281000087029E015480078022810D11648007881
:10282000012808D1002013498870084602F068FC8E
:1028300000201149087003200C49087014E00B486F
:102840000078032803D10520084908700CE00748E8
:102850000078052803D005480078062804D1002018
:10286000024908700549087010BD0000F4000020FE
:10287000F6000020F9000020F7000020F8000020FA
:10288000F8B50024002500263548007800281ED120
:1028900034480078002803D101203249087016E03E
:1028A00030480078012803D102202E4908700EE03C
:1028B0002C480078022803D103202A49087006E03A
:1028C00028480078032802D10020264908702448AF
:1028D000007801280ED10124172500262248012363
:1028E000324629460090204601F020FE01201F4973
:1028F000087034E01A48007802280FD101243B25E3
:1029000000261948401C01233246294600902046E3
:1029100001F00CFE01201649087020E010480078F4
:1029200003280DD1FEF736F9002803D10120114903
:10293000087102E000200F4908710DF079FB0EE0EC
:1029400007480078052803D106200549087006E0ED
:1029500003480078062802D1052001490870F8BD17
:10296000F4000020F5000020F9000020F60000200F
:10297000F70000203828002010B5044623000DF091
:1029800085FB095B060E16171819595A5E00FAF7EF
:102990003FF82C49884201D3FFF772FF50E0FAF765
:1029A00037F82849884201D3FFF716FF48E047E08F
:1029B00046E045E0FAF72CF82249884239D301F085
:1029C00071FD21480078032814D1204800780028A0
:1029D00010D1FEF7EBF8002806D101201C498860D1
:1029E0008868FAF7D9FF05E00020194988608868EF
:1029F000FAF7D2FF14480078012805D1134800786F
:102A0000002801D1FAF796F910480078052803D17B
:102A10000120104908700AE00C480078062803D10C
:102A200002200C49087002E000200A4908700BF0EF
:102A3000CBF805E004E003E0FFF7AAFD00E000BFEB
:102A400000BF10BDB80B0000F5000020F40000200E
:102A500038280020F800002001460020054A1268AE
:102A600052898A4201DC012002E0024A1268118187
:102A7000704700008C07002001460020084A1268B9
:102A800012898A4201DB012009E0054A1268928915
:102A90008A4201DC012002E0014A1268518170473C
:102AA0008C07002001460020084A126852898A4299
:102AB00001DB012009E0054A1268D2898A4201DC63
:102AC000012002E0014A1268918170478C070020C2
:102AD00001460020054A126892898A4201DB0120E2
:102AE00002E0024A1268D181704700008C07002082
:102AF000024600200C4B1B681B8A934201DD01201B
:102B000010E08A4201DB01200CE0074B1B689B8828
:102B10008B4201DC012005E0034B1B681A80024B4D
:102B20001B685980704700008C0700200246002077
:102B30000C4B1B681B8A934201DD012010E08A4286
:102B400001DB01200CE0074B1B685B88934201DB33
:102B5000012005E0034B1B689A80024B1B68D9805B
:102B6000704700008C07002070B5044600250C203B
:102B70006043FE49096840184068002807D00C21CE
:102B80006143FA4A126889184868804705460C2054
:102B90006043F6490968085C002873D10C20604343
:102BA000F249096840188068002874D02001F04973
:102BB00009684018C07A02280AD1032D08D10C20D8
:102BC0006043EA4A1268801881680120884762E001
:102BD0002001E74909684018C07A02280AD1042D6B
:102BE00008D10C206043E14A1268801881680220F5
:102BF000884750E02001DE4909684018C07A022861
:102C00000AD1052D08D10C206043D84A12688018DB
:102C10008168032088473EE02001D54909684018B3
:102C2000C07A02280AD1062D08D10C206043CF4A71
:102C3000126880188168042088472CE02001CC4964
:102C400009684018C07A02280AD1072D08D10C2043
:102C50006043C64A126880188168052088471AE0D8
:102C60002001C34909684018C07A02280BD1082DF9
:102C700009D10C206043BD4A126880188168062083
:102C8000884708E00DE00C206043B84A12688018BD
:102C90008168002088472001B54909684018C5723D
:102CA0000CE30C206043B1490968085C012873D12A
:102CB0000C206043AD49096840188068002874D032
:102CC0002001AB4909684018C07A03280AD1022DB7
:102CD00008D10C206043A54A126880188168012041
:102CE000884762E02001A24909684018C07A042898
:102CF0000AD1022D08D10C2060439C4A126880182A
:102D000081680220884750E02001994909684018ED
:102D1000C07A05280AD1022D08D10C206043934ABD
:102D2000126880188168032088473EE0200190499E
:102D300009684018C07A06280AD1022D08D10C2053
:102D400060438A4A126880188168042088472CE012
:102D50002001874909684018C07A07280AD1022D46
:102D600008D10C206043814A1268801881680520D0
:102D700088471AE020017E4909684018C07A08286F
:102D80000BD1022D09D10C206043784A12688018BB
:102D900081680620884708E00DE00C206043734AF4
:102DA00012688018816800208847200170490968EE
:102DB0004018C57282E20C2060436C490968085CC7
:102DC0000228F7D1002D7DD1200169490968085AF0
:102DD00068490968098A884275DA200164490968E6
:102DE000085A0A3081B22001614A1268115220014A
:102DF0005F490968085A5F490968098A884231DBD6
:102E000020015B490968401840885A4909680988C7
:102E1000884227DB200156490968401840885549F7
:102E20000968498888421DDC00202101504A126847
:102E30008918488020014E4909684018807A002886
:102E4000B8D10C20604349490968401880680028BF
:102E5000B0D00C206043454A126880188168012078
:102E600088472BE2200142490968085A414909680C
:102E7000098A88429EDB20013D4909684018408844
:102E80003C4909688988884294DB200138490968EF
:102E90004018408837490968C98888428ADC002080
:102EA0002101334A12688918488020013049096895
:102EB0004018807A0028D4D10C2060432B4909683F
:102EC000401801E063E00BE080680028C9D00C20C6
:102ED0006043264A12688018816802208847EDE125
:102EE00000202101224A1268891848802101204AC5
:102EF00012688918C872002120011D4A12688018C2
:102F0000C18020011A4A1268801841722001184AB3
:102F1000126880188172184801782001144A1268DA
:102F20008018017200202101114A126889188880D6
:102F300021010F4A12688918087321010C4A12688E
:102F40008918487321010A4A126889188873002178
:102F50002001074A12688018C1730C20604303499E
:102F60000968401880680028B9D007E08807002069
:102F7000900700208C070020840700200C2060436D
:102F8000CF4A1268801881680020884796E1012D99
:102F9000A5D12001CB4909684018C07AA84225D0A4
:102FA00000212001C74A12688018418000202101B9
:102FB000C44A12688918C8802001C24909684018AB
:102FC000C572C14800782101BE4A1268891848724A
:102FD00000202101BB4A126889188880BA4801780C
:102FE0002001B84A12688018017267E12001B549D2
:102FF00009684018007AB4490978884220D0B2485C
:1030000000782101AF4A1268891808722001AD4981
:1030100009684018407AAC490978884209D02001F3
:10302000A8490968401880882101A64A12688918B1
:10303000C88000212001A34A12688018818012E014
:103040002001A049096840188088A04988420AD216
:1030500020019C490968401880880A302101994A5A
:1030600012688918888020019649096840184088AC
:10307000964988420AD2200192490968401840883E
:103080000A3021018F4A12688918488020018D4931
:1030900009684018407A8C490978884205D0012097
:1030A0002101884A126889188872200185490968B7
:1030B00040184088864909680988884204DB002155
:1030C0002001804A1268115220017E490968401887
:1030D000807A00287ED10C20604379490968401825
:1030E0008068002877D02001764909684018408818
:1030F000774909680989884214DB20017149096808
:103100004018007B00280DD10C2060436C4A1268E7
:10311000801881680320884701202101694A1268CC
:103120008918087320016749096840184088684970
:1031300009684989884214DB2001624909684018FE
:10314000407B00280DD10C2060435D4A1268801836
:10315000816804208847012021015A4A1268891891
:103160004873200157490968401840885849096840
:103170008989884214DB2001524909684018807B04
:1031800000280DD10C2060434D4A126880188168D8
:1031900005208847012021014A4A1268891888734E
:1031A0002001484909684018408849490968C98987
:1031B000884210DB2001434909684018C07B002881
:1031C0007CD10C2060433E4A12688018816806203A
:1031D000884701E007E03BE001202101394A1268FD
:1031E0008918C8736AE02001364909684018407A96
:1031F00001282ED13448007802282AD120013149F3
:1032000009684018C08832490968498A884255DBF4
:1032100020012C490968401880882D490968898A4D
:1032200088424BDB0C2060432549096840188068C0
:10323000002843D00C206043214A1268801881681E
:1032400007208847002021011E4A12688918487209
:1032500034E020011B4909684018407A02282DD12A
:1032600019480078012829D1200116490968401819
:10327000C08817490968898A88421FDB20011149E3
:1032800009684018808812490968498A884215DB14
:103290000C2060430A4909684018806800280DD056
:1032A0000C206043064A126880188168082088470D
:1032B00000202101034A12688918487270BD00007D
:1032C000880700209007002084070020F0FF0000FE
:1032D0008C07002010B5002400BF04E02046FFF753
:1032E00043FC601CC4B202484078A042F6DC10BD2A
:1032F0008407002010B50024044802F033F90028A8
:1033000000D000E00124204610BD000003040000AE
:1033100010B5074B14781C7054785C70054B19601D
:10332000054B186003461833044C236010BD0000A1
:1033300084070020880700208C07002090070020C9
:1033400010B50446012C09D1FF220C21002000F009
:10335000EFF80121022004F0D5FD08E000220C2145
:10336000104600F0E5F80021022004F0CBFD10BD6E
:1033700010B5002404210848F7F7DEFE552801D1D6
:10338000012407E0042000F0FFFF002801D0002402
:1033900000E00124204610BD5008002010B504466E
:1033A000012C09D1FF221C21002000F0C1F80121CD
:1033B000062004F0A7FD08E000221C21104600F0C2
:1033C000B7F80021062004F09DFD10BD10B50024C3
:1033D000062000F0D9FF002801D0012400E00024DD
:1033E000204610BD10B50446012C09D1FF2217213B
:1033F000002000F09DF80121042004F083FD08E086
:1034000000221721104600F093F80021042004F058
:1034100079FD10BD00200449097A002901D001205E
:1034200000E0002070470000580A002010B5044654
:10343000022C1CD100220D21104600F079F8FDF776
:103440009BFC002809D0FF220B21002000F070F81F
:1034500001210D2004F056FD58E000220B211046FA
:1034600000F066F800210D2004F04CFD4EE0032C26
:103470001CD100220B21104600F05AF8FDF77CFC0D
:10348000002809D0FF220D21002000F051F8012171
:103490000D2004F037FD39E000220D21104600F028
:1034A00047F800210D2004F02DFD2FE0042C0ED153
:1034B000FF220D21002000F03BF800220B211046D6
:1034C00000F036F801210D2004F01CFD1EE0012C57
:1034D0000ED100220D21104600F02AF8FF220B2108
:1034E000002000F025F801210D2004F00BFD0DE077
:1034F00000220D21104600F01BF800220B2110467F
:1035000000F016F800210D2004F0FCFC10BD10B5F1
:103510000024FCF797FD022801D1022406E0FCF705
:1035200091FD012801D1032400E00424204610BDB0
:1035300010B5064B1B78834207DD242905D22423CE
:103540004343034C24681B195A5410BD142F002008
:10355000C807002010B574480068407903000CF0DB
:1035600095FD0B0711D325D35A6D77D38DA8D300C2
:1035700008F012FE6C4800684079401C6A490968EE
:103580004871CFE069494969087808F07DFE6648CE
:1035900000684079401C64490968487162480068C5
:1035A0004079401C604909684871BBE000F028F987
:1035B000002811D17F2008F067FE5B480068407941
:1035C000401C594909684871574800684079401CB7
:1035D0005549096848711DE0534800684078401C0F
:1035E00051490968487050480068407803280BD357
:1035F00000204D4909684870AA204B490968887025
:10360000032049490968C87008F0F0FD00204649C8
:103610000968487186E000F0F3F8002807D14248B5
:1036200000684079401C40490968487103E0002067
:103630003D490968487108F0D9FD73E008F0ACFD18
:10364000394800684079401C37490968487169E089
:10365000364949690978491CC8B208F015FE324854
:1036600000684079401C3049096848712E4800685C
:103670004079401C2C490968487153E000F0C0F8BB
:1036800000280FD108F05AFD2749096888700120E9
:1036900008F0CEFD244800684079401C22490968A2
:1036A000487105E008F0A2FD00201F490968487133
:1036B00038E01D480068807818280CD102201A498B
:1036C00009680870002018490968487004201649E4
:1036D0000968C87011E0144800684078401C12491D
:1036E00009684870104800684078032805D300F046
:1036F00027F900200C490968487008F077FD002080
:103700000949096848710DE008F070FD002006497C
:1037100009684871044909684870AA200249096883
:10372000887000BF00BF10BDD0070020142F0020FC
:1037300010B5314800684079002804D001280CD029
:10374000032848D11DE008F027FD2B480068407988
:10375000401C2949096848714BE0284909690878E3
:1037600008F092FD244800684079401C224909680D
:103770004871214800684079401C1F490968487118
:1037800037E000F03DF800280CD101201A49096803
:103790000870002018490968487004201649096813
:1037A000C87011E0144800684078401C124909684C
:1037B0004870114800684078032805D300F0C0F82D
:1037C00000200D490968487008F010FD00200A49E2
:1037D000096848710DE008F009FD002006490968F4
:1037E0004871054909684870AA200349096888702A
:1037F00000BF00BF10BD0000D0070020142F002024
:1038000010B508F093FC04461F48006800780028B3
:1038100038D01D480068C078042833D3002C09D163
:10382000002119480068C07A8200174800681430E7
:10383000815027E014480068C07A8100124800686F
:10384000143040581149884211D20F480068C07A9C
:1038500081000D48006814304058401C0A4909682E
:10386000C97A8A0008490968143188500AE000F0D2
:1038700067F8002104480068C07A820002480068A6
:1038800014308150204610BDD0070020B80B000036
:1038900000B587B0012069460871084802900848C1
:1038A000039008480490084805900848069001A92C
:1038B000074800F00FF807B000BD0000F93B010019
:1038C00051570100190202004D1202004C12020071
:1038D000B0280020F8B506460F46002400253946DA
:1038E000304600F0EFF900BF14E000250EE00021A3
:1038F000242060430B4A12688018415524206043FD
:10390000094A126880184155681CC5B2242DEED3AF
:10391000601CC4B205480078A042E6DC00F010F854
:10392000F8BD0000C8070020CC070020142F00209D
:10393000012002490968087170470000D007002083
:1039400010B500F073F900200349096808700249B6
:103950000968C87010BD0000D00700200748006843
:10396000C078062808D105480068C079002803D12E
:10397000012002490968C87170470000D007002083
:1039800010B555480068C07803000CF07FFB08674D
:103990001D1A1714110E056650484068002803D000
:1039A0004E4841680020884793E000F0E5F890E039
:1039B00000F0C6F88DE000F0D1F88AE0FFF7B8FE1D
:1039C00087E0FFF7C7FD84E044484068002803D043
:1039D00042484168012088473F480068407C0028F1
:1039E0001AD03E48C068002803D03C48C168C820AF
:1039F00088470020384909684862374800680078DD
:103A0000002804D0042034490968C87024E002204A
:103A100031490968C8701FE02F480068406A401C9F
:103A20002D49096848622C480068406A7D21C90018
:103A3000884211D300202849096848622648006856
:103A40000078002804D0042023490968C87003E0E6
:103A5000022021490968C8703BE000BF1F48406848
:103A6000002803D01D484168002088471A48006894
:103A7000407C002813D01948C068002803D017489C
:103A8000C168C82088470020134909684862124865
:103A90000068C078401C10490968C87018E00E48DA
:103AA0000068406A401C0C49096848620A4800687E
:103AB000406A7D21C90088420AD30020064909686E
:103AC000486205480068C078401C03490968C8700E
:103AD00000BF00BF10BD0000D0070020142F002041
:103AE00010B515480068C078072824D00120124975
:103AF0000968487408E011488068002802D00F491E
:103B000088688047FFF73CFF0B480068C0780628AC
:103B1000F1D109480068007A0028ECD10648006815
:103B2000C0790028E7D104480068807A0028E2D1F3
:103B300001490968487410BDD0070020142F0020E7
:103B400010B5054800680078012802D1FDF702FF92
:103B500001E0F5F7CDFD10BDD007002010B50548F8
:103B600000680078012802D1FEF720F901E0F6F79D
:103B70009DF910BDD007002010B51D480068807A5F
:103B8000002829D11A480068007A002803D00220B2
:103B900017490968887216480068C079002803D060
:103BA00001201349096888721148006800790128CA
:103BB00012D100200E49096808710D490968887200
:103BC00007200B490968C8700A484068002803D0DC
:103BD00008484168002088470548006800780128A7
:103BE00002D1FEF7BDF901E0F6F73AFA10BD000088
:103BF000D0070020142F002010B5044621460848A5
:103C000001F0CCFC07480078002805D1002C03D037
:103C100032210548FCF774FD0248047010BD000015
:103C2000010300000201002050C3000000202449CD
:103C300009684870AA202249096888700020204934
:103C4000096848621E49096808711D490968487178
:103C50001B49096888711A490968C87118490968B7
:103C6000087217490968887215490968C8721449A9
:103C700009680873242012490968487310490968C3
:103C800088730F490968C87300200D4909680874D2
:103C90000B49096848740A49096888740849096821
:103CA000C8740749096848610021054800688161B6
:103CB00003480068C1610248006801627047000063
:103CC000D007002010B50A780D4B18600346283342
:103CD0000C4C236024235343044628341B190A4CFC
:103CE00023600A4C4B6863608B68A360CB68E36019
:103CF0004B6963610B6923610B78237010BD000071
:103D0000D0070020C8070020CC070020142F002077
:103D100007480068C078062808D105480068007A7E
:103D2000002803D101200249096808727047000089
:103D3000D007002010B50446012C09D1FF22202114
:103D40000020FFF7F5FB0121084604F0DBF808E04E
:103D5000002220211046FFF7EBFB0021012004F098
:103D6000D1F810BD10B50024032000F00DFB002891
:103D700001D0012400E00024204610BD10B5044607
:103D8000032C0ED1FF2215210020FFF7D1FB0022CA
:103D900014211046FFF7CCFB01210E2004F0B2F8ED
:103DA00039E0022C1CD1FCF7E7FF002809D0FF22E4
:103DB00014210020FFF7BCFB01210E2004F0A2F823
:103DC00008E0002214211046FFF7B2FB00210E206C
:103DD00004F098F8002215211046FFF7A9FB1AE01D
:103DE000012C0ED1FF2214210020FFF7A1FB01219D
:103DF0000E2004F087F8002215211046FFF798FBEB
:103E000009E0002215211046FFF792FB0022142141
:103E10001046FFF78DFB10BD10B50024F8F7F8FD34
:103E2000094988420DD3FCF7FFFF002807D1FCF7B2
:103E300071FE012801DD032404E0022402E00224D3
:103E400000E00124204610BDB80B000010B5044668
:103E5000012C09D1FF221D210020FFF769FB012160
:103E6000002004F04FF808E000221D211046FFF763
:103E70005FFB0021084604F045F810BD10B5002492
:103E8000022000F081FA002801D0012400E0002483
:103E9000204610BD10B50446012C09D1FF221E2179
:103EA0000020FFF745FB0121092004F02BF808E072
:103EB00000221E211046FFF73BFB0021092004F0E1
:103EC00021F810BD70B5002400250026FCF7DEFCAB
:103ED0000546FCF7E7FC064602210848F7F72CF9EF
:103EE000552800D108E0012E01D1002404E0012D65
:103EF00001D1012400E00024204670BD50080020BC
:103F000010B50446012C09D1FF221F210020FFF724
:103F10000FFB0121082003F0F5FF08E000221F211C
:103F20001046FFF705FB0021082003F0EBFF10BD52
:103F300070B500240025FCF733FD054603211A481F
:103F4000F7F7FAF8552806D1012018490880002013
:103F50001749088023E016480088012811D1144928
:103F60000880FCF737FC762803DA01200F49088027
:103F700015E0FCF72FFC782811DB00200B490880A6
:103F80000DE001200A490880FCF724FC762803DABA
:103F900001200649088002E0002004490880034807
:103FA0000488204670BD0000500800201E0100203B
:103FB0002001002010B50446012C09D1FF22212147
:103FC0000020FFF7B5FA0121072003F09BFF08E06E
:103FD000002221211046FFF7ABFA0021072003F051
:103FE00091FF10BD10B50024FCF7ACFD002801D1F5
:103FF000012400E00024204610BD10B50446012C29
:1040000009D1FF2216210020FFF792FA0121032097
:1040100003F078FF08E0002216211046FFF788FA27
:104020000021032003F06EFF10BD10B50024052011
:1040300000F0AAF9002801D0012400E00024204665
:1040400010BD10B50446012C09D1FF221921002012
:10405000FFF76EFA0121052003F054FF3CE0022C2B
:1040600017D1FCF789FE002809D0FF221921002072
:10407000FFF75EFA0121052003F044FF2CE0002247
:1040800019211046FFF754FA0021052003F03AFFEA
:1040900022E0032C17D1FCF775FE002809D0FF227F
:1040A00019210020FFF744FA0121052003F02AFF1F
:1040B00012E0002219211046FFF73AFA00210520EC
:1040C00003F020FF08E0002219211046FFF730FA24
:1040D0000021052003F016FF10BD000010B50024DC
:1040E000FCF764FD01282FD104211948F7F724F8C3
:1040F000552801D1012428E0FCF7E0FB01280BD072
:10410000FCF7DCFB022807D0FCF7D8FB032803D020
:10411000FCF7D4FB052801D1012416E0FCF7CEFB07
:10412000042801D1022410E0FCF7C8FB062801D1C5
:1041300003240AE0FCF7C2FB002803D0FCF7BEFB17
:10414000072802D1002400E00024204610BD000012
:104150005008002010B50446012C0ED1FF221B216F
:104160000020FFF7E5F900221A211046FFF7E0F9D9
:1041700001210A2003F0C6FE1EE0022C0ED1FF2210
:104180001A210020FFF7D4F900221B211046FFF767
:10419000CFF901210A2003F0B5FE0DE000221A211B
:1041A0001046FFF7C5F900221B211046FFF7C0F9A2
:1041B00000210A2003F0A6FE10BD10B50024FCF774
:1041C000E7FD022803D0FCF7D3FE022807D1FCF755
:1041D0009DFE012801D1012402E0022400E0022416
:1041E000204610BD10B5F8F72DFC0446204610BD42
:1041F00010B5034B08220349034800F013F910BD22
:10420000E5410100EC1102007028002070B506465F
:104210005C488068002804D05A4988688047054671
:1042200000E000250024A6E0564841680C206043C9
:1042300008184088A84207D0524841680C206043C3
:104240000818408802287DD14E4841680C20604300
:104250000818806800280CD04A494A680C2161433C
:1042600051188868804747490968E20089184870F2
:1042700009E0444841680C206043095C41480068FB
:10428000E200801841703F480068E1004018407823
:104290003C490968E200895C88420FD039480068CF
:1042A000E1004018417837480068E200815400205E
:1042B00034490968E200891848605AE031480068CA
:1042C000E100401841782F4842680C2060431018E4
:1042D000407881421FD12B480068E10040184168B6
:1042E000284842680C2060431018808881420BD80F
:1042F00024480068E1004018406880192149096895
:10430000E2008918486034E001201E490968E20093
:10431000891848802DE01B480068E100401841687A
:10432000184842680C2060431018C08881420DD89C
:1043300014480068E100401840688119114800687D
:10434000E20000E009E08018416012E000200D4921
:104350000968E200891848800BE0002009490968D3
:10436000E20089184880002106480068E2008018B1
:104370004160601C84B203488089A04200DD53E79D
:1043800070BD0000CC2E00200146064A92898A4268
:1043900005DD044A1268CB00D218508800E00020E6
:1043A00070470000CC2E0020002000BF14E00D4913
:1043B0004A680C2141435118498801290AD100213A
:1043C000084A1268C300D2185180064A1268C30016
:1043D000D2185160411C88B2024989898142E6DCC9
:1043E00070470000CC2E0020002000BF13E00C49D5
:1043F0004A680C21414351184988002909D1084ACB
:104400001268C300D2185180054A1268C300D2183E
:104410005160411C88B2024989898142E7DC7047BA
:10442000CC2E0020F0B504460020164DAB6069602C
:104430002C60AA8100BF1FE0124D6E680C25454319
:10444000755D104E3668C700F61975700D4D6E68B3
:104450000C254543755D0B4E3668C700F5550025A4
:10446000084E3668C700F6197580064E3668C700D4
:10447000F6197560451CA8B2024DAD898542DBDC9A
:10448000F0BD0000CC2E002070B505460E46002E73
:1044900005D031462846F3F753FE044600E02C468B
:1044A000204670BD10B5FCF74DFB00280DD1074824
:1044B0000078012809D005480078032805D0044871
:1044C0000078002801D1F8F799FF10BDF500002011
:1044D000F400002008B50020009001226946052064
:1044E000F9F722FE05490098886000200449087009
:1044F000044908700449087008BD000038280020ED
:10450000F4000020F6000020F700002008B500208D
:104510000090012269460520F9F706FE00200249B5
:1045200008710098886008BD3828002070B5049C88
:104530002578914216DD01280AD18D4206DAFF2640
:10454000F61AAE420ED3EE18F5B20BE0154609E0AE
:10455000022807D1954204DD9D4203DBEE1AF5B235
:1045600000E00D46257070BD0D4A416851608169BB
:104570009161C168D160416A5162016A116201684A
:1045800011604169516181689160C169D1610169BE
:104590001161816A91620021024A11707047000026
:1045A000E82E0020C407002010B5FFF7FDFEF8F745
:1045B0008FF800210148F6F7C9FE10BD5C08002005
:1045C00010B5F8F785F8FFF70FFF09F03FFD09F088
:1045D000DBFDFBF7DDFBFAF70FF9FFF77BFFF8F7E1
:1045E000B1FCF6F7AFFCF9F7E3F955210548F6F70A
:1045F000ADFEF8F7DFFAF9F759F9FBF789F8F6F7A6
:104600009BFE10BD5C0800201CB5002032490870DC
:1046100007F072FD0020FCF70BFD0CF05FF8F7F7D8
:1046200093F955212D48F6F791FEF8F7C3FAF9F7FB
:104630003DF9F6F77FF8F6F7FDFAE12040020BF0BE
:104640008FFC00F071FAF6F77DFC07F035FFF8F704
:104650003FF8F9F717FFF8F701FDF8F77FFCFFF7D0
:10466000C7FDFEF781F8FFF713F9FFF739FAF9F7FD
:10467000FBFDFBF7B9FBFAF7BFF8194AFF219131AF
:10468000012009F047FE00221146012009F086FDB5
:1046900009F0C2FC09F078FDFFF738FFF9F7B6F929
:1046A0000020104988714871087101208870487095
:1046B0001420087007226846F3F7D9FD0199009885
:1046C00000F0BCFF0221012000F094FEFBF720F86F
:1046D000F6F732FE1CBD0000010100205C0800203E
:1046E0000090D003120100207047000010B504466E
:1046F000552C03D105494869804702E00349086801
:10470000804700200249087010BD0000E82E0020FC
:10471000C407002010B54648007803000BF0B6FC33
:104720000A06111B26303B465051738141484068B0
:10473000002802D03F494868804701203C49087062
:1047400000BF3C488068002804D03A498868804708
:104750003749087069E03748C068002802D03549F9
:10476000C868804703203249087000BF314800699B
:10477000002804D02F49086980472D49087054E06B
:104780002C484069002802D02A4948698047002007
:104790002749087049E027488069002802D0254948
:1047A0008869804706202249087000BF2148C069F7
:1047B000002804D01F49C86980471D49087034E0AB
:1047C00000BF1B48007807280AD11A48006A002851
:1047D00002D01849086A804709201549087011E07D
:1047E0001348007808280AD11248406A002802D0ED
:1047F0001049486A804709200D49087002E00020EE
:104800000B49087000BF0A480078002808D0094802
:10481000806A002804D00749886A804704490870E4
:1048200003E000200249087000BF00BF10BD000077
:10483000C4070020E82E00207047000010B50020BB
:104840000CF008F808F012FD08F066FD08F07CFD99
:1048500000F0C4FCF6F77EFA0220FCF7E9FB00202A
:1048600007490870FFF73CF9FFF762F8FFF788F88F
:10487000F6F7D0F810200AF063F900F0AFFD10BD94
:104880009801002010B5012408F0BEF8012801D1DC
:10489000052407E0F8F7B6F80349884201D201245D
:1048A00000E00224204610BD204E000010B5062472
:1048B00008F0AAF8002800D1002408F0ABF801287D
:1048C00003D008F0A7F8072800D90924204610BD16
:1048D00010B5F6F73FFA00221146012009F090FDCD
:1048E00000213C48F6F732FD00203B4908800024B7
:1048F00000BF00F02DFF32217D200001FBF700FFFB
:104900000020364908700AE0002234480178104639
:10491000FEF70EFE31480078401C304908702F48E1
:1049200000782428F0DB00202D49087009E00021E0
:104930002B48007809F078F929480078401C28496C
:104940000870274800780D28F1DBFFF719F8F5F714
:1049500037FF07F0ABFF23480078401C214908705F
:1049600008460078052812D300200870FEF7F6FFED
:104970001D4800780A2805D300201B490870FFF75E
:10498000C7F904E018480078401C1749087008F07F
:1049900041F80128ADD908F03DF80728A9D2002038
:1049A0000F49087008E00E48007809F057F90C48E4
:1049B0000078401C0A490870094800780D28F2DB8D
:1049C000F6F738F955210348F6F7C0FCF7F7F0FF82
:1049D000204610BD5C0800207C0000201B01002048
:1049E000190100201A0100201C01002010B5032429
:1049F00008E000F0ADFE012000F0B4FD002801D079
:104A0000042400E0F5E700BF204610BD10B50020EB
:104A10002949086007F070FB0120FCF709FBF6F755
:104A200093FF55212548F6F791FCF8F7C3F8F8F7FE
:104A30003DFF0BF053FEF5F77DFEF9F7EBFCF6F7C3
:104A4000F9F807F043FFF9F71DFDF9F7B9FEF8F79C
:104A500005FBFFF7CDFBFDF787FEFFF7C5FCFFF772
:104A600039FDFEF715FFFFF73BF800F05DF8E12098
:104A700040020BF075FAF6F765FAFBF7B5F9F9F7AE
:104A8000BBFE0F4AFF219131012009F043FC0022B7
:104A90001146012009F082FB09F0BEFA09F074FB0F
:104AA000F8F786FF0221012000F0A4FCFAF730FE9F
:104AB000F6F742FC10BD0000500000205C0800200A
:104AC0000090D00370B506460D4614460E480660A9
:104AD0000E4805600E49206808600E49606808604D
:104AE0000D49A06808600D49206908600C49E0681C
:104AF00008600C496069086005480068002802D019
:104B000003480068804770BDC8000020D000002026
:104B1000B0000020B4000020B8000020BC0000203D
:104B2000C0000020C400002000B587B00C480190F0
:104B30000C4802900C4803900020049005900B480C
:104B4000069000200A49086048600A4908604860E9
:104B500001AA0121C9020848FFF7B4FF07B000BD50
:104B60007D4B0100214F0100A94E0100D54D0100F0
:104B70006C120020640A0020741700200120704786
:104B8000F3B5C3B00446449E0020009057E002E015
:104B9000641C761E00BF022E05D32078EB28F7D1C7
:104BA00060789028F4D1072E00D24AE0A778FD1C47
:104BB000B54200D945E0A81E205C0002691E615C78
:104BC00008434290042D38D9291FA01C0BF0A0FDEA
:104BD0004299884226D11D480068002804D0B91E99
:104BE000E01C1A4A1268904719480068002824D02F
:104BF000E178684601712079811168464171207918
:104C00008106890E68468171381FC1B26846C1713C
:104C1000C279611D02A8F3F72AFB01A80C490968B3
:104C200088470AE00020009002E00098401C0090B5
:104C30000098A842F9D3002000906419761B072E33
:104C4000A5D200BF4498801B45B0F0BDBC00002039
:104C5000C4000020F7B5C0B0154600260027E81DA7
:104C6000FF210131884202DD002043B0F0BDEB217D
:104C70006846017090214170281DC1B2684681705C
:104C80000021C1704098C1B2684601710524002618
:104C900005E04198805D69460855641C761CAE426B
:104CA000F7DBA11E00A802300BF032FD07463812D8
:104CB00069460855641C0F55641C064800680028A6
:104CC00005D021466846034A12689047CDE7002088
:104CD000CBE70000B400002070B5002400250026BA
:104CE0001B4840681A490968884200D170BD1848BD
:104CF000406817490968884205D915484068144931
:104D00000968451A07E01248006811494968401AC5
:104D1000012189020D1AFF2D01D9FF2600E02E4640
:104D200000240DE00A4801680830405C0949085534
:104D300007480088401C8005800D05490860641CF8
:104D4000B442EFD3B1B203480BF066F900BFCDE730
:104D50006C1200207416002070B500251A480068F7
:104D6000002830D0194A1288FF230133991A184AB3
:104D70001268164B1B88D018134A126890470546D4
:104D8000002D20D01148008840191049088008469D
:104D900001880F480068FFF7F3FE0446002C0DDD84
:104DA0000A480088844209DA08480088021B08483B
:104DB0000068011906480068F3F759FA03480088AB
:104DC000001B0249088070BDB8000020CC00002004
:104DD000C800002038B5044600200090A0781028B4
:104DE0000CD120792D49087008460078012853D14C
:104DF000002211462020FFF72DFF4DE0A078122859
:104E000003D120792549087246E0A078052803D10E
:104E10002079224988723FE0A07802281DD12079AC
:104E20001E4948720846407A012806D100900122A6
:104E300069460420FFF70EFF2EE01848407A02284A
:104E40002AD100BFBFF34F8F15481649C860BFF382
:104E50004F8F00BF00BF00BFFDE7A07801281BD126
:104E60002079332803D101200C49487005E02079CE
:104E7000352802D1002009494870607907498870B7
:104E8000607A0006217A09040843E179090208439F
:104E9000A17908430149486038BD0000580A002044
:104EA0000400FA0500ED00E070B50346002200247E
:104EB00000251A484068194E3668B04201D10020DA
:104EC00070BD16484068154E3668B04205D9134883
:104ED0004068124E3668841B07E0104800680F4E89
:104EE0007668801B0126F602341AA14201D92546B4
:104EF00000E00D4600220CE0084806680830805D9E
:104F0000985406480088401C4005400D034E306010
:104F1000521CAA42F0D32846D2E70000640A0020BF
:104F200070B503460022002415484068144D2D68D2
:104F3000A84208D312484068114D2D68401B012536
:104F4000AD022C1A04E00E4800680D4D6D68441B3C
:104F5000A14201D9012070BD00220CE09D5C0848EF
:104F600046680830855508388088401C8005800DCB
:104F7000034D6860521C8A42F0D30020EBE700002A
:104F80006C12002010B50248FFF7EEFA10BD0000C9
:104F9000D41202000021014A1175704740600040A0
:104FA000014600BFF020084000110A235843024682
:104FB0000807000F8018C0B270470146002204E0C5
:104FC000501CC2B208460A38C1B20A29F8DA1007E2
:104FD000000E08437047000010B5044601218020F0
:104FE000F6F73EFA607A012805D14248C0781021D0
:104FF00008434049C870607AA22805D13E48007F26
:10500000802108433C490877607A3B4908770020B3
:105010003A4948770846407F21780843374948771E
:10502000E07B002805D00846407F20210843334913
:1050300048773248407FC008C000A17A08432F4912
:1050400048770846807FF72108402C498877E07828
:10505000FFF7B3FF29498874A078FFF7AEFF27490F
:10506000C8746078FFF7A9FF2449087520780028E4
:1050700005D10846007D2179084320490875E0796B
:10508000FFF79BFF1D4988756079FFF796FF1B4965
:105090004875A079FFF791FF1849C875207AFFF786
:1050A0008CFF164908760846807F4006400E8877B8
:1050B000E07A002806D00846807F402108430F4947
:1050C000887703E00D48807F0C498877A07BFFF745
:1050D00074FF0A498876607BFFF76FFF0749C8763F
:1050E000207B08770846807F102188430349887712
:1050F00010BD00002004024060040440404F044002
:1051000010B504461B48807F012108431949887760
:105110002078FFF752FF174908756078FFF74DFFB9
:105120001449C874A078FFF748FF124988742078A2
:105130000C2806DD0846407F082108430D494877C2
:1051400009E00C48407F0B4948770846007DE1782C
:105150000843084908750748807F40084000054912
:10516000887700BF0348807F022108400028F9D1DA
:1051700010BD0000404F044010B5002014490876CF
:1051800016200AF0A9FF0021124801761248407F3C
:1051900080210843104948770846807F0121084351
:1051A0000D49887700BF0C48807F02210840002805
:1051B000F9D00948807F400840000749887700BF40
:1051C0000548807F022108400028F9D110BD000069
:1051D0004060004040610040404F044010B5002056
:1051E0000749087000212020F6F73AF90121054807
:1051F000017500200449087515200AF055FF10BDFF
:1052000000500440406100404060004070B50446DA
:105210000D46002C14D0002D12D0042D10D800F013
:1052200013F800280CD1002608E00649885D2246C4
:105230000121F4F79BF8A41C701CC6B2AE42F4DB4B
:1052400070BD00005012020000200549897DC90789
:10525000C90F002901D0012000E0002070470000A4
:105260000050044030B585B005460C460020039040
:105270000490009001900290072C0BDC0120A040CC
:1052800081B2684681810121C17303A90220FAF726
:10529000EBFE3EE0082C01D0092C0BD10120A040F0
:1052A00081B2684681810121C17303A90120FAF707
:1052B000DBFE2EE00A2C03D00B2C01D00D2C0BD1E1
:1052C0000120A04081B2684681810121C17303A9F8
:1052D0000020FAF7C9FE1CE00C2C01D00F2C0BD1DA
:1052E0000120A04081B2684681810121C17303A9D8
:1052F0000E20FAF7B9FE0CE00E2C0AD10120A040D6
:1053000081B2684681810121C17303A90C20FAF79B
:10531000ABFE002168460170C170417001218170AF
:1053200000210171C1720D218172FF2101720021E2
:105330004172F4F77BF803491520FDF7DFF805B05B
:1053400030BD0000954F010010B5002010490875D0
:1053500015200AF0A9FE00210E480175152000282D
:1053600009DB00BF00BFC206D20E012191400A4AEC
:10537000116000BF00BF00BF08488079801103287A
:1053800005D006480078802108430449087010BD04
:10539000406000404061004000E100E000500440F7
:1053A00010B5F4F73DF910BD10B501231A460021E0
:1053B0001846F6F711F8012211461046F6F782F862
:1053C000F6F76EF803480BF07BF9024802490860D3
:1053D00010BD00000090D0034807002000BF044823
:1053E0000069042108430249086130BF00BF7047CB
:1053F00000ED00E0F3B585B0054600240027002647
:10540000002003900490EEB22804070E0F2F54DA08
:10541000082E52DA002009E00C214143284A515A53
:10542000A94201D1044603E0411CC8B21728F3D3B6
:1054300000BF0120B04086B20C20604320494018D4
:10544000C3780C20604340188278F8B2314601904E
:10545000FAF7AEFE68468681012181730021C1738F
:1054600002214174F8B203A9FAF7FEFD0C21614351
:10547000134A8918C888FBF701FF0C2060431049C4
:105480004018C1886846018169460698887202A85A
:10549000FBF70EFE0C226243094BD21891680C22D6
:1054A0006243D21804201056FDF728F80C216143FE
:1054B000034A8918C888FBF765FE07B0F0BD0000F5
:1054C0006C140200FEB505460C460020C043029055
:1054D000EFB22804060E0F2E42DA082F40DA012020
:1054E000B8406946088080202040002816D101205D
:1054F0008870A007800F022801D1487109E0A00739
:10550000800F012802D16946487102E000206946F7
:105510004871F0B26946FAF7A7FD1FE0002069461E
:1055200088700E202040002800D000BF10202040AE
:10553000002802D16946087102E00120694608711D
:10554000E007C00F002802D16946887102E00120FF
:1055500069468871F0B26946FAF786FD002002902C
:105560000298FEBD30B50146CAB20C04230E0020DD
:105570000F2B0FDA082A0DDA01249440A2B2064C50
:1055800003252D026419E45C1440002C01D0012095
:1055900000E0002030BD000000000440F8B50446E3
:1055A0000F460020C0430090E6B22004050E0F2DE8
:1055B00011DA082E0FDA0120B04086B2002F04D194
:1055C000E8B23146FAF74CFE03E0E8B23146FAF7AA
:1055D00057FE002000900098F8BD00001649897F12
:1055E00001221143144A917700BF1349897F022297
:1055F00011400029F9D01049897C81700E49C97C7D
:1056000041700D49097D01700B498A7D8271497D88
:1056100001710949CA7D42710A7EC271897F4908B8
:105620004900054A917700BF0349897F0222114052
:105630000029F9D170470000404F044003B585B000
:10564000002001900290039004900021684641736D
:10565000817E01A8C1706846417E01A881706846BC
:10566000017E4171002101A8017108216846017184
:10567000817D01A8C1716846C17D4172417D01A84B
:1056800081716846017D01A801720021684681731D
:10569000C17301A881730C214173412168460174D3
:1056A0000021C17401A8FFF797FC1A2004498882E1
:1056B00004491620FCF722FF00F006F807B000BDF1
:1056C000204F04400D08020010B5FFF755FD10BD36
:1056D00070B504460D46601E0D49884200D901246C
:1056E000002C00D1012440200A49087008460078A7
:1056F0006043094948610321081F0AF005FD0020A5
:1057000005498861072008610448056070BD0000F4
:10571000FFFFFF007401002000E000E070010020A6
:105720000020C043002809DBC206D20E01219140AF
:10573000054A1160BFF34F8FBFF36F8F00BF00208A
:10574000024908618861704780E100E000E000E004
:1057500010B50AF07FFC10BD1A20084908722B20F2
:1057600048723C2088724D20C8727F200449096825
:105770000860AC20034948707047000000040240F4
:10578000780100200010024010B51C480078012864
:1057900012D11B480078642809DB0220194948719E
:1057A00008710020164908701449087004E0144874
:1057B0000078401C124908701348007801281CD159
:1057C00012480078012804D10020104908701049BF
:1057D00008700F48007832280ADBF7F733FA002107
:1057E0000C48F5F763FD55210B48F5F7AFFD04E0D4
:1057F00007480078401C0649087010BD15070020B6
:1058000014070020040700200E07002010070020C6
:105810000F070020500800205C080020F8B504465F
:105820000D460027002000900320000320400013B5
:105830000090102C04D0122C02D01148844217D1B1
:1058400022202840222806D127073F0F39460098FA
:10585000F4F75CFF06461220284012280ED12007DC
:10586000000F471C39460098F4F750FF064605E044
:105870002107090F0098F4F749FF06463046F8BDA6
:1058800010100000F8B504460D4600260027012040
:10589000000320400713102C04D0122C02D00F4814
:1058A000844215D122202840222805D12607360F10
:1058B00031463846FAF7D0F81220284012280CD189
:1058C0002007000F461C31463846FAF7C5F804E0B9
:1058D0002107090F3846FAF7BFF8F8BD101000008D
:1058E000FFB58BB01C460020079006900590384805
:1058F000049010210B980840002801D0022707E0EF
:1059000040210B980840002801D0012700E0002723
:10591000002C04D0149804700120089001E010209D
:105920000890002548E0002C08D025466000294A50
:10593000115A0C98F2F704FC079006E06800254A1B
:10594000115A0C98F2F7FCFB07903E4630E0711CB0
:105950000798F2F7F5FB400806900D98F2F746FD20
:1059600003900D9A0699881AF2F740FD18490190A4
:10597000F2F7C1FC02900399F2F7FAFC0590059842
:10598000F2F73BFD49004908039102900498F2F7B1
:1059900034FD4900490801910090039B029AF2F7F7
:1059A00041FD03D20A95099605980490701CC6B271
:1059B0007F2ECCDD681CC5B208988542B3DB1499F4
:1059C0000A98087014990998487004980FB0F0BDAF
:1059D0000000C842801502000246412A2ED010DC89
:1059E000212A2AD006DC102A45D0122A4BD0202AA0
:1059F00059D11CE0222A26D0232A2AD0402A52D16B
:105A000016E081235B01D01A9A4228D008DC422A92
:105A10001AD0432A1ED025481018002843D13AE056
:105A2000012822D020281BD021283CD11EE000BF15
:105A30001F4803890B43038136E000BF1C4843899C
:105A40000B43438130E000BF194883890B438381B6
:105A50002AE000BF1648C3890B43C38124E000BF7E
:105A6000144883880B4383801EE000BF1148C3881D
:105A70000B43C38018E00E4843890B4343810389DD
:105A80000B43038110E00A48C3890B43C381838918
:105A90000B43838108E00748C3880B43C380838896
:105AA0000B43838000E000BF00BF7047F0EFFFFFB3
:105AB0000011044000140440F0B505460E46412D87
:105AC00030D010DC212D2CD006DC102D51D0122D21
:105AD00056D0202D62D11CE0222D2AD0232D30D08B
:105AE000402D5BD116E081214901681A8D4230D0EA
:105AF00008DC422D1ED0432D24D02A482818002827
:105B00004CD144E001282CD0202823D0212845D195
:105B100028E000BF244F3888314600F049F8044699
:105B20003DE000BF204F7888314600F041F8044640
:105B300035E000BF1C4FB888314600F039F8044604
:105B40002DE000BF184FF888314600F031F80446C8
:105B500025E000BF154F3888314600F029F804468B
:105B60001DE000BF114F7888314600F021F804464F
:105B700015E00D4F7888314600F01AF804460EE023
:105B8000094FF888314600F013F8044607E0074F44
:105B90007888314600F00CF8044600E000BF00BFF2
:105BA0002046F0BDF0EFFFFF001104400014044058
:105BB0000246002013460B40002B01D0012000E0DC
:105BC00000207047FFB581B00E461746012F07D160
:105BD000F748407D00090001C01DF549487505E002
:105BE000F348407D00090001F149487504980128F7
:105BF0007ED10A210198F2F7A3FA0546ED48445DEB
:105C0000E007C00F002807D0E948007C0009000128
:105C1000C01DE749087405E0E548007C0009000163
:105C2000E349087402202040002807D0E048C07BE8
:105C3000F02188437030DE49C87305E0DC48C07B42
:105C4000F0218843DA49C87304202040002807D097
:105C5000D748807C00090001C01DD549887405E043
:105C6000D348807C00090001D14988740820204075
:105C7000002807D0CE48407CF02188437030CC49C2
:105C8000487405E0CA48407CF0218843C8494874FC
:105C900010202040002807D0C548407C00090001A2
:105CA000C01DC349487405E0C148407C000900019B
:105CB000BF49487420202040002807D0BC48007C01
:105CC000F02188437030BA49087405E0B848007C78
:105CD000F0218843B649087440202040002808D0AD
:105CE000B348807CF02188437030B149887406E065
:105CF0008BE0AF48807CF0218843AD4988740A214D
:105D00000198F2F71DFA0D46AA48445DE007C00F5E
:105D1000002807D0A648807BF02188437030A44932
:105D2000887305E0A248807BF0218843A0498873EE
:105D300002202040002807D09D48807B00090001F8
:105D4000C01D9B49887305E09948807B00090001CC
:105D50009749887304202040002807D09448007D8C
:105D6000F021884370309249087505E09048007D25
:105D7000F02188438E49087508202040002807D06C
:105D80008B48007D00090001C01D8949087505E0A8
:105D90008748007D000900018549087510202040D2
:105DA000002807D08248C07CF021884370308049A9
:105DB000C87405E07E48C07CF02188437C49C874E3
:105DC00020202040002807D07948C07B000900012E
:105DD000C01D7749C87305E07548C07B0009000104
:105DE0007349C87340202040002807D07048C07C09
:105DF00000090001C01D6E49C87454E06C48C07CA5
:105E0000000900016A49C8744DE06948007C000936
:105E10000001674908740846C07BF0218843644943
:105E2000C8730846807C0009000188740846407CDD
:105E3000F02188435E4948740846407C000900010F
:105E400048740846007CF021884359490874084684
:105E5000807CF0218843564988740846807BF02175
:105E60008843534988730846807B00090001887382
:105E70000846007DF02188434D4908750846007D9D
:105E80000009000108750846C07CF0218843484994
:105E9000C8740846C07B00090001C8730846C07C6E
:105EA00000090001C8740A9801287DD10A213046F2
:105EB000F2F746F905463F48445DE007C00F002869
:105EC00007D03B48407B00090001C01D384948739A
:105ED00005E03748407B000900013549487302203E
:105EE0002040002807D03248007BF02188437030E2
:105EF0002F49087305E02E48007BF02188432C4988
:105F0000087304202040002807D02948807DF02114
:105F1000884370302649887505E02548807DF0214A
:105F200088432349887508202040002807D020484E
:105F3000807D00090001C01D1D49887505E01C48D1
:105F4000807D000900011A49887510202040002832
:105F500007D01748407DF0218843703014494875B8
:105F600005E01348407DF021884311494875202001
:105F70002040002807D00E48407BF0218843703035
:105F80000B49487305E00A48407BF02188430849E3
:105F900048734020204000280ED00548C07D0009ED
:105FA0000001C01D024900E092E0C8750AE000004F
:105FB00048260020C00F02006D48C07D0009000186
:105FC0006B49C8750A213046F2F7BAF80D466948A0
:105FD000445DE007C00F002807D06548C07AF02173
:105FE000884370306249C87205E06148C07AF02188
:105FF00088435F49C87202202040002807D05C48CF
:10600000C07A00090001C01D5949C87205E058480E
:10601000C07A000900015649C872042020400028B7
:1060200007D05348407E00090001C01D5049487602
:1060300005E04F48407E000900014D4948760820A0
:106040002040002807D04A48007EF0218843703065
:106050004749087605E04648007EF02188434449D8
:10606000087610202040002807D04148007E000913
:106070000001C01D3E49087605E03D48007E00094C
:1060800000013B49087620202040002807D03848EE
:10609000007B00090001C01D3549087305E0344844
:1060A000007B00090001324908734020204000288D
:1060B00007D02F48C07DF021884370302C49C87527
:1060C00054E02B48C07DF02188432949C8754DE034
:1060D0002748407B00090001254948730846007B9A
:1060E000F0218843224908730846807DF0218843C7
:1060F0001F4988750846807D00090001887508469B
:10610000407DF02188431A4948750846407BF021BC
:106110008843174948730846C07D00090001C875C7
:106120000846C07AF02188431149C8720846C07AEF
:1061300000090001C8720846407E00090001487647
:106140000846007EF0218843094908760846007E0B
:106150000009000108760846007B00090001087369
:106160000846C07DF02188430149C87505B0F0BDDF
:1061700048260020C00F0200FFB581B00E4617462A
:10618000019801287ED10498002828D1FB48007886
:10619000012824D0F6F73CFCF94988421FD3FAF7CE
:1061A000EBFD00280DD0F748807DF021884370304A
:1061B000F44988750846C07C00090001C01DC874F8
:1061C0001AE0F048807DF02188431030ED49887551
:1061D0000846C07C00090001401CC8740CE0E94876
:1061E000807DF02188437030E64988750846C07C80
:1061F00000090001C01DC874E248C07CF02188433A
:106200007030E049C8740846007EF0218843703041
:10621000DC4908760846807D00090001401C88752D
:106220000846407DF02188431030D649487508461D
:10623000407D00090001401C48750846007DF021A2
:1062400088431030CF4908750846007D00090001D9
:10625000401C0875330009F019FF062E261E140C89
:10626000042FC848007D00090001C01DC5490875FC
:1062700000BFC448007DF02188437030C1490875D3
:1062800000BF00E0AFE1BF48407D00090001C01D34
:10629000BC49487500BFBB48407DF0218843703041
:1062A000B849487500BFB748807D00090001C01D8E
:1062B000B449887500BF00E000BF00BF0498002803
:1062C0005ED1AE48007801285AD0F6F7A1FBAC4960
:1062D000884255D3AB48C07FF0218843A949C8778D
:1062E0000846807F0009000188770846407FF0213A
:1062F0008843A44948770846007FF0218843A14994
:1063000008770846C07DF02188439E49C875084635
:10631000C07F00090001C8770846807FF0218843CC
:10632000984988770846407F00090001C01D4877DA
:106330000846807EF0218843924988760846807E10
:106340000009000188760846407E00090001487671
:106350000846007E0009000108760846007F000913
:10636000000108770846C07EF02188438549C87639
:106370000846407EF0218843703082494876B8E173
:1063800064213846F1F7DCFE0546012D07D17D4832
:10639000C07FF021884370307A49C87705E079489A
:1063A000C07FF02188437749C8770A213846F1F742
:1063B000C7FE0A210090F1F7C3FE0D46642F02D3F9
:1063C0007148445D01E07148445DE007C00F00285A
:1063D00007D06C48807F00090001C01D694988779B
:1063E00005E06848807F000900016649887702203F
:1063F0002040002807D06348407FF0218843703058
:106400006049487705E05F48407FF02188435D4957
:10641000487704202040002807D05A48007FF02108
:10642000884370305749087705E05648007FF021CF
:1064300088435449087708202040002807D0514855
:10644000C07DF021884370304E49C87505E04D4845
:10645000C07DF02188434B49C8751020204000289A
:1064600007D04848C07F00090001C01D4549C877D2
:1064700005E04448C07F000900014249C877202058
:106480002040002807D03F48807FF02188437030AB
:106490003C49887705E03B48807FF02188433949B3
:1064A000887740202040002807D03648407F0009E8
:1064B0000001C01D3349487705E03248407F00099C
:1064C0000001304948770A213846F1F739FE0D4678
:1064D0002D48445DE007C00F002807D02948807E82
:1064E000F021884370302749887605E02548807E72
:1064F000F02188432349887602202040002807D0D5
:106500002048807E00090001C01D1E49887605E0F4
:106510001C48807E000900011A498876042020402A
:10652000002807D01748407E00090001C01D15490A
:10653000487605E01348407E00090001114948767D
:1065400008202040002807D00E48007E00090001E6
:10655000C01D0C49087605E00A48007E00090001CC
:106560000849087610202040002811D00548007FF7
:1065700000090001C01D034908770FE00101002058
:10658000B80B00001C270020C00F0200D30F020030
:106590005948007F00090001574908772020204012
:1065A000002807D05448C07EF021884370305249FB
:1065B000C87605E05048C07EF02188434E49C87631
:1065C00040202040002807D04B48407EF0218843DF
:1065D0007030494948768CE04748407EF021884336
:1065E0004549487685E04448807D000900014249DC
:1065F00088750846407DF02188433F494875084624
:10660000407D0009000148750846007DF02188435F
:10661000394908750846007D0009000108750846DB
:10662000C07C00090001C8740846807DF0218843C1
:10663000314988750846C07CF02188432E49C874CA
:106640000846007EF02188432B4908760846C07F23
:10665000F02188432849C8770846807F0009000157
:1066600088770846407FF0218843234948770846C9
:10667000007FF0218843204908770846C07DF0213B
:1066800088431D49C8750846C07F00090001C877C6
:106690000846807FF0218843174988770846407F65
:1066A0000009000148770846807EF021884312499E
:1066B00088760846807E0009000188760846407E7C
:1066C0000009000148760846007E000900010876AE
:1066D0000846007F0009000108770846C07EF021C7
:1066E00088430549C8760846407EF0218843024920
:1066F000487605B0F0BD00001C27002010B501460B
:10670000002200200A0EFE4B985CC307DB0F002B13
:1067100007D0FC4BDB7FF024A3437033F94CE377C5
:1067200005E0F84BDB7FF024A343F64CE37702232C
:106730000340002B07D0F34BDB7F1B091B01DB1D44
:10674000F04CE37705E0EF4BDB7F1B091B01ED4CC1
:10675000E37704230340002B07D0EA4B9B7F1B0900
:106760001B01DB1DE74CA37705E0E64B9B7F1B0974
:106770001B01E44CA37708230340002B09D0E14B15
:1067800020335B781B091B01DB1DDE4C203463705A
:1067900007E0DC4B20335B781B091B01D94C20340C
:1067A000637010230340002B09D0D64B20331B7895
:1067B000F024A3437033D34C2034237007E0D14B33
:1067C00020331B78F024A343CE4C203423702023A5
:1067D0000340002B09D0CB4B20331B781B091B0136
:1067E000DB1DC84C2034237007E0C64B20331B78D8
:1067F0001B091B01C34C2034237040230340002B92
:1068000007D0C04B9B7FF024A3437033BD4CA377CC
:1068100005E0BC4B9B7FF024A343BA4CA377FF2336
:106820001B040B401A0CB64B985CC307DB0F002B04
:1068300007D0B44B1B7F1B091B01DB1DB14C237719
:1068400005E0B04B1B7F1B091B01AE4C23770223D5
:106850000340002B07D0AB4BDB7EF024A343703307
:10686000A84CE37605E0A74BDB7EF024A343A54CC0
:10687000E37604230340002B07D0A24B9B7EF02439
:10688000A34370339F4CA37605E09E4B9B7EF02480
:10689000A3439C4CA37608230340002B07D0994BBD
:1068A0005B7FF024A3437033964C637705E0954BF0
:1068B0005B7FF024A343934C637710230340002BAA
:1068C00007D0904B5B7F1B091B01DB1D8D4C637751
:1068D00005E08C4B5B7F1B091B018A4C63772023EF
:1068E0000340002B07D0874B1B7FF024A34370335A
:1068F000844C237705E0834B1B7FF024A343814C1A
:10690000237740230340002B07D07E4BDB7E1B09FF
:106910001B01DB1D7B4CE37605E07A4BDB7E1B091C
:106920001B01784CE376FF231B020B401A0A744BC1
:10693000985CC307DB0F002B07D0724B1B7EF02443
:10694000A34370336F4C237605E06E4B1B7EF0241F
:10695000A3436C4C237602230340002B07D0694BE2
:106960001B7E1B091B01DB1D664C237605E0654B76
:106970001B7E1B091B01634C237604230340002B61
:1069800007D0604BDB7D1B091B01DB1D5D4CE375F4
:1069900005E05C4BDB7D1B091B015A4CE3750823AA
:1069A0000340002B07D0574B9B7E1B091B01DB1DAF
:1069B000544CA37605E0534B9B7E1B091B01514CA5
:1069C000A37610230340002B07D04E4B5B7EF024B0
:1069D000A34370334B4C637605E04A4B5B7EF02457
:1069E000A343484C637620230340002B07D0454B3C
:1069F0005B7E1B091B01DB1D424C637605E0414BAE
:106A00005B7E1B091B013F4C637640230340002B38
:106A100007D03C4BDB7DF024A3437033394CE37546
:106A200005E0384BDB7DF024A343364CE375CAB256
:106A3000334B985CC307DB0F002B07D0314B1B7D1A
:106A4000F024A34370332F4C237505E02D4B1B7DA1
:106A5000F024A3432B4C237502230340002B07D0C3
:106A6000284B1B7D1B091B01DB1D264C237505E0F4
:106A7000244B1B7D1B091B01224C2375042303405F
:106A8000002B07D01F4BDB7C1B091B01DB1D1D4CA2
:106A9000E37405E01B4BDB7C1B091B01194CE37401
:106AA00008230340002B07D0164B9B7CF024A34304
:106AB0007033144CA37405E0124B9B7CF024A34369
:106AC000104CA37410230340002B07D00D4B5B7DAB
:106AD000F024A34370330B4C637505E0094B5B7DD9
:106AE000F024A343074C637520230340002B0BD0F5
:106AF000044B5B7D1B091B01DB1D024C637509E028
:106B0000C00F0200FC2600200C4B5B7D1B091B0103
:106B10000A4C637540230340002B07D0074BDB7CF6
:106B2000F024A3437033054CE37405E0034BDB7C96
:106B3000F024A343014CE37410BD0000FC260020A8
:106B400000B501287ED1FE4AD278F0239A437032F4
:106B5000FB4BDA701A46127912091201D21D1A7112
:106B60001A461279F0239A437032F54B1A711A467D
:106B7000527912091201D21D5A711A465279F02324
:106B80009A437032EE4B5A711A46D27912091201A9
:106B9000D21DDA711A46D279F0239A437032E84B4B
:106BA000DA711A46527A12091201D21D5A721A4625
:106BB000527AF0239A437032E14B5A721A46927A13
:106BC000F0239A437032DE4B9A721A469278F02381
:106BD0009A437032DA4B9A701A46D27A120912012D
:106BE000D21DDA721A46527812091201D21D5A7059
:106BF0001A46D27AF0239A437032D14BDA721A468F
:106C0000203AD27FF0239A437032CD4B203BDA7783
:106C1000CB4A127B12091201D21D20331A731A4675
:106C2000203A927F12091201D21D203B9A77C44A62
:106C3000127BF0239A437032C14B1A731A46203AE2
:106C4000127F00E0F2E1F0239A437032BC4B203B0C
:106C50001A77BB4A527B12091201D21D20335A7394
:106C60001A46203AD27E12091201D21D203BDA7652
:106C7000B44AD278F0239A437032B24BDA701A4693
:106C8000127B12091201D21D1A731A4612791209C7
:106C90001201D21D1A711A46927AF0239A43703269
:106CA000A84B9A721A461279F0239A437032A54B78
:106CB0001A711A46527912091201D21D5A711A46D6
:106CC000927912091201D21D9A711A46127A12098A
:106CD0001201D21D1A721A46127AF0239A437032A8
:106CE000984B1A721A46527A12091201D21D5A7220
:106CF000934A927912091201521C914B9A711A46C9
:106D00009279F0239A4310328D4B9A711A46127A77
:106D100012091201521C1A721A46127AF0239A436F
:106D20001032874B1A721A46927A12091201521CBB
:106D30009A721A46D27812091201521CDA701A4657
:106D4000927812091201521C9A701A465278F02356
:106D50009A4310327A4B5A701A461278F0239A43AB
:106D60001032774B1A701A46127812091201521C0F
:106D70001A701A46203AD27F12091201521C203B87
:106D8000DA771A46927FF0239A4310326C4B203BFD
:106D90009A771A46527FF0239A431032684B203B71
:106DA0005A771A46527F12091201521C5A771A4614
:106DB000127F12091201521C1A771A46D27EF02352
:106DC0009A4310325E4B203BDA761A46927EF023CD
:106DD0009A4310325A4B203B9A765A4A127BF02340
:106DE0009A431032574B1A731A46D27AF0239A43B9
:106DF0001032544BDA721A46D27A12091201521C1E
:106E0000DA721A46927A12091201521C9A721A46C2
:106E1000527AF0239A4310324A4B5A721A465279E8
:106E2000F0239A431032474B5A711A46D279F02315
:106E30009A431032434BDA710B0009F027F919F32A
:106E4000E9DFD5CBC1B7ADA3998F87786E645A506F
:106E5000463E362E261E160EF5003A4AD279F0230B
:106E60009A437032374BDA7100BF364A5279F023B9
:106E70009A437032334B5A7100BF324A527AF02330
:106E80009A4370322F4B5A7200BF2E4A927A1209DF
:106E90001201D21D2B4B9A7200BF2A4AD27A1209D4
:106EA0001201D21D274BDA7200BF264AD27AF02394
:106EB0009A437032234BDA7200BF224A127BF023CE
:106EC0009A4370321F4B1A7300BF1D4A203A927EBC
:106ED000F0239A4370321A4B203B9A7600BF184A2F
:106EE000203AD27EF0239A437032154B203BDA765B
:106EF00000BF134A203A127F12091201D21D104B13
:106F0000203B1A7700BF0E4A203A527F1209120125
:106F1000D21D0B4B203B5A7700BF094A203A527FC3
:106F2000F0239A437032064B203B5A7700BF044A45
:106F3000203A927FF0239A437032014B203B03E0CA
:106F4000682600203C2700209A7700BFDC4AD27FC9
:106F500012091201D21DDA4BDA7700BFD84A20326B
:106F6000127812091201D21DD54B20331A7000BFBE
:106F7000D34A20321278F0239A437032D04B203318
:106F80001A7000BFCE4A20325278F0239A437032F2
:106F9000CB4B20335A7000BFC94A20329278120975
:106FA0001201D21DC64B20339A7000BFC44A203252
:106FB000D27812091201D21DC14B2033DA7000BF02
:106FC000BF4A2032927A12091201D21DBC4B2033E3
:106FD0009A7200BFBA4A2032127AF0239A43703272
:106FE000B74B20331A7200BFB54A2032127A120909
:106FF0001201D21DB24B20331A7200BFB04A2032A8
:107000009279F0239A437032AD4B20339A7100BFCE
:10701000AB4A2032927912091201D21DA84B2033BB
:107020009A7100BF01E0FFE700BF47E1A44A2032A8
:10703000D278F0239A43A24B2033DA701A461279A1
:10704000120912011A711A461279F0239A439C4BC5
:1070500020331A711A465279120912015A711A46CE
:107060005279F0239A43964B20335A711A46D279BB
:1070700012091201DA711A46D279F0239A43904B21
:107080002033DA711A46527A120912015A721A46DC
:10709000527AF0239A438A4B20335A721A46927AD4
:1070A000F0239A43864B20339A721A469278F02343
:1070B0009A43834B20339A701A46D27A12091201EE
:1070C000DA721A465278120912015A701A46D27AA6
:1070D000F0239A437A4B2033DA72794AD27FF02335
:1070E0009A43774BDA771A462032127B1209120143
:1070F00020331A73724A927F12091201203B9A7749
:107100001A462032127BF0239A436D4B20331A73B8
:107110006B4A127FF0239A43694B1A771A46203242
:10712000527B1209120120335A73654AD27E12092A
:107130001201203BDA76634AD278F0239A43614BFE
:10714000DA701A46127B120912011A731A46127962
:10715000120912011A711A46927AF0239A43594B76
:107160009A721A461279F0239A43564B1A711A46AC
:107170005279120912015A711A46927912091201B2
:107180009A711A46127A120912011A721A46127A62
:10719000F0239A434B4B1A721A46527A1209120183
:1071A0005A72474A2032927912091201444B203315
:1071B0009A711A469279F0239A43414B20339A717F
:1071C0001A46127A120912011A721A46127AF0231A
:1071D0009A433B4B20331A721A46927A12091201D3
:1071E0009A721A46D27812091201DA701A46927807
:1071F000120912019A701A465278F0239A43304BC2
:1072000020335A701A461278F0239A432C4B2033BD
:107210001A701A461278120912011A70284AD27F7F
:1072200012091201203BDA771A46927FF0239A4323
:10723000234B9A771A46527FF0239A43204B5A7772
:107240001A46527F120912015A771A46127F120902
:1072500012011A771A46D27EF0239A43184BDA7637
:107260001A46927EF0239A43154B9A76154A127B62
:10727000F0239A43134B1A731A46D27AF0239A4397
:10728000104BDA721A46D27A12091201DA721A46D1
:10729000927A120912019A721A46527AF0239A438C
:1072A000084B5A721A465279F0239A43054B5A7189
:1072B0001A46D279F0239A43024BDA7100BD0000DE
:1072C000482600203C270020F7B582B00646174626
:1072D000002500200190002E7ED1F9F72DFC052815
:1072E0005FD1F9F749FD00280DD0FA484079F02127
:1072F00088437030F74948710846807800090001DA
:10730000C01D88700AE0F3484079F0218843F149B4
:10731000487108468078000900018870ED48C079FE
:1073200000090001EB49C871084680790009000195
:107330008871084640790009000148710846007AC2
:10734000F0218843E34908720846007A00090001E9
:1073500008720846C079F0218843DE49C8710846A2
:10736000C07800090001C87008468078F021884381
:10737000D849887008464078F0218843D54948703C
:107380000846407800090001487008460079000965
:10739000000108710846C078F0218843CD49C870C3
:1073A00029E2CC484079F02188437030C9494871BE
:1073B0000846807800090001C01D88700846C07921
:1073C00000090001C8710846807900090001887130
:1073D00008464079000900E034E0000148710846A1
:1073E000007AF0218843BB4908720846007A0009F8
:1073F000000108720846C079F0218843B549C87178
:107400000846C07800090001C87008468078F0215D
:107410008843B049887008464078F0218843AD49D8
:107420004870084640780009000148700846007915
:107430000009000108710846C078F0218843A54979
:10744000C870E8E3012E5FD1F9F796FC00280DD053
:10745000A0484079F021884370309E494871084621
:10746000807800090001C01D88700AE099484079C1
:10747000F021884397494871084680780009000147
:1074800088709448C079000900019249C871084683
:1074900080790009000188710846407900090001DF
:1074A00048710846007AF02188438A4908720846E4
:1074B000007A0009000108720846C079F02188436B
:1074C0008449C8710846C07800090001C8700846A0
:1074D0008078F02188437F49887008464078F02101
:1074E00088437C494870084640780009000148708C
:1074F000084600790009000108710846C078F021AB
:1075000088437449C87086E3022E7DD1F9F714FBD5
:1075100005287AD1F9F730FC002877D0012F76D1F1
:107520000A210398F0F70CFE0546F9F745FB002801
:1075300002D16948445D01E06848445DE007C00F3E
:10754000002807D06348C07900090001C01D6149C7
:10755000C87105E05F48C079000900015D49C87144
:1075600002202040002807D05A48807900090001F5
:10757000C01D5849887105E056488079000900010E
:107580005449887104202040002807D05148407990
:1075900000090001C01D4F49487105E04D48407980
:1075A000000900014B49487108202040002807D0FD
:1075B0004848007AF021884370304649087205E057
:1075C0004448007AF0218843424908721020204044
:1075D000002807D03F48007A00090001C01D3D493E
:1075E000087205E03B48007A000900013949087239
:1075F0002020204000280BD03648C079F021884355
:1076000070303449C87109E0AEE242E1F4E0A4E030
:107610003048C079F02188432E49C871402020406D
:10762000002807D02B484079F02188437030294941
:10763000487105E027484079F02188432549487181
:107640000A210398F0F77CFD0D462348445DE007CE
:10765000C00F002807D01F48C07800090001C01DD6
:107660001C49C87005E01B48C07800090001194991
:10767000C87002202040002807D016488078F021EA
:10768000884370301349887005E012488078F021F3
:1076900088431049887004202040002807D00D48F6
:1076A0004078F021884370300A49487005E0094865
:1076B0004078F0218843074948700820204000287E
:1076C0000ED00448407800090001C01D01494870EF
:1076D0000CE0000088260020C00F0200D30F02003B
:1076E000FE48407800090001FC4948701020204005
:1076F000002807D0F948007900090001C01DF749AA
:10770000087105E0F548007900090001F3490871A6
:1077100020202040002807D0F048C078F02188437E
:107720007030EE49C87005E0EC48C078F02188431D
:10773000EA49C87040202040002807D0E7488078F8
:1077400000090001C01DE549887064E2E3488078C3
:1077500000090001E14988705DE2E0484079F021CC
:1077600088437030DD49487108468078000900017F
:10777000C01D88700846C07900090001C87108461C
:1077800080790009000188710846407900090001EC
:1077900048710846007AF0218843D04908720846AB
:1077A000007A0009000108720846C079F021884378
:1077B000CA49C8710846C07800090001C870084667
:1077C0008078F0218843C549887008464078F021C8
:1077D0008843C24948700846407800090001487053
:1077E000084600790009000108710846C078F021B8
:1077F0008843BA49C8700EE2B8484079F0218843FE
:10780000B64948710846807800090001887008462A
:10781000C07900090001C87108468079000900019B
:107820008871084640790009000148710846007ACD
:10783000F0218843A94908720846007A000900012E
:1078400008720846C079F0218843A449C8710846E7
:10785000C07800090001C87008468078F02188438C
:107860009E49887008464078F02188439B494870BB
:107870000846407800090001487008460079000970
:10788000000108710846C078F02188439349C87008
:10789000C1E1012F73D10A210398F0F751FC05468D
:1078A000F9F78AF9002802D18D48445D01E08D483E
:1078B000445DE007C00F002807D08848C079000960
:1078C0000001C01D8549C87105E08448C0790009E0
:1078D00000018249C87102202040002807D07F485B
:1078E000807900090001C01D7C49887105E07B4852
:1078F000807900090001794988710420204000281E
:1079000007D07648407900090001C01D73494871CD
:1079100005E072484079000900017049487108206B
:107920002040002807D06D48007AF021884370304D
:107930006A49087205E06948007AF021884367497E
:10794000087210202040002807D06448007A0009FF
:107950000001C01D6149087205E06048007A000915
:1079600000015E49087220202040002808D05B48B2
:10797000C079F021884370305849C87106E09DE015
:107980005648C079F02188435449C87140202040AE
:10799000002807D051484079F021884370304F4982
:1079A000487105E04D484079F02188434B494871C2
:1079B0000A210398F0F7C4FB0D464948445DE007EF
:1079C000C00F002807D04548C07800090001C01D3D
:1079D0004249C87005E04148C078000900013F49AC
:1079E000C87002202040002807D03C488078F02151
:1079F000884370303949887005E038488078F02134
:107A000088433649887004202040002807D0334836
:107A10004078F021884370303049487005E02F48A5
:107A20004078F02188432D494870082020400028E4
:107A300007D02A48407800090001C01D2749487036
:107A400005E02648407800090001244948701020CC
:107A50002040002807D02148007900090001C01DFE
:107A60001E49087105E01D480079000900011B4905
:107A7000087120202040002807D01848C078F02145
:107A8000884370301549C87005E01448C078F0216B
:107A900088431249C87040202040002807D00F4872
:107AA000807800090001C01D0C498870B3E00B48C4
:107AB00080780009000109498870ACE007484079E6
:107AC000F0218843703005494871084680780009E4
:107AD0000001C01D88700846C07905E08826002096
:107AE000C00F0200D30F020000090001C871084650
:107AF0008079000900018871084640790009000179
:107B000048710846007AF0218843444908720846C3
:107B1000007A0009000108720846C079F021884304
:107B20003E49C8710846C07800090001C87008467F
:107B30008078F02188433949887008464078F021E0
:107B4000884336494870084640780009000148706B
:107B5000084600790009000108710846C078F02144
:107B600088432E49C87056E0032E54D12B48007923
:107B7000F021884370302949087108464079F02186
:107B80008843703025494871084680780009000113
:107B9000C01D88700846C07900090001C8710846F8
:107BA00080790009000188710846407900090001C8
:107BB00048710846007AF02188431849087208463F
:107BC000007A0009000108720846C079F021884354
:107BD0001249C8710846C07800090001C8700846FB
:107BE0008078F02188430D49887008464078F0215C
:107BF00088430A49487008464078000900014870E7
:107C0000084600790009000108710846C078F02193
:107C100088430249C87005B0F0BD000088260020E6
:107C200070B505460C46012D7ED1B348407D000954
:107C30000001C01DB04948750846007DF021884309
:107C40001030AD4908750846007D00090001401C50
:107C500008750846C07CF02188431030A649C874D6
:107C60000846807CF02188431030A3498874084678
:107C7000807C00090001401C8874F9F7D5F80228BF
:107C800003D0F9F7D1F801286ED19C48007801287B
:107C90006AD0F4F7BDFE9A49884265D3F9F76CF8CB
:107CA00000282FD09448007DF021884370309249FD
:107CB00008750846007D00090001C01D08750846CA
:107CC000C07CF021884370308B49C8740846807CA2
:107CD000F02188437030884988740846807C000908
:107CE0000001C01D88740846407DF0218843703033
:107CF000814948750846407CF021884370307E49B0
:107D00004874F8E07C48007DF021884310307A49BF
:107D100008750846007D00090001401C08750846EA
:107D2000C07CF021884300E0B8E010307249C8748C
:107D30000846807CF021884310306F4988740846DB
:107D4000807C00090001401C88740846407DF021B9
:107D500088431030684948750846407CF0218843C4
:107D6000103065494874C6E0F8F7D4FE002826D1E3
:107D7000F4F74EFE6249884221D3F8F7FDFF002850
:107D80000ED05D48407DF021884370305A494875D7
:107D90000846407CF02188437030574948741CE005
:107DA0005548407DF02188431030534948750846B6
:107DB000407CF021884310304F4948740DE04E4814
:107DC000407DF021884370304B4948750846407C1F
:107DD000F0218843703048494874F8F79BFE012829
:107DE0002AD146480078012826D0F4F711FE4449EC
:107DF000884221D34048407DF021884370303E497D
:107E000048750846407CF021884370303A494874F0
:107E1000F8F7B2FF002807D03748007DF0218843EB
:107E200070303549087566E03348007DF02188439D
:107E30001030314908755EE0230008F027F9062C60
:107E4000241C140C042D2C48807C00090001C01D4A
:107E50002949887400BF2848807CF021884370300D
:107E60002549887400BF2448C07CF02188437030C5
:107E70002149C87400BF2048007D00090001C01DD1
:107E80001D49087500BF1C48007DF02188437030F3
:107E90001949087500BF00E000BF2CE01648407D7E
:107EA000F0218843144948750846007DF021884335
:107EB000114908750846007D00090001087508464B
:107EC000C07CF02188430C49C8740846807CF021AE
:107ED0008843094988740846807C00090001887439
:107EE0000846407D0009000148750846407CF021A5
:107EF00088430149487470BD6826002001010020B4
:107F0000B80B000030B50246002901D1002000E086
:107F10000720130008F0BAF80F09141F2B3743503D
:107F20005D67727C88929FA9B500574B5B7EF024F9
:107F3000A3430401F0252C402343534C6376A1E076
:107F4000524B9B79F024A3430401F0252C4023439A
:107F50004E4CA37196E04D4B2033DB791B091B017E
:107F60000407240F2343494C2034E3718AE0464B35
:107F70002033DB7C1B091B010407240F2343424CE5
:107F80002034E3747EE0404B40331B781B091B0117
:107F90000407240F23433C4C4034237072E03A4BD7
:107FA0002033DB7FF024A3430401F0252C4023433E
:107FB000354C2034E37765E0334B20335B7BF02492
:107FC000A3430401F0252C4023432F4C203463733A
:107FD00058E02E4B9B791B091B010407240F2343F8
:107FE0002A4CA3714EE0294B9B7CF024A34304014F
:107FF000F0252C402343254CA37443E0234BDB7E28
:108000001B091B010407240F2343204CE37639E0AE
:108010001D4B2033DB7F1B091B010407240F234367
:10802000194C2034E3772DE0174B9B7E1B091B0175
:108030000407240F2343144CA37623E0134B20336F
:108040009B79F024A3430401F0252C4023430F4CDB
:108050002034A37116E00D4BDB7D1B091B010407C7
:10806000240F2343094CE3750CE0074B20335B7C62
:108070001B091B010407240F2343034C20346374A2
:1080800000E000BF00BF30BD482600201C270020B4
:10809000F7B582B00746154600260024FE48007852
:1080A000012804D0F4F7B4FCFC49884279D2FC489A
:1080B000407CF02188437030F94948740846807C40
:1080C00000090001C01D88740846007D00090001F8
:1080D000C01D08750846007DF02188437030F049C6
:1080E00008750846807CF02188437030EC4988741C
:1080F0000846C07C00090001C01DC8740846C07C49
:10810000F02188437030E649C8740846407C000975
:108110000001C01D48740846407D00090001C01DD3
:1081200048750846407DF02188437030DC49487529
:108130000846007CF02188437030D949087408460D
:10814000007C00090001C01D08740846C07BF021B6
:1081500088437030D249C873FF220A210020FBF700
:10816000E7F9FF2213210020FBF7E2F9FF2211219A
:108170000020FBF7DDF9FF2212210020FBF7D8F9E0
:10818000FF220E210020FBF7D3F9FF220F21002050
:10819000FBF7CEF9FF2210210020FBF7C9F9F4E329
:1081A000FFE7039836283DD019DC08287ED007DC8D
:1081B000801E030007F06AFF0635A8FCFBFAF97E73
:1081C000102874D006DC092872D00D2871D00E2832
:1081D00070D1FDE333286ED03428F9D170E13F2807
:1081E0006AD00FDC3738082864D243007B449B8870
:1081F0005B009F448A009702FF025F005F006503F7
:10820000CB0318004E287BD006DC402879D04128CB
:1082100078D04D28DCD1BBE14F2874D05028D7D17D
:108220004FE100BF00BF9E48407CF02188439C493D
:1082300048740846807C0009000188740846007D67
:1082400000090001C01D08750846007DF021884323
:108250007030934908750846807CF0218843904926
:1082600088740846C07C00090001C01DC874084617
:10827000C07CF02188438A49C8740846407C0009C4
:10828000000148740846407D000900014875084611
:10829000407DF0218843824948750846007CF021E2
:1082A00088437F4908740846007C06E0A1E2FDE3AC
:1082B00037E2D2E3FBE394E028E000090001087410
:1082C0000846C07BF02188437549C873FF220A2104
:1082D0000020FBF72DF9FF2213210020FBF728F9DE
:1082E00000220E211046FBF723F900220F21104631
:1082F000FBF71EF9002210211046FBF719F977E26F
:10830000ABE110E2DDE26DE000BF00BF6448407CFD
:10831000F0218843624948740846807C00090001C6
:1083200088740846007D00090001C01D08750846D4
:10833000007DF02188437030594908750846807CDB
:10834000F0218843564988740846C07C0009000122
:10835000C8740846C07CF02188435149C874084657
:10836000407C0009000148740846407D0009000176
:10837000C01D48750846407DF0218843484948752E
:108380000846007CF0218843454908740846007C73
:108390000009000108740846C07BF0218843404969
:1083A000C873FF220A21002003E055E1EFE086E0D8
:1083B00016E0FBF7BDF8FF2213210020FBF7B8F809
:1083C00000220E211046FBF7B3F800220F211046C1
:1083D000FBF7AEF8002210211046FBF7A9F88EE754
:1083E00000BF00BF2E48407CF02188432C494874D0
:1083F0000846807C00090001C01D88740846007D85
:1084000000090001C01D08750846007DF021884361
:108410007030234908750846807CF021884370300D
:108420001F4988740846C07C00090001C8740846CA
:10843000C07CF02188431A49C8740846407C000972
:10844000000148740846407D00090001487508464F
:10845000407DF0218843124948750846007CF02190
:1084600088430F4908740846007C0009000108741D
:108470000846C07BF02188430949C873FF220A21BE
:108480000020FBF755F8FF2213210020FBF750F8DE
:1084900000220E21104605E001010020B80B00006B
:1084A00088260020FBF744F800220F211046FBF736
:1084B0003FF8002210211046FBF73AF81FE700BFF3
:1084C00000BFFE48407CF0218843FC4948740846C0
:1084D000807C00090001C01D88740846007D0009E9
:1084E0000001C01D08750846007DF02188437030EA
:1084F000F24908750846807CF0218843EF4988746A
:108500000846C07C00090001C8740846C07CF02100
:108510008843EA49C8740846407C00090001C01D30
:1085200048740846407D0009000148750846407DB2
:10853000F0218843E14948750846007CF0218843D2
:10854000DE4908740846007C0009000108740846EA
:10855000C07BF0218843D949C873FF220A2100203B
:10856000FAF7E6FFFF2213210020FAF7E1FF0022CD
:108570000E211046FAF7DCFF00220F211046FAF711
:10858000D7FF002210211046FAF7D2FFF6E300BF12
:10859000CA48407CF0218843C84948740846807C1A
:1085A0000009000188740846007D00090001087573
:1085B0000846007DF02188437030C04908750846A0
:1085C000807CF0218843BD4988740846C07C00093E
:1085D0000001C8740846C07CF02188437030B74958
:1085E000C8740846407C0009000148740846407D74
:1085F0000009000148750846407DF0218843AF49D5
:1086000048750846007CF0218843AC490874084648
:10861000007C0009000108740846C07BF0218843F3
:10862000A649C873FF220A210020FAF781FFFF2222
:1086300013210020FAF77CFF00220E211046FAF7E2
:1086400077FF00220F211046FAF772FF0022102157
:108650001046FAF76DFF91E300BF9848407CF02187
:108660008843964948740846807C00090001887454
:108670000846007D0009000108750846007DF021CC
:10868000884370308D4908750846807CF021884306
:108690008A4988740846C07C00090001C8740846ED
:1086A000C07CF02188438549C8740846407C000995
:1086B000000148740846407D0009000148750846DD
:1086C000407DF021884370307C4948750846007C25
:1086D000F0218843794908740846007C00090001AC
:1086E00008740846C07BF02188437449C873FF2290
:1086F0000A210020FAF71CFFFF2213210020FAF7BD
:1087000017FF00220E211046FAF712FF00220F2158
:108710001046FAF70DFF002210211046FAF708FF65
:108720002CE300BF00BF6548407CF02188437030D7
:10873000624948740846807C00090001C01D8874A5
:108740000846007D00090001C01D08750846007D2F
:10875000F02188437030594908750846807CF02123
:108760008843564988740846C07C00090001C874D3
:108770000846C07CF02188435049C8740846407CB4
:108780000009000148740846407D00090001487551
:108790000846407DF0218843484948750846007CDA
:1087A000F0218843454908740846007C000900010F
:1087B00008740846C07BF02188434049C873FF22F3
:1087C0000A210020FAF7B4FEFF2213210020FAF755
:1087D000AFFE00220E211046FAF7AAFE00220F215A
:1087E0001046FAF7A5FE002210211046FAF7A0FE67
:1087F000C4E200BF3148407CF02188432F494874CF
:108800000846807C0009000188740846007D000944
:10881000000108750846007DF02188437030274923
:1088200008750846807CF0218843244988740846EE
:10883000C07C00090001C8740846C07CF021884350
:1088400070301E49C8740846407C00090001487415
:108850000846407D0009000148750846407DF0212A
:108860008843164948750846007CF021884313491F
:1088700008740846007C0009000108740846C07BA3
:10888000F02188430D49C873FF220A210020FAF71E
:108890004FFEFF2213210020FAF74AFE00220E218C
:1088A0001046FAF745FE00220F211046FAF740FE67
:1088B000002210211046FAF73BFE5FE288260020D6
:1088C00000BFFC48407CF0218843FA4948740846C0
:1088D000807C0009000188740846007D00090001C1
:1088E00008750846007DF02188437030F14908750D
:1088F0000846807CF0218843EE4988740846C07C95
:1089000000090001C8740846C07CF0218843E94989
:10891000C8740846407C0009000148740846407D40
:108920000009000148750846407DF02188437030F9
:10893000E04948750846007CF0218843DD49087409
:108940000846007C0009000108740846C07BF0213D
:108950008843D849C873FF220A210020FAF7E8FDAE
:10896000FF2213210020FAF7E3FD00220E2110461A
:10897000FAF7DEFD00220F211046FAF7D9FD00229A
:1089800010211046FAF7D4FDF8E1F8E1C948407C1F
:10899000F02188437030C74948740846807C00093C
:1089A0000001C01D88740846007D00090001C01D3B
:1089B00008750846007DF0218843BE4908750846C1
:1089C000807CF0218843BB4988740846C07C00E065
:1089D000A9E000090001C8740846C07CF021884362
:1089E000B449C8740846407C000900014874084630
:1089F000407D0009000148750846407DF02188430C
:108A0000AC4948750846007CF0218843A9490874A0
:108A10000846007C0009000108740846C07BF0216C
:108A20008843A449C873FF220A210020FAF780FD79
:108A3000FF2213210020FAF77BFD00220E211046B1
:108A4000FAF776FD00220F211046FAF771FD002299
:108A500010211046FAF76CFD90E19648407CF02119
:108A60008843944948740846807C00090001887452
:108A70000846007D0009000108750846007DF021C8
:108A800088438C4908750846807CF02188438949D1
:108A900088740846C07C00090001C8740846C07C80
:108AA000F02188438349C874084601E09EE003E151
:108AB000407C0009000148740846407D000900011F
:108AC00048750846407DF02188437A494875084634
:108AD000007CF0218843774908740846007C00092F
:108AE000000108740846C07BF0218843703071494A
:108AF000C87300220A211046FAF71AFD002213213A
:108B00001046FAF715FDFF220E210020FAF710FD9E
:108B100000220F211046FAF70BFD0022102110460B
:108B2000FAF706FD2AE16348407CF0218843614959
:108B300048740846807C0009000188740846007D5E
:108B40000009000108750846007DF0218843594955
:108B500008750846807CF021884356498874084689
:108B6000C07C00090001C8740846C07CF02188431D
:108B70005049C8740846407C000900014874084602
:108B8000407D0009000148750846407DF02188437A
:108B9000484948750846007CF021884345490874D7
:108BA0000846007C00090001C01D08740846C07B0F
:108BB000F02188433F49C87300220A211046FAF782
:108BC000B7FC002213211046FAF7B2FC00220E2156
:108BD0001046FAF7ADFCFF220F210020FAF7A8FC9F
:108BE000002210211046FAF7A3FCC7E03148407C70
:108BF000F02188432F4948740846807C0009000111
:108C000088740846007D0009000108750846007D4B
:108C1000F0218843274908750846807CF021884365
:108C2000244988740846C07C00090001C8740846BD
:108C3000C07CF02188431F49C8740846407C000965
:108C4000000148740846407D000900014875084647
:108C5000407DF0218843174948750846007CF02183
:108C600088437030134908740846007C00090001ED
:108C700008740846C07BF02188430E49C87300225F
:108C80000A211046FAF754FC002213211046FAF785
:108C90004FFC00220E211046FAF74AFC00220F2159
:108CA0001046FAF745FCFF2210210020FAF740FC9D
:108CB00064E0000088260020FB48407CF0218843C7
:108CC000F94948740846807C000900018874084608
:108CD000007D0009000108750846007DF0218843E9
:108CE000F14908750846807CF0218843EE49887474
:108CF0000846C07C00090001C8740846C07CF02109
:108D00008843E949C8740846407C0009000148745A
:108D10000846407D0009000148750846407DF02165
:108D20008843E14948750846007CF0218843DE49C4
:108D300008740846007C0009000108740846C07BDE
:108D4000F0218843D849C87300220A211046FAF757
:108D5000EFFB002213211046FAF7EAFB00220E2156
:108D60001046FAF7E5FB00220F211046FAF7E0FB68
:108D7000002210211046FAF7DBFB00BF00BF002FD6
:108D800003D0CA48007A002804D1F3F741FEC8494D
:108D9000884272D2FF2211210020FAF7C9FBFF227C
:108DA00012210020FAF7C4FBC2480078012804D041
:108DB000F3F72EFEBE49884216D2BF48807BF021D1
:108DC00088437030BC498873084640300078F021F1
:108DD00088437030B849403108700846007800096F
:108DE0000001C01D08702DE07D20C000854214D216
:108DF000B148807BF0218843AF49887308464030F2
:108E00000078F02188437030AB4940310870084643
:108E1000007800090001087014E0A748807BF02169
:108E200088437030A4498873084640300078F021A8
:108E30008843A149403108700846007800090001C4
:108E4000C01D08707D20C000854205D2014628461D
:108E5000EFF776F9064604E098492846EFF770F9EF
:108E6000064694480078012804D0F3F7D1FD9049D4
:108E7000884203D29248845D02E0A0E29148845D7A
:108E8000E007C00F002809D08B484030C0780009A7
:108E90000001C01D88494031C87007E08648403055
:108EA000C0780009000184494031C8700220204088
:108EB000002807D08048C07900090001C01D7E4904
:108EC000C87105E07C48C079000900017A49C87181
:108ED00004202040002807D077488079000900014D
:108EE000C01D7549887105E073488079000900014B
:108EF0007149887108202040002807D06E484079C9
:108F0000F021884370306C49487105E06A48407927
:108F1000F02188436849487110202040002807D07C
:108F20006548407900090001C01D6349487105E0AA
:108F300061484079000900015F49487120202040C4
:108F4000002807D05C480079F021884370305A49E6
:108F5000087105E058480079F021884356490871A6
:108F600040202040002807D053488079F0218843D2
:108F700070305149887105E04F488079F02188436D
:108F80004D4988717D20C000854213D26421284656
:108F9000EFF7D6F8064647480078012804D0F3F7E3
:108FA00037FD4349884202D24548845D23E0454865
:108FB000845D20E0642128463230EFF7C1F87D213E
:108FC000C9000090EFF7BCF8019164210198EFF718
:108FD000B7F806463C48854208D236480078012852
:108FE00004D0F3F715FD3249884202D23448845D3B
:108FF00001E03448845DE007C00F002809D02E4806
:1090000040308078F021884370302B49403188709F
:1090100007E0294840308078F021884326494031D4
:10902000887002202040002807D02348807A000959
:109030000001C01D2049887205E01F48807A0009A0
:1090400000011D49887204202040002807D01A48DA
:10905000407A00090001C01D1749487205E0164812
:10906000407A000900011449487208202040002875
:1090700007D01148007AF021884370300E490872F9
:1090800005E00D48007AF02188430B490872102052
:10909000204000281AD00848007A00090001C01DAD
:1090A0000549087218E0000088260020580A0020B0
:1090B000B80B000001010020FC260020A086010062
:1090C000C00F0200D30F020010270000FE48007AF4
:1090D00000090001FC49087220202040002807D028
:1090E000F948C079F02188437030F749C87105E02C
:1090F000F548C079F0218843F349C87140202040E9
:10910000002807D0F048407AF02188437030EE49BB
:10911000487205E0EC48407AF0218843EA494872F9
:109120007D20C000854219D20A212846EFF708F8B1
:109130000A210190EFF704F80E460A2D08D2E34801
:109140000078012804D0F3F763FCE149884202D299
:10915000E048845D12E0E048845D0FE06421284629
:109160003230EEF7EDFF0A210090EEF7E9FF0A2119
:109170000190EEF7E5FF0E46D6498C5DE007C00F83
:10918000002809D0D0484030807800090001C01D77
:10919000CD494031887007E0CB48403080780009E5
:1091A0000001C9494031887002202040002807D0C2
:1091B000C548807B00090001C01DC349887305E0D4
:1091C000C148807B00090001BF498873042020400A
:1091D000002807D0BC48407B00090001C01DBA49E7
:1091E000487305E0B848407B00090001B649487360
:1091F00008202040002807D0B348007BF021884396
:109200007030B149087305E0AF48007BF021884316
:10921000AD49087310202040002807D0AA48C07A22
:1092200000090001C01DA849C87205E0A648C07A1F
:1092300000090001A449C87220202040002807D05E
:10924000A148807AF021884370309F49887205E0F8
:109250009D48807AF02188439B49887240202040B5
:10926000002807D09848407BF02188437030964909
:10927000487305E09448407BF02188439249487345
:109280007D20C000854207D20A212846EEF758FF0C
:109290000E469048845D0BE0642128463230EEF79C
:1092A0004FFF0A210190EEF74BFF0E4689498C5D76
:1092B000E007C00F002809D0834840304078F021F3
:1092C0008843703080494031487007E07E48403024
:1092D0004078F02188437C4940314870022020408A
:1092E000002809D078484030407800090001C01DAE
:1092F00075494031487007E07348403040780009B4
:10930000000171494031487004202040002807D0F6
:109310006D48007CF021884370306B49087405E08B
:109320006948007CF0218843674908740820204080
:10933000002807D06448007C00090001C01D624974
:10934000087405E06048007C000900015E4908746B
:1093500010202040002807D05B48C07BF0218843C4
:1093600070305949C87305E05748C07BF0218843E5
:109370005549C87320202040002807D05248C07BA0
:1093800000090001C01D5049C87305E04E48C07B6C
:10939000000900014C49C87340202040002807D034
:1093A0004948407C00090001C01D47494874ECE071
:1093B0004548407C0009000143494874E5E000222B
:1093C0000A211046FAF7B4F8002213211046FAF7E2
:1093D000AFF8002211211046FAF7AAF80022122154
:1093E0001046FAF7A5F800220E211046FAF7A0F869
:1093F00000220F211046FAF79BF800221021104698
:10940000FAF796F830484030C078000900012E493C
:109410004031C8702C48C079000900014039C8713A
:109420000846807900090001887108464079F021DA
:109430008843254948710846407900090001487170
:1094400008460079F02188431F4908710846807951
:10945000F02188431C498871084640308078F0210B
:1094600088431949403188701748807A0009000103
:10947000403988720846407A00090001487208465F
:10948000007AF0218843104908720846007A0009E2
:10949000000108720846C079F02188430A49C87162
:1094A0000846407AF0218843074948720846403010
:1094B000807800090001403188700348807B0009F2
:1094C00000014039887309E0FC26002001010020DA
:1094D000B80B0000C00F0200D30F02000846407B0B
:1094E0000009000148730846007BF02188432849A1
:1094F00008730846C07A00090001C8720846807ADD
:10950000F0218843224988720846407BF021884335
:109510001F494873084640304078F02188431C4971
:1095200040314870084640780009000148701848EA
:10953000007CF0218843164908740846007C000925
:10954000000108740846C07BF02188431049C873A5
:109550000846C07B00090001C8730846407C00092A
:10956000000148740846807BF021884308498873CD
:10957000084640300078F0218843054940310870A2
:109580000846007800090001087005B0F0BD000031
:10959000FC260020F7B582B007460E460121FF20C9
:1095A0000830FBF7FBFF0121FC48FBF7F7FFFC4805
:1095B000007801287ED0F3F72BFAFA49884279D354
:1095C000F7F7BAFA032843D1F7F7B0FA002803D027
:1095D000F7F7ACFA01283BD1002F1CD1F7F7CCFBF1
:1095E00000280CD0F048407CF0218843EE494874B4
:1095F0000846807C00090001C01D8874EEE0EA483E
:10960000407CF0218843E84948740846807C000982
:1096100000018874E2E0F7F7AFFB00280CD0E248C5
:10962000407CF02188437030DF4948740846807CD4
:10963000000900018874D1E0DB48407CF0218843B8
:10964000D94948740846807C000900018874C5E047
:10965000F7F76CFA002803D0F7F768FA012865D10C
:10966000002F0CD1D048407CF0218843CE4948746B
:109670000846807C00090001C01D88740BE0CA48C0
:10968000407CF02188437030C74948740846807C8C
:10969000000900018874F7F749FA002821D1C2486F
:1096A0002030C078F02188437030BF492031C87025
:1096B000BD4800E064E0807D000900012039887524
:1096C0000846807DF0218843B7498875FF22232111
:1096D0000020F9F72DFF002222211046F9F728FF7C
:1096E0007CE0F7F723FA012878D1AF482030C07822
:1096F000F0218843AC492031C870AB48807D000917
:109700000001C01D203988750846807DF0218843FE
:109710007030A5498875002223211046F9F708FF0B
:10972000FF2222210020F9F703FF57E09E48407CEA
:10973000F02188439C4948740846807C0009000158
:10974000887408462030C078F0218843964920313B
:10975000C8709548807D0009000120398875084649
:10976000807DF0218843904988750022232110468E
:10977000F9F7DEFE002222211046F9F7D9FE2DE08E
:109780008948407CF02188437030874948740846F6
:10979000807C00090001C01D887408462030C07814
:1097A000F0218843703080492031C8707E48807D28
:1097B00000090001C01D203988750846807DF02110
:1097C0008843703078498875FF2223210020F9F7FB
:1097D000AFFEFF2222210020F9F7AAFEF7F7A6F933
:1097E000002808D06E480078012804D0F3F710F95B
:1097F0006C49884276D26D48864209D96A48203041
:109800004079F0218843703067492031487107E082
:10981000654820304079F021884363492031487100
:1098200063493046EEF78CFC0A210190EEF788FC84
:109830000D465E48401C864202D35E48445D01E00E
:109840005D48445DE007C00F002809D0564820302D
:10985000C07800090001C01D53492031C87007E0DD
:1098600051482030C078000900014F492031C870AC
:1098700002202040002809D04B4820308078F02179
:109880008843703048492031887007E046482030CE
:109890008078F0218843444920318870042020409A
:1098A000002809D0404820304078F02188437030AB
:1098B0003D492031487007E03B4820304078F02196
:1098C00088433949203148700820204000280AD0B8
:1098D00035482030407900090001C01D324920314F
:1098E000487108E0A1E230482030407900090001C9
:1098F0002D492031487110202040002809D02A48E5
:1099000020300079F02188437030274920310871D8
:1099100007E0254820300079F02188432249203192
:10992000087120202040002809D01F4820300079ED
:1099300000090001C01D1C492031087107E01A48C8
:1099400020300079000900011749203108714020BA
:109950002040002809D014482030807800090001F8
:10996000C01D11492031887007E00F4820308078F1
:10997000000900010C49203188707D21C900304662
:10998000EEF7DEFB0A210190EEF7DAFB0D46084800
:10999000864213D30748445D12E00000050500002D
:1099A00001010020B80B0000FC2600209F8601006A
:1099B00010270000C00F0200D30F0200F948445DD9
:1099C000E007C00F002807D0F748C07FF021884388
:1099D0007030F549C87705E0F348C07FF02188432F
:1099E000F149C87702202040002807D0EE48C07F08
:1099F00000090001C01DEC49C87705E0EA48C07FB6
:109A000000090001E849C87704202040002807D059
:109A1000E548807F00090001C01DE349887705E023
:109A2000E148807F00090001DF4988770820204055
:109A3000002809D0DC482030407800090001C01D12
:109A4000D9492031487007E0D748203040780009D4
:109A50000001D5492031487010202040002809D04D
:109A6000D14820300078F02188437030CE49203131
:109A7000087007E0CC4820300078F0218843CA49BC
:109A80002031087020202040002809D0C64820300E
:109A9000007800090001C01DC3492031087007E0AB
:109AA000C1482030007800090001BF49203108700A
:109AB00040202040002807D0BB48807FF021884309
:109AC0007030B949887705E0B748807FF021884336
:109AD000B549887764213046EEF732FB0A210190C0
:109AE000EEF72EFB0D467D20C000864202D3AF4824
:109AF000445D01E0AB48445DE007C00F002807D09B
:109B0000A948007F00090001C01DA749087705E0AA
:109B1000A548007F00090001A349087702202040E2
:109B2000002807D0A048C07EF021884370309E49AD
:109B3000C87605E09C48C07EF02188439A49C876E3
:109B400004202040002807D09748807EF0218843D9
:109B500070309549887605E09348807EF0218843EF
:109B60009149887608202040002807D08E48407F01
:109B7000F021884370308C49487705E08A48407F5F
:109B8000F02188438849487710202040002807D0DA
